:020000020000FC
:020000000C945E
:1000020093040C9400000C9400000C9400000C94D7
:1000120000000C9400000C9400000C9400000C945E
:1000220000000C9400000C9400000C9400000C944E
:10003200CD800C9400000C9400000C9400000C94F1
:1000420098350C9400000C9400000C9400000C9461
:1000520000000C94B2BA0C94E0BA0C9400000C9418
:1000620000000C9430360C9400000C9400000C94A8
:1000720000000C9400000C9400000C9400000C94FE
:1000820000000C9400000C9400000C9400000C94EE
:100092000000000000000102030400060705010041
:1000A20006FF050402FF09080CFF0AFF0F0E0106F6
:1000B2000807050204030C0B100A090D0F0E0406B3
:1000C2000802030107050C10090F0D0B0E0A0101AE
:1000D200010101010101010101010101010101FF10
:1000E20002FF04FFFFFF03FF05FF06FF00FF436F50
:1000F2004465496E466F00C9020D0000000FAA5503
:100102008A61707220333020323032362031303AF8
:1001120030383A33320000670101656400000001A3
:100122000101020202030303040404050505060695
:10013200060707074142434142434142434142438A
:100142004142434142434142434142430000000095
:10015200EF006A02900800000000000000000000AA
:100162000000000000000000000000006400230105
:10017200C602D504820F000000000000000000004B
:10018200000000000000000000000000F000F0008D
:100192005402D203F6090000000000000000000033
:1001A2000000000000000000000000002A03C80355
:1001B2002105E3064D1000000000000000000000D1
:1001C2000000000000000000000000000E00020815
:1001D200040A0C000000F000000043414E72783A1D
:1001E20020253033580A000043414E696E70757401
:1001F200436E743D25752121210A0043414E2D2570
:10020200753A20300A0043414E2D25753A20310AB5
:100212000043414E2D25753A2025750A0043414E73
:100222002025750044656C61792074696D657220C2
:1002320025750000466163746F7279446566617565
:100242006C740A00485038343433004572724C6F73
:1002520067506F733D25752C204E6F3D25750A0042
:100262004572723A2025752025750A002575204FA2
:1002720066660A002575204F6E0A00466C61736837
:100282002074696D65722025750048503834343306
:100292000043666753756D3D253034580A0020557A
:1002A2007064617465640A004850383434332076CF
:1002B20065722E2025752E25752E2575206170728A
:1002C20020333020323032362031303A30383A332F
:1002D200320A0053657269616C3A2025750A005929
:1002E2006561723A203230253032752C20576565AF
:1002F2006B3A2025750A004857207665723A202508
:10030200632E25632C204F7074696F6E733A20251B
:100312003032580A00436C6F636B3A202530386CD8
:10032200580A0043666743686B53756D3A2025305F
:10033200345820004F4B0A0020457272210A0043B4
:1003420066675665724572723A20257520282575B2
:1003520029210A004545507665724572723A202578
:10036200752028257529210A00526573746F7265FC
:10037200436E743D25752025752025750A0044615C
:1003820074614572723D2530325820253032580A48
:10039200004850383434330A00004144436D696EDA
:1003A2004572726F725B25755D3D25752121210AAB
:1003B2000000496E707574733A002025753D2575ED
:1003C20000496E2D313A2025750A00496E2D323AC8
:1003D2002025750A00496E2D333A2025750A0049F9
:1003E2006E2D343A2025750A00496E2D25753A2066
:1003F20025750A00496E412D2575204F66663A2003
:1004020025755B6D565D0A00496E412D2575204F9D
:100412006E3A2025755B6D565D0A005377697463E9
:100422006820257500416E616C6F6720332E25753B
:1004320000416E616C6F6720342E257500004B659C
:10044200795061643D00426C696E6B3A25303258D6
:1004520020253032580A004772617968696C6C2035
:1004620043414E6F70656E0A004772617968696C2C
:100472006C204A313333390A004850393634320A53
:10048200004E6F6E650A00004B65795061642E4321
:100492006F6E6E2025750A004B65795061642E449B
:1004A20069736F6E6E6E2025750A00004F75745069
:1004B20075736850756C6C3A2025750A004F757417
:1004C20048696768536964654F6E6C793A2025758F
:1004D2000A0043202532753A202534750043616CA9
:1004E20069627261746520004F4B0A006F75747007
:1004F2007574202575206661696C65642121210A65
:10050200002532753A2025352E32665B415D0A00A0
:100512002532753A204E6F20666565646261636BB1
:100522002C204F75742D25750A002532753A204608
:100532006565646261636B206572726F722C204F15
:1005420075742D25750A004F757470757420746565
:10055200737400426174742063616C696220203A92
:1005620020257500416E616C6F672063616C696262
:100572003A20333D25752C20343D25750043616CAE
:100582006962726174696F6E4D61736B3A202558AE
:100592000A0020202532753A2534752C2536752C13
:1005A2002536752C2536752C2536750042617474F6
:1005B200657279206661696C65642121210A0041B6
:1005C2006E616C6F67206661696C65642121210A26
:1005D20000206E6F7420636F6D706C6574656421AA
:1005E20021210A004F75745273744572725B25752E
:1005F2005D0A004F75742D25753A204F6E0A004F23
:1006020075742D25753A205325752D3E25752C20A0
:100612004F6E3D25752C205365743D25750A0041AA
:1006220044433A002025753D25750020204261741F
:10063200743D2575004C6F77426174744F66663D58
:100642002025750A004C6F77426174744F6E3D200D
:10065200257530300A0042617474657279536B6992
:100662007046423A20252E31665B565D0A00426191
:1006720074746572794642204F4B3A20252E3166BA
:100682005B565D0A002020416E612D333D202575A9
:10069200002020416E612D343D202575004F757478
:1006A2002D25753A2025750A004F75742025752071
:1006B200474E442D31210A004F757420257520477D
:1006C2004E442D32210A004F7574202575206C6925
:1006D2006D6974210A004F7574412D25753A2053B6
:1006E20025752D3E25752C204F6E3D25752C2053EA
:1006F20065743D25750A004F7574707574733A0AF6
:10070200002534753A2046423D2575204144433D3B
:1007120025752025755B6D415D0A00526573657410
:100722004572726F720A004F757470757420257568
:10073200004F75742D25753A205325752C204F6E68
:100742003D25752025632C202575305B6D415D0AA2
:1007520000004F75747075742067726F7570202574
:100762007500506F776572446F776E0A0057616B40
:100772006555703A2025750A00004F7574412D2584
:10078200753A205325752D3E25752C204F6E3D253B
:10079200750A000043616C69622E20737461727481
:1007A2002025755B416D705D0A0054657374206F7E
:1007B20075740A0043616C69622E20626174740A66
:1007C2000043616C696220616E6128352C305620CD
:1007D2007265662E290A0043616C69623F006330CC
:1007E20000633100633300633600633230006362BA
:1007F20000636100746573746F7574005061737384
:10080200776F72643F0050573A20272573270A00FA
:1008120050573A204E6F6E650A00505772657365E5
:10082200740050577265736574202D204F4B0A0077
:100832004144433F00496E7075743F004C6F6164E0
:100842003F0048507374617475733F005252657370
:10085200746F7265005252204F4B0A0052657365E5
:1008620074005365744F75742025753D2025750AF3
:10087200005265736574206572726F720A004F7060
:1008820074696F6E3A20253032580A0052657365DA
:10089200740A00005365712025633A20004F666692
:1008A2000A0025630A0053657175656E636520252C
:1008B200750020204F4B0A0020204661696C656458
:1008C2002121210A000056696E2D25753A202575D1
:1008D2000A005669727475616C20257500005769AB
:1008E2007065723A205325752D3E5325750A000016
:1008F20001002D4E414E00494E4600002D4E414E04
:10090200000001000200D60100000700BC034602FD
:1009120000000700C3038C0200000100B90DF208B9
:1009220000000000F894EE27EFBBF1E0F5BFE5BF51
:10093200E0937400E09375008DE0A2E0BB27ED9395
:100942008A95E9F780EF9FE0A0E0B1E0ED9301978F
:10095200E9F7E4E0F9E0D0E0DBBF879197910097F7
:1009620081F0A791B79107901790C791D791BF01D6
:10097200DBB7F001CBBF07900D920197E1F7FB01C6
:10098200EBCFE0E0EEBBEFEEEDBFE0E1EEBFCCEB94
:10099200D3E00C9448330E945CCCAD014093D20367
:1009A2005093D303A5E2B1E00E9453CEE07111F05F
:1009B200E1E001C0E0E0AFECB3E0E170EE0F0E2E3B
:1009C200EC91ED7FE029EC93A6E7B2E00E9453CED2
:1009D200E093D103A7E7B2E00E9453CEE0935C0418
:1009E200A091D103A13010F0AD3008F004C0E09125
:1009F200CF03E46003C0E091CF03EB7FE093CF032A
:100A0200E1E0E093D800FA01E436A0E0FA0741F40D
:100A1200E2E1E093E200ECE0E093E300E7E335C0DB
:100A2200ED37A0E0FA0741F4EEE0E093E200ECE0FB
:100A3200E093E300E7E329C0E83CA0E0FA0741F4D1
:100A4200E8E0E093E200ECE0E093E300E7E31DC0BE
:100A5200EA3FA0E0FA0741F4E6E0E093E200ECE0CE
:100A6200E093E300E7E311C0E43FA1E0FA0711F4E9
:100A7200E6E005C0E83EA3E0FA0749F4E2E0E093CD
:100A8200E200E4E0E093E300E3E1E093E40010E15C
:100A9200103F88F41093ED002EEE30E0E8EFF0E026
:100AA2002E173F0730F4D901E0E0EC932F5F3F4F60
:100AB200F5CF105FEDCFE091D800E260E093D8006F
:100AC20010E4103FA0F41093ED002EEE30E0E8EFBA
:100AD200F0E02E173F0730F4D901E0E0EC932F5FEE
:100AE2003F4FF5CFE8E8E093EF00105FEACF0E94B6
:100AF20063CC2696089564970E945CCCE091D00363
:100B0200E03009F414C2E17089F0E0E0E093ED0016
:100B1200E091EE00E17551F0E091D003EE7FE093B9
:100B2200D003E0E0E093EE00E093EF00E091D00329
:100B3200E27089F0E0E1E093ED00E091EE00E17512
:100B420051F0E091D003ED7FE093D003E0E0E09339
:100B5200EE00E093EF00E091D003E47089F0E0E270
:100B6200E093ED00E091EE00E17551F0E091D003E9
:100B7200EB7FE093D003E0E0E093EE00E093EF0040
:100B8200E091D003E87089F0E0E3E093ED00E091BA
:100B9200EE00E17551F0E091D003E77FE093D003DE
:100BA200E0E0E093EE00E093EF00A091D003AF30DD
:100BB20009F4BDC1A0915604E0915704EA1709F463
:100BC200B6C1A4EDB3E0E0915604F0E0BD01ADE0A2
:100BD200B0E00E9411CDDB01AE0FBF1FEC91E071BE
:100BE200B1F041E0A4EDB3E0E0915604F0E0BD01C4
:100BF200ADE0B0E00E9411CDDB01AE0FBF1F119638
:100C02000E94CECDEB8BFC8B6D8B7E8B13C040E0B4
:100C1200A4EDB3E0E0915604F0E0BD01ADE0B0E038
:100C22000E9411CDDB01AE0FBF1F1196ED91FD9118
:100C3200EF8BF88FA4EDB3E0E0915604F0E0BD0134
:100C4200ADE0B0E00E9411CDDB01AE0FBF1FEC9111
:100C5200EF700E2F098F403019F0E98DE061E98FB6
:100C6200E091D003E17009F051C0E0E0E093ED00C3
:100C7200E98DE093EF004030D1F0EB89EE0FEE0FFB
:100C8200EE0FE093F000AB89BC89E5E00E9497CCBF
:100C9200E093F100AB89BC898D899E89EDE00E94C9
:100CA200BFCCE093F200E5E10E94BFCC0AC0EF891D
:100CB200E295E07FEE0FE093F200EF89F88D0E945B
:100CC200EACCE093F30010E01017B0F4A4EDB3E027
:100CD200E0915604F0E0BD01ADE0B0E00E9411CD1C
:100CE200DB01AE0FBF1F1596EE27A10FBE1FEC91C1
:100CF200E093FA001F5FE8CFE98DE05CE093EF003C
:100D0200E091D003E160E093D00303C1E091D0030E
:100D1200E27009F051C0E0E1E093ED00E98DE0936B
:100D2200EF004030D1F0EB89EE0FEE0FEE0FE093C3
:100D3200F000AB89BC89E5E00E9497CCE093F1001A
:100D4200AB89BC898D899E89EDE00E94BFCCE0937E
:100D5200F200E5E10E94BFCC0AC0EF89E295E07F94
:100D6200EE0FE093F200EF89F88D0E94EACCE09357
:100D7200F30010E01017B0F4A4EDB3E0E0915604D4
:100D8200F0E0BD01ADE0B0E00E9411CDDB01AE0F9D
:100D9200BF1F1596EE27A10FBE1FEC91E093FA003C
:100DA2001F5FE8CFE98DE05CE093EF00E091D003B4
:100DB200E260E093D003ADC0E091D003E47009F0AB
:100DC20051C0E0E2E093ED00E98DE093EF004030A6
:100DD200D1F0EB89EE0FEE0FEE0FE093F000AB894E
:100DE200BC89E5E00E9497CCE093F100AB89BC8915
:100DF2008D899E89EDE00E94BFCCE093F200E5E18F
:100E02000E94BFCC0AC0EF89E295E07FEE0FE0932B
:100E1200F200EF89F88D0E94EACCE093F30010E033
:100E22001017B0F4A4EDB3E0E0915604F0E0BD0178
:100E3200ADE0B0E00E9411CDDB01AE0FBF1F1596F1
:100E4200EE27A10FBE1FEC91E093FA001F5FE8CFDF
:100E5200E98DE05CE093EF00E091D003E460E09381
:100E6200D00357C0E091D003E87009F051C0E0E32D
:100E7200E093ED00E98DE093EF004030D1F0EB8993
:100E8200EE0FEE0FEE0FE093F000AB89BC89E5E0C8
:100E92000E9497CCE093F100AB89BC898D899E8931
:100EA200EDE00E94BFCCE093F200E5E10E94BFCCEE
:100EB2000AC0EF89E295E07FEE0FE093F200EF893E
:100EC200F88D0E94EACCE093F30010E01017B0F422
:100ED200A4EDB3E0E0915604F0E0BD01ADE0B0E076
:100EE2000E9411CDDB01AE0FBF1F1596EE27A10F99
:100EF200BE1FEC91E093FA001F5FE8CFE98DE05C42
:100F0200E093EF00E091D003E860E093D00301C0EA
:100F12000EC0E0915604EF5FE0935604E150A091B9
:100F22005604AA3018F0E0E0E093560443CEE0E025
:100F32005E2F2E2F30E4303F08F032C13093ED00A7
:100F4200E091EE00E07209F41EC1E091EF00EF7053
:100F52000E2EEE81E07FE029EE83EF70E93020F083
:100F6200EE81E07FE860EE83E091EF00E07109F44A
:100F72006DC0E091F300FF2766277727EB8BFC8B90
:100F82006D8B7E8BAB89BC898D899E89E8E00E943E
:100F9200A8CCEB8BFC8B6D8B7E8BE091F200AB8946
:100FA200BC898D899E89FF2766277727EA2BFB2B31
:100FB200682B792BEB8BFC8B6D8B7E8BAB89BC8981
:100FC2008D899E89E8E00E94A8CCEB8BFC8B6D8B0F
:100FD2007E8BE091F100AB89BC898D899E89FF27C8
:100FE20066277727EA2BFB2B682B792BEB8BFC8B65
:100FF2006D8B7E8BAB89BC898D899E89E5E00E94D1
:10100200A8CCEB8BFC8B6D8B7E8BE091F000F0E03B
:101012000E94E1CCAB89BC898D899E896F2F660FB6
:10102200660B762FEA2BFB2B682B792BEB8BFC8B39
:101032006D8B7E8BEE81E061EE83EB89FC896D899D
:101042007E89EF83F88769877A871DC0E091F30074
:10105200F0E0EF8BF88F0E94D8CCEF8BF88FE09105
:10106200F200F0E0F595E7950E94DFCCAF89B88DEC
:10107200EA2BFB2BEF8BF88FEE81EF7EEE83EF896D
:10108200F88DEF83F88710E0EE81EF701E1758F4A9
:10109200E12FF0E0DE011B96AE0FBF1FE091FA00D8
:1010A200EC931F5FF1CF2F5FE091CF03E17081F0EE
:1010B200ECEDF1E060E070E00E94E5CDEB8DFC8D9F
:1010C200662777270E94E5CD84E00E94E3CB28962D
:1010D200A091D103A03069F0AF89B88D109749F47F
:1010E200EE81EF70E23028F0E091D103AC85EA178F
:1010F20009F017C0EB85F0E0E130A0E0FA0721F437
:10110200E091CF03EB7F0BC0E230A0E0FA0721F0C1
:10111200E038A0E0FA0729F4E091CF03E460E0931D
:10112200CF03E091CF03E47069F5DE0116960E94C9
:10113200D219E0918C09E27021F0DE0116960E942C
:10114200F583E091AB07F0E0E130A0E0FA0729F483
:10115200DE0116960E949B4615C0E230A0E0FA0717
:1011620021F0E330A0E0FA0729F4DE0116960E948E
:10117200735408C0E430A0E0FA0721F4DE011696A9
:101182000E94625C05C0E091EE00EE7039F05F5F94
:10119200E0E0E093EE00E0E8E093EF00305FCBCEDA
:1011A200222319F4552309F462C0213020F1E09181
:1011B200CE03E03041F4E091E508E160E093E50818
:1011C200E0E0E093E208EEE1E093CE03E091CF03AA
:1011D200E27089F0A2E3B1E00E944FCEFF70A4E872
:1011E200BDE0FF700F01ED91FD91E070F07FE0290D
:1011F200F129FE93EE93A0915804B0915904A13FB6
:10120200EFEFBE0740F4A0915A04B0915B04A13FF6
:10121200EFEFBE0760F1E0915804F0915904F695A2
:10122200E795E0935804F0935904E0915A04F09141
:101232005B04F695E795E0935A04F0935B04A09162
:101242005804B0915904E22FF0E0EA0FFB1FE0933B
:101252005804F0935904A0915A04B0915B04E52F0D
:10126200F0E0EA0FFB1FE0935A04F0935B040E9444
:1012720063CC6A960895BA93AA9324970E945CCC91
:10128200E091CF03E47009F07FC1E0916304E0785C
:1012920021F0AA85BB850E94D219AA85BB85EC9153
:1012A200EF700E2F202FEC91E07151F031E02061B0
:1012B20011960E94CECDEE83FF836887798706C0A0
:1012C20030E0AA85BB8511964D915C91E091D003E7
:1012D200E17009F047C0E0E0E093ED002093EF00F9
:1012E2003030D1F0EE81EE0FEE0FEE0FE093F00012
:1012F200AE81BF81E5E00E9497CCE093F100AE8120
:10130200BF8188859985EDE00E94BFCCE093F20011
:10131200E5E10E94BFCC0CC0E0E0E093F000E42FD6
:10132200E295E07FEE0FE093F200FA010E94EACC30
:10133200E093F30010E0101758F4AA85BB851596C8
:10134200EE27A10FBE1FEC91E093FA001F5FF3CFCF
:10135200E22FE05CE093EF00E091D003E160E093E4
:10136200D00312C1E091D003E27009F047C0E0E17E
:10137200E093ED002093EF003030D1F0EE81EE0FDC
:10138200EE0FEE0FE093F000AE81BF81E5E00E9428
:1013920097CCE093F100AE81BF8188859985EDE01D
:1013A2000E94BFCCE093F200E5E10E94BFCC0CC0EA
:1013B200E0E0E093F000E42FE295E07FEE0FE093AF
:1013C200F200FA010E94EACCE093F30010E0101759
:1013D20058F4AA85BB851596EE27A10FBE1FEC9186
:1013E200E093FA001F5FF3CFE22FE05CE093EF009F
:1013F200E091D003E260E093D003C6C0E091D00355
:10140200E47009F047C0E0E2E093ED002093EF00C2
:101412003030D1F0EE81EE0FEE0FEE0FE093F000E0
:10142200AE81BF81E5E00E9497CCE093F100AE81EE
:10143200BF8188859985EDE00E94BFCCE093F200E0
:10144200E5E10E94BFCC0CC0E0E0E093F000E42FA5
:10145200E295E07FEE0FE093F200FA010E94EACCFF
:10146200E093F30010E0101758F4AA85BB85159697
:10147200EE27A10FBE1FEC91E093FA001F5FF3CF9E
:10148200E22FE05CE093EF00E091D003E460E093B0
:10149200D0037AC0E091D003E87009F047C0E0E3DE
:1014A200E093ED002093EF003030D1F0EE81EE0FAB
:1014B200EE0FEE0FE093F000AE81BF81E5E00E94F7
:1014C20097CCE093F100AE81BF8188859985EDE0EC
:1014D2000E94BFCCE093F200E5E10E94BFCC0CC0B9
:1014E200E0E0E093F000E42FE295E07FEE0FE0937E
:1014F200F200FA010E94EACCE093F30010E0101728
:1015020058F4AA85BB851596EE27A10FBE1FEC9154
:10151200E093FA001F5FF3CFE22FE05CE093EF006D
:10152200E091D003E860E093D0032EC0E09157042D
:10153200EF5F1E2F1A3008F010E0E0915604E11719
:1015420059F4EF5FE0935604E150A0915604AA309B
:1015520018F0E0E0E0935604A4EDB3E0E091570404
:10156200F0E0BD01ADE0B0E00E9411CDE60FF71F43
:10157200FA93EA93EC85FD85FA93EA93ADE0B0E045
:101582000E9449C5109357040E9463CC2C9608957B
:101592001A930A938D011396ED91FD91A091D203B6
:1015A200B091D303EA17FB0721F0F801A381B481BC
:1015B200F2D9E091E508E07851F4E091E508E068BD
:1015C200E093E508E1E0E093E2080E94A537F80124
:1015D200E581EF70E93018F4D80115964CDE0991D7
:1015E20019910895A091CE03A13078F0E091CE0335
:1015F200E150E093CE03E03041F4E091E508EE7F64
:10160200E093E508E0E0E093E20808951A93A3E589
:10161200B5E00E9453CEE0939E0D11E1163048F0E2
:10162200A8E5B5E0EE27A10FBE1F0E9453CEE03021
:1016320009F002C01150F2CFE12FE550E0939F0D67
:10164200E0E0E093A00DAAE6B5E00E9453CEE0935D
:10165200A10DAFE9B5E00E9453CEE093A20DA4ED37
:10166200B5E00E9453CEE093A30DA9E1B6E00E943B
:1016720053CEE093A40DA091A40DA13019F4E2E0A1
:10168200E093A40DE091A40DE093A50DAAE1B6E0CC
:101692000E944BCEE093A70DF093A80D6093A90D85
:1016A2007093AA0DEFEFE093A60DAEE1B6E00E94B3
:1016B2004FCEE093AB0DF093AC0D309719F4E0E010
:1016C200E093A50DABE3B1E00E944BCE30976040B2
:1016D200704011F4E0E00BC0AFE3B1E00E9453CEE2
:1016E200E093AD0DA091AD0DA63018F0E5E0E093CA
:1016F200AD0D10E01330B0F5AFEABDE0E12FF0E040
:10170200EE0FFF1FEA0FFB1F3196FF93EF93A1E24B
:10171200B6E0E12FF0E0BD01A5E1B0E00E9411CDFD
:10172200DB01AE0FBF1F14960E9453CEAF91BF9143
:10173200EC93AFEABDE0E12FF0E0EE0FFF1FAE0F3A
:10174200BF1FEC91E078E560EC93AFEABDE0E12FDA
:10175200F0E0EE0FFF1FAE0FBF1FEC91EF77EC939F
:101762001F5FC8CF1991089561970E945CCCE091E8
:101772006304E07421F40E9463CC67960895A091FB
:10178200A50DA13008F4ABC6E091A50DE150E093A0
:10179200A50DEF5FE091A50DE03009F0A0C6E09144
:1017A200A40DE093A50DE091A60DEF5FE093A60DC9
:1017B200E150A091A60DAF3018F0E0E0E093A60D45
:1017C200EA85E07FE860EA87FE013F96FA93EA93B2
:1017D200E0E0EA93A8E0B0E00E945BC5E091A60DCC
:1017E200F0E0309709F056C1E091AB0DF091AC0DED
:1017F200E17009F44BC100E0E0919307E17009F058
:101802000160E0919407E17009F00260E0919507B0
:10181200E17009F00460E0919607E17009F0086058
:10182200E0919707E17009F00061E0919807E1709B
:1018320009F00062E0919907E17009F00064E0911B
:101842009A07E17009F000680F8700E0E0919B07BA
:10185200E17009F00160E0919C07E17009F002601B
:10186200E0919D07E17009F00460E0919E07E1704C
:1018720009F00860FE017096008300E0E091D60C4A
:10188200E07409F00160E091DE0CE07409F002609E
:10189200E091E60CE07409F00460E091EE0CE07473
:1018A20009F00860E091F60CE07409F00061E09143
:1018B200FE0CE07409F00062E091060DE07409F09C
:1018C2000064E0910E0DE07409F00068FE0171966B
:1018D200008300E0E091160DE07409F00160E091F0
:1018E2001E0DE07409F00260E091260DE07409F02B
:1018F2000460E0912E0DE07409F00860E091360D6D
:10190200E07409F00061E0913E0DE07409F00062BC
:10191200E091460DE07409F00064E0914E0DE07430
:1019220009F00068FE017296008300E0E0917704FE
:10193200E07809F00160E0918504E07809F0026046
:10194200E0919304E07809F00460E091A104E0786A
:1019520009F00860E091AF04E07809F00061E091DD
:10196200BD04E07809F00062E091CB04E07809F070
:101972000064E091D904E07809F00068FE017396F2
:10198200008300E0E091E704E07809F00160E09173
:10199200F504E07809F00260E0910305E07809F0CF
:1019A2000460E0911105E07809F00860E0911F05FC
:1019B200E07809F00061E0912D05E07809F000621D
:1019C200E0913B05E07809F00064E0914905E07898
:1019D20009F00068FE017496008300E0E09157056B
:1019E200E07809F00160E0916505E07809F00260B5
:1019F200E0917305E07809F00460E0918105E078F8
:101A020009F00860E0918F05E07809F00061E0914B
:101A12009D05E07809F00062E0919D05E07809F00B
:101A22000064E091B905E07809F00068FE0175965E
:101A3200008300E0E091C705E07809F00160E091E1
:101A4200D505E07809F00260E091E305E07809F05D
:101A52000460E091F105E07809F00860E091FF058B
:101A6200E07809F00061E0910D06E07809F000628B
:101A7200E0911B06E07809F00064E0912906E07825
:101A820009F00068FE0176960083EFC4E1E0E0937E
:101A9200A60D05C0E130A0E0FA0709F0DCC0E09134
:101AA200AB0DF091AC0DE27009F4D1C0E091F708F2
:101AB200E077E03321F4E091F708E47009F403C021
:101AC200E6E6EF870DC0E091F708E295E770FF27A1
:101AD20066277727E85EFE4F6F4F6BBF06900F8633
:101AE200E0910009E077E03321F4E0910009E4702D
:101AF20009F403C0E6E6E88B0DC0E0910009E29527
:101B0200E770FF2766277727E85EFE4F6F4F6BBFB0
:101B12000690088AE0910909E077E03321F4E09128
:101B22000909E47009F403C0E6E6E98B0DC0E0910F
:101B32000909E295E770FF2766277727E85EFE4FDF
:101B42006F4F6BBF0690098AE0911209E077E0338C
:101B520021F4E0911209E47009F403C0E6E6EA8B8D
:101B62000DC0E0911209E295E770FF2766277727FB
:101B7200E85EFE4F6F4F6BBF06900A8AE0911B0929
:101B8200E077E03321F4E0911B09E47009F403C02B
:101B9200E6E6EB8B0DC0E0911B09E295E770FF27AB
:101BA20066277727E85EFE4F6F4F6BBF06900B8A62
:101BB200E0912409E077E03321F4E0912409E47014
:101BC20009F403C0E6E6EC8B0DC0E0912409E2952E
:101BD200E770FF2766277727E85EFE4F6F4F6BBFE0
:101BE20006900C8AE0912D09E077E03321F4E09130
:101BF2002D09E47009F403C0E6E6ED8B0DC0E09117
:101C02002D09E295E770FF2766277727E85EFE4FEA
:101C12006F4F6BBF06900D8AE0913609E077E03393
:101C220021F4E0913609E47009F403C0E6E6EE8B94
:101C32000DC0E0913609E295E770FF276627772706
:101C4200E85EFE4F6F4F6BBF06900E8A0EC4E2E055
:101C5200E093A60D05C0E230A0E0FA0709F0DCC06F
:101C6200E091AB0DF091AC0DE47009F4D1C0E091BC
:101C72003F09E077E03321F4E0913F09E47009F491
:101C820003C0E6E6EF870DC0E0913F09E295E770F9
:101C9200FF2766277727E85EFE4F6F4F6BBF0690E0
:101CA2000F86E0914809E077E03321F4E09148099A
:101CB200E47009F403C0E6E6E88B0DC0E091480940
:101CC200E295E770FF2766277727E85EFE4F6F4FA2
:101CD2006BBF0690088AE0915109E077E03321F466
:101CE200E0915109E47009F403C0E6E6E98B0DC006
:101CF200E0915109E295E770FF2766277727E85EB2
:101D0200FE4F6F4F6BBF0690098AE0915A09E07748
:101D1200E03321F4E0915A09E47009F403C0E6E6E5
:101D2200EA8B0DC0E0915A09E295E770FF2766271A
:101D32007727E85EFE4F6F4F6BBF06900A8AE091ED
:101D42006309E077E03321F4E0916309E47009F478
:101D520003C0E6E6EB8B0DC0E0916309E295E77004
:101D6200FF2766277727E85EFE4F6F4F6BBF06900F
:101D72000B8AE0916C09E077E03321F4E0916C0981
:101D8200E47009F403C0E6E6EC8B0DC0E0916C0947
:101D9200E295E770FF2766277727E85EFE4F6F4FD1
:101DA2006BBF06900C8AE0917509E077E03321F46D
:101DB200E0917509E47009F403C0E6E6ED8B0DC00D
:101DC200E0917509E295E770FF2766277727E85EBD
:101DD200FE4F6F4F6BBF06900D8AE0917E09E07750
:101DE200E03321F4E0917E09E47009F403C0E6E6F1
:101DF200EE8B0DC0E0917E09E295E770FF27662722
:101E02007727E85EFE4F6F4F6BBF06900E8A2DC399
:101E1200E3E0E093A60D04C0E330A0E0FA0721F46A
:101E2200E4E0E093A60D04C0E430A0E0FA0721F458
:101E3200E5E0E093A60D05C0E530A0E0FA0709F061
:101E4200B0C0E091AB0DF091AC0DE07209F4A5C009
:101E52004091FE085091FF084C3EE3E15E0738F4E2
:101E6200DA01E4E1F0E00E9457CD0E2F01C00FEF3E
:101E72000F87A0910309A63319F4E0E0E88B13C0A1
:101E820040910709509108094C3EE3E15E0738F49E
:101E9200DA01E4E1F0E00E9457CD0E2F01C00FEF0E
:101EA200FE017096008340911009509111094C3E39
:101EB200E3E15E0738F4DA01E4E1F0E00E9457CD95
:101EC2000E2F01C00FEFFE0171960083A09115093C
:101ED200A63319F4E0E0EA8B13C04091190950913E
:101EE2001A094C3EE3E15E0738F4DA01E4E1F0E07E
:101EF2000E9457CD0E2F01C00FEFFE017296008394
:101F020040912209509123094C3EE3E15E0738F4E7
:101F1200DA01E4E1F0E00E9457CD0E2F01C00FEF8D
:101F2200FE017396008340912B0950912C094C3E7F
:101F3200E3E15E0738F4DA01E4E1F0E00E9457CD14
:101F42000E2F01C00FEFFE017496008340913409F9
:101F5200509135094C3EE3E15E0738F4DA01E4E1E1
:101F6200F0E00E9457CD0E2F01C00FEFFE017596D3
:101F7200008340913D0950913E094C3EE3E15E07EA
:101F820038F4DA01E4E1F0E00E9457CD0E2F01C0EF
:101F92000FEFFE017696008368C2E6E0E093A60D9D
:101FA20005C0E630A0E0FA0709F0A2C0E091AB0D4F
:101FB200F091AC0DE07409F497C04091460950913C
:101FC20047094C3EE3E15E0738F4DA01E4E1F0E070
:101FD2000E9457CD0E2F01C00FEF0F8740914F097E
:101FE200509150094C3EE3E15E0738F4DA01E4E136
:101FF200F0E00E9457CD0E2F01C00FEFFE01709648
:10200200008340915809509159094C3EE3E15E0723
:1020120038F4DA01E4E1F0E00E9457CD0E2F01C05E
:102022000FEFFE01719600834091610950916209A0
:102032004C3EE3E15E0738F4DA01E4E1F0E00E94AD
:1020420057CD0E2F01C00FEFFE0172960083409113
:102052006A0950916B094C3EE3E15E0738F4DA01FC
:10206200E4E1F0E00E9457CD0E2F01C00FEFFE0118
:102072007396008340917309509174094C3EE3E1D9
:102082005E0738F4DA01E4E1F0E00E9457CD0E2F4A
:1020920001C00FEFFE017496008340917C095091BC
:1020A2007D094C3EE3E15E0738F4DA01E4E1F0E059
:1020B2000E9457CD0E2F01C00FEFFE0175960083CF
:1020C20040918509509186094C3EE3E15E0738F460
:1020D200DA01E4E1F0E00E9457CD0E2F01C00FEFCC
:1020E200FE0176960083C1C1E7E0E093A60D04C02D
:1020F200E730A0E0FA0721F4E8E0E093A60D04C07F
:10210200E830A0E0FA0721F4E9E0E093A60D04C06C
:10211200E930A0E0FA0741F5E091AB0DF091AC0D8A
:10212200F270F1F0A091ED08AA236AF0A091EC08F8
:10213200B091ED08EAE0F0E00E943FCDAF010E94CD
:10214200E8CCAF0102C040E050E05F87FE0170962C
:102152004083E0919A0DE98BE091990DEA8B85C15C
:10216200EAE0E093A60D04C0EA30A0E0FA07D9F451
:10217200E091AB0DF091AC0DF47089F0A091F508EF
:10218200B091F608E4E1F0E00E9457CDAF015B8B1D
:10219200FE0174964083E0E0ED8BEE8B66C1EBE0CE
:1021A200E093A60D04C0EB30A0E0FA07C9F5E09178
:1021B200AB0DF091AC0DF87079F100E0E091560DA5
:1021C200E07409F00160E0915E0DE07409F00260D4
:1021D200E091660DE07409F00460E0916E0DE07428
:1021E20009F008600F87E0919209E17021F0E09117
:1021F2009309E695EC8BE0919A09E17021F0E09168
:102202009B09E695ED8BE091A209E17021F0E09146
:10221200A309E695EE8B29C1ECE0E093A60D04C07C
:10222200EC30A0E0FA07C9F5E091AB0DF091AC0DEE
:10223200F07179F1E2E0EF87EDE0E88BA6E1B0E042
:102242000E9453CEE98BA5E1B0E00E9453CEEA8B07
:10225200E091AA09E17021F0E091AB09E695EB8BE0
:10226200E091B209E17021F0E091B309E695EC8BBF
:10227200E091BA09E17021F0E091BB09E695ED8B9E
:10228200E091C209E17021F0E091C309E695EE8B7D
:10229200ECC0EDE0E093A60D05C0ED30A0E0FA073A
:1022A20009F0A6C0E091AB0DF091AC0DF07209F40B
:1022B2009BC0E091AE0DEF5FE093AE0DE150EF8772
:1022C20000E0E0919C0DE03009F00160E0919D0D8D
:1022D200E03009F00260E091F008E17009F004607A
:1022E200E091F008E27009F00860E091F008E07215
:1022F20009F00061E091EF08E07809F00062A5E3DF
:10230200B1E00E9453CEA091900DAE1708F0006488
:10231200A091CE03A13008F00068FE017096008300
:10232200E091840DF091850DFF70EF2FF0E0E98BC5
:10233200E091840DF091850DEA8BE0E01E2F0E2FC7
:1023420031E0183060F4A3E01A9FF001ED5BF84F22
:10235200E081E27009F0032B1F5F330FF2CFFE0121
:102362007396008300E018E031E0103160F4A3E0DE
:102372001A9FF001ED5BF84FE081E27009F0032B48
:102382001F5F330FF2CFFE017496008300E010E16D
:1023920031E0143160F4A3E01A9FF001ED5BF84FD5
:1023A200E081E27009F0032B1F5F330FF2CFFE01D1
:1023B20075960083E0E01E2F0E2F31E0153080F479
:1023C200E12FAFE7B7E0F0E00E94DACCAE0FBF1F1B
:1023D2001396EC91E17009F0032B1F5F330FEECFE0
:1023E200FE017696008341C0EEE0E093A60D04C0A4
:1023F200EE30A0E0FA07C9F5E091AB0DF091AC0D1B
:10240200F07479F1E0917508F09176080E94ECCCB5
:10241200AF015F87FE0170964083E0917708F091EB
:1024220078080E94ECCCAF01598BFE017296408372
:1024320000E0E091F008E47009F00160E091F0083A
:10244200E87009F00260E091F008E07109F00460C0
:10245200E091F008E07209F00860FE0173960083D3
:1024620004C0E0E0E093A60DB9C9A091A70DB09118
:10247200A80D8091A90D9091AA0DE091A60DF0E012
:102482006F2F660F660B762FEA0FFB1F681F791FEF
:10249200EE83FF8368877987AE81BF8188859985BE
:1024A200A030E8E0BE07E0E08E07E0E09E0740F4DF
:1024B200EA85EF7EEA87EE81FF81EB87FC870BC01E
:1024C200EA85E061EA87EE81FF8168857985EB879D
:1024D200FC876D877E87DE011A960E943C090E9466
:1024E20063CC6796089564970E945CCCE091630484
:1024F200E07409F423C4EF81E07FE860EF83A091E8
:10250200AD0DA13008F44FC0E091AD0DE150E09364
:10251200AD0DEF5FE091AD0DE03009F044C0AFE3E7
:10252200B1E00E9453CEE093AD0DABE3B1E00E9467
:102532004BCEEC8BFD8B6E8B7F8BAC89BD898E89EC
:102542009F89A030E8E0BE07E0E08E07E0E09E074A
:1025520040F4EF81EF7EEF83EC89FD89E887F9870C
:102562000BC0EF81E061EF83EC89FD896E897F8981
:10257200E887F9876A877B87A9E3B1E00E9453CE97
:10258200EC87AAE3B1E00E9453CEED87E2E0EE874A
:10259200EDE0EF87E0E0E88BE98BEA8BEB8BDE0185
:1025A20017960E943C09A0919E0DA13008F421C10A
:1025B200E0919E0DE150E0939E0DE03009F019C1CB
:1025C200FE013C96FA93EA93E0E0EA93A8E0B0E0D9
:1025D2000E945BC5A3E5B5E00E9453CEE0939E0D39
:1025E200A4E5B5E00E944BCEEC8BFD8B6E8B7F8B0E
:1025F200AC89BD898E899F89A030E8E0BE07E0E002
:102602008E07E0E09E0740F4EF81EF7EEF83EC89D6
:10261200FD89E887F9870BC0EF81E061EF83EC89E0
:10262200FD896E897F89E887F9876A877B87A09110
:102632009F0DA13090F1E091A00DEF5FE093A00D0E
:10264200E150A091A00DE0919F0DEA1718F4E1E08E
:10265200E093A00DE091A00DEC87A8E5B5E0F0E0D5
:102662003496AE0FBF1F0E9453CE4E2F4F3010F044
:102672004F3108F012C0E42FF0E03F97A9E0B0E03C
:102682000E9411CDE250F74FDF01ED91FD91DF0184
:10269200E4E1F0E00E9457CDEB8BADE5B5E00E949E
:1026A20053CE4E2F4F3010F04F3108F012C0E42FAE
:1026B200F0E03F97A9E0B0E00E9411CDE250F74F61
:1026C200DF01ED91FD91DF01E4E1F0E00E9457CDE1
:1026D200EA8BACE5B5E00E9453CE4E2F4F3010F09E
:1026E2004F3108F012C0E42FF0E03F97A9E0B0E0CC
:1026F2000E9411CDE250F74FDF01ED91FD91DF0114
:10270200E4E1F0E00E9457CDE98BABE5B5E00E9431
:1027120053CE4E2F4F3010F04F3108F012C0E42F3D
:10272200F0E03F97A9E0B0E00E9411CDE250F74FF0
:10273200DF01ED91FD91DF01E4E1F0E00E9457CD70
:10274200E88BAAE5B5E00E9453CE4E2F4F3010F031
:102752004F3108F012C0E42FF0E03F97A9E0B0E05B
:102762000E9411CDE250F74FDF01ED91FD91DF01A3
:10277200E4E1F0E00E9457CDEF87A9E5B5E00E94C1
:1027820053CE4E2F4F3010F04F3108F012C0E42FCD
:10279200F0E03F97A9E0B0E00E9411CDE250F74F80
:1027A200DF01ED91FD91DF01E4E1F0E00E9457CD00
:1027B200EE87A8E5B5E00E9453CE4E2F4F3010F0C1
:1027C2004F3108F012C0E42FF0E03F97A9E0B0E0EB
:1027D2000E9411CDE250F74FDF01ED91FD91DF0133
:1027E200E4E1F0E00E9457CDED87DE0117960E94EA
:1027F2003C09A091A10DA13008F47CC0E091A10D8B
:10280200E150E093A10DEF5FE091A10DE03009F0FE
:1028120071C0FE013C96FA93EA93E0E0EA93A8E0E5
:10282200B0E00E945BC5AAE6B5E00E9453CEE093F9
:10283200A10DABE6B5E00E944BCEEC8BFD8B6E8B0F
:102842007F8BAC89BD898E899F89A030E8E0BE0765
:10285200E0E08E07E0E09E0740F4EF81EF7EEF8339
:10286200EC89FD89E887F9870BC0EF81E061EF838E
:10287200EC89FD896E897F89E887F9876A877B877A
:10288200E0E00E2F1E2F2E2F51E0103300F5AFE6A1
:10289200B5E0EE27A10FBE1F0E9453CE4E2F40304F
:1028A20031F0A42F0E948A3BE03009F0052B50380A
:1028B20059F4E22F2F5FF0E0DE011C96EA0FFB1FB6
:1028C200008351E000E001C0550F1F5FDECFA091F1
:1028D200F508B091F608AC39E3E6BE0728F4E4E661
:1028E200F0E00E9457CD01C0EFEFEA8BDE011796B0
:1028F2000E943C09A091A20DA13008F4A9C0E09168
:10290200A20DE150E093A20DEF5FE091A20DE03045
:1029120009F09EC0AFE9B5E00E9453CEE093A20D4C
:10292200A0EAB5E00E944BCEEC8BFD8B6E8B7F8BC9
:10293200AC89BD898E899F89A030E8E0BE07E0E0BE
:102942008E07E0E09E0740F4EF81EF7EEF83EC8993
:10295200FD89E887F9870BC0EF81E061EF83EC899D
:10296200FD896E897F89E887F9876A877B87E0E03E
:102972000E2F1E2F2E2F51E0103308F055C0A4EA5F
:10298200B5E0EE27A10FBE1F0E9453CE4E2F40305E
:10299200D9F14F3010F04F3108F024C04F3108F513
:1029A200E42FF0E03F97A9E0B0E00E9411CDE9509A
:1029B200F74FE081E295E770EE83E42FF0E03F9776
:1029C200A9E0B0E00E9411CDE950F74FE081E47038
:1029D20039F4AE81A13021F0A43011F0A53009F410
:1029E200052B12C0473310F04C3308F007C0A42F58
:1029F2000E945D7CE03009F0052B06C0A42F0E94E6
:102A02008A3BE03009F0052B503859F4E22F2F5F52
:102A1200F0E0DE011C96EA0FFB1F008351E000E0AC
:102A220001C0550F1F5FA8CFA091EC08B091ED082F
:102A320000240A160B0624F4EA89E295EF7001C01D
:102A4200E0E0EA8BE0E0EB8BDE0117960E943C09A6
:102A5200A091A30DA13008F4A8C0E091A30DE1500C
:102A6200E093A30DEF5FE091A30DE03009F09DC06C
:102A7200FE013C96FA93EA93E0E0EA93A8E0B0E024
:102A82000E945BC5A4EDB5E00E9453CEE093A30D76
:102A9200A5EDB5E00E944BCEEC8BFD8B6E8B7F8B50
:102AA200AC89BD898E899F89A030E8E0BE07E0E04D
:102AB2008E07E0E09E0740F4EF81EF7EEF83EC8922
:102AC200FD89E887F9870BC0EF81E061EF83EC892C
:102AD200FD896E897F89E887F9876A877B87E0E0CD
:102AE2000E2F1E2F2E2F51E0103408F05AC0A9EDE0
:102AF200B5E0EE27A10FBE1F0E9453CE4E2F4030ED
:102B020009F43FC0103220F04F3010F04F3108F07E
:102B120024C04F3108F5E42FF0E03F97A9E0B0E080
:102B22000E9411CDE950F74FE081E295E770EE8304
:102B3200E42FF0E03F97A9E0B0E00E9411CDE95008
:102B4200F74FE081E47039F4AE81A13021F0A43076
:102B520011F0A53009F4052B14C0103220F04733D0
:102B620010F04C3308F007C0A42F0E945D7CE030C7
:102B720009F0052B06C0A42F0E948A3BE03009F021
:102B8200052B503859F4E22F2F5FF0E0DE011C963E
:102B9200EA0FFB1F008351E000E001C0550F1F5FE9
:102BA200A3CFDE0117960E943C0910E0133008F013
:102BB200C5C0AFEABDE0E12FF0E0EE0FFF1FAE0FA0
:102BC200BF1F11964C91403009F4B6C0AFEABDE088
:102BD200E12FF0E0EE0FFF1FAE0FBF1FEC91EF777A
:102BE2003E2FA42F0E948A3B0E2FAFEABDE0E12FB9
:102BF200F0E0EE0FFF1FAE0FBF1FEC91EE1FE0E003
:102C0200EE1FE1700E1799F031E0AFEABDE0E12F5F
:102C1200F0E0EE0FFF1FAE0FBF1FE02FE170E79550
:102C2200E0E0E7950E2EEC91EF77E029EC9331305E
:102C320008F473C03150303009F06FC0A0E2B6E042
:102C42000E9453CE3E2FA1E2B6E0E12FF0E0BD019B
:102C5200A5E1B0E00E9411CDDB01AE0FBF1F0E94C3
:102C62004BCEEC8BFD8B6E8B7F8BAC89BD898E89B5
:102C72009F89A030E8E0BE07E0E08E07E0E09E0713
:102C820040F4EF81EF7EEF83EC89FD89E887F987D5
:102C92000BC0EF81E061EF83EC89FD896E897F894A
:102CA200E887F9876A877B87EF81E07FE860EF83B7
:102CB200AFEABDE0E12FF0E0EE0FFF1FAE0FBF1F46
:102CC200EC91E07869F0A1E2B6E0E12FF0E0BD011D
:102CD200A5E1B0E00E9411CDE60FF71F35960CC0BA
:102CE200A1E2B6E0E12FF0E0BD01A5E1B0E00E9473
:102CF20011CDE60FF71F3D96E88FF98FFE013C9646
:102D0200FA93EA93EA8DFB8DFA93EA93A8E00E9484
:102D1200F925DE0117960E943C09AFEABDE0E12FDA
:102D2200F0E0EE0FFF1FAE0FBF1FE32FEF770E2E67
:102D3200EC91E078E029EC931F5F38CF0E9463CCDE
:102D42006A9608951A93A3E5B5E0E0E00E946FCE7B
:102D5200A4E5B5E0E0E0F0E060E070E00E945FCE64
:102D620010E0123148F4A8E5B5E0EE27A10FBE1F2E
:102D72000E946FCE1F5FF5CFE0E2F6E0FA93EA938E
:102D8200AAE60E942E26E0E9F6E4FA93EA93A0E589
:102D9200B0E00E94CE29AAE6B5E0E0E00E946FCE44
:102DA200ABE6B5E0E0E0F0E060E070E00E945FCE0C
:102DB20010E0103348F4AFE6B5E0EE27A10FBE1FD6
:102DC2000E946FCE1F5FF5CFAFE9B5E0E0E00E9451
:102DD2006FCEA0EAB5E0E0E0F0E060E070E00E94D3
:102DE2005FCE10E0103348F4A4EAB5E0EE27A10F5D
:102DF200BE1F0E946FCE1F5FF5CFA4EDB5E0E0E0ED
:102E02000E946FCEA5EDB5E0E0E0F0E060E070E09A
:102E12000E945FCE10E0103448F4A9EDB5E0EE2731
:102E2200A10FBE1F0E946FCE1F5FF5CFA9E1B6E0D2
:102E3200E0E00E946FCEAAE1B6E0E0E0F0E060E000
:102E420070E00E945FCEAEE1B6E0E7E6FEEF0E94E0
:102E520067CEA5C21A93ACE6B2E00E944FCEDF0164
:102E62000E94CC04A5E7B2E00E9453CEE170A5EE29
:102E7200B8E0E170E795E0E0E7950E2EEC91EF7790
:102E8200E029EC93E0E0E093E208EDE5F4E0FA9368
:102E9200EA93E0E0EA93A6EEB2E00E945BC5A0E707
:102EA200B2E00E9453CEE0935E04A0915E04A5308E
:102EB20018F4E5E0E0935E04A5E7B2E00E9453CE89
:102EC200E695E170A3E6B4E0E170E795E0E0E7950E
:102ED2000E2EEC91EF77E029EC93A1E7B2E00E948D
:102EE2004BCEE0935F04F0936004609361047093AF
:102EF2006204E0E0E0936A0410E0143308F01DC2BB
:102F0200ABE7B2E0E12FF0E0BD01AEE0B0E00E943D
:102F120011CDDB01AE0FBF1F1A960E9453CEE0788F
:102F220009F409C2ABE6B4E0E12FF0E0BD01AEE086
:102F3200B0E00E9411CDDB01AE0FBF1F1A96EC91DB
:102F4200E068EC93ABE6B4E0E12FF0E0BD01AEE067
:102F5200B0E00E9411CDE60FF71FFF93EF93ABE7AE
:102F6200B2E0E12FF0E0BD01AEE0B0E00E9411CD91
:102F7200DB01AE0FBF1F0E944BCEAF91BF91ED930D
:102F8200FD936D937C93ABE6B4E0E12FF0E0BD01DD
:102F9200AEE0B0E00E9411CDE60FF71F3496FF932A
:102FA200EF93ABE7B2E0E12FF0E0BD01AEE0B0E0BD
:102FB2000E9411CDDB01AE0FBF1F14960E944FCEAF
:102FC200AF91BF91ED93FC93ABE6B4E0E12FF0E05B
:102FD200BD01AEE0B0E00E9411CDE60FF71F3696BC
:102FE200FF93EF93ABE7B2E0E12FF0E0BD01AEE07B
:102FF200B0E00E9411CDDB01AE0FBF1F16960E94FA
:103002004FCEAF91BF91ED93FC93ABE6B4E0E12FCD
:10301200F0E0BD01AEE0B0E00E9411CDE60FF71F77
:103022003896FF93EF93ABE7B2E0E12FF0E0BD01FA
:10303200AEE0B0E00E9411CDDB01AE0FBF1F1896CB
:103042000E944FCEAF91BF91ED93FC93ABE6B4E0FB
:10305200E12FF0E0BD01AEE0B0E00E9411CDE60F3D
:10306200F71F3A96FF93EF93ABE7B2E0E12FF0E060
:10307200BD01AEE0B0E00E9411CDDB01AE0FBF1F7B
:103082001A960E9453CEEF70AF91BF91EF700E2E41
:10309200EC91E07FE029EC93ABE6B4E0E12FF0E0C5
:1030A200BD01AEE0B0E00E9411CDE60FF71F3A96E7
:1030B200FF93EF93ABE7B2E0E12FF0E0BD01AEE0AA
:1030C200B0E00E9411CDDB01AE0FBF1F1A960E9425
:1030D20053CEE295E770AF91BF91E770E295E07F42
:1030E2000E2EEC91EF78E029EC93ABE6B4E0E12F01
:1030F200F0E0BD01AEE0B0E00E9411CDE60FF71F97
:103102003B96FF93EF93ABE7B2E0E12FF0E0BD0116
:10311200AEE0B0E00E9411CDDB01AE0FBF1F1B96E7
:103122000E9453CEEF70AF91BF91EF700E2EEC91D3
:10313200E07FE029EC93ABE6B4E0E12FF0E0BD01E3
:10314200AEE0B0E00E9411CDE60FF71F3B96FF9371
:10315200EF93ABE7B2E0E12FF0E0BD01AEE0B0E00B
:103162000E9411CDDB01AE0FBF1F1B960E9453CEF2
:10317200E295EF70AF91BF91EF70E295E07F0E2E76
:10318200EC91EF70E029EC93ABE6B4E0E12FF0E0D4
:10319200BD01AEE0B0E00E9411CDE60FF71F3C96F4
:1031A200FF93EF93ABE7B2E0E12FF0E0BD01AEE0B9
:1031B200B0E00E9411CDDB01AE0FBF1F1C960E9432
:1031C20053CEE170AF91BF91E1700E2EEC91EE7F84
:1031D200E029EC93ABE6B4E0E12FF0E0BD01AEE014
:1031E200B0E00E9411CDE60FF71F3C96FF93EF93DC
:1031F200ABE7B2E0E12FF0E0BD01AEE0B0E00E944B
:1032020011CDDB01AE0FBF1F1C960E9453CEE69577
:10321200E170AF91BF91E170EE0F0E2EEC91ED7F58
:10322200E029EC93ABE6B4E0E12FF0E0BD01AEE0C3
:10323200B0E00E9411CDE60FF71F3C96FF93EF938B
:10324200ABE7B2E0E12FF0E0BD01AEE0B0E00E94FA
:1032520011CDDB01AE0FBF1F1C960E9453CEE69527
:10326200E695E370AF91BF91E370EE0FEE0F0E2E75
:10327200EC91E37FE029EC93ABE6B4E0E12FF0E0E0
:10328200BD01AEE0B0E00E9411CDE60FF71F3C9603
:10329200FF93EF93ABE7B2E0E12FF0E0BD01AEE0C8
:1032A200B0E00E9411CDDB01AE0FBF1F1C960E9441
:1032B20053CEE295E170AF91BF91E170E295E07F6C
:1032C2000E2EEC91EF7EE029EC93ABE6B4E0E12F19
:1032D200F0E0BD01AEE0B0E00E9411CDDB01AE0F27
:1032E200BF1F1C96EC91EC70E43089F0ABE6B4E0C1
:1032F200E12FF0E0BD01AEE0B0E00E9411CDDB01B4
:10330200AE0FBF1F1C96EC91EC70EC3081F4ABE673
:10331200B4E0E12FF0E0BD01AEE0B0E00E9411CDDB
:10332200DB01AE0FBF1F1C96EC91E068EC93E12F1E
:10333200EF5FE0936A041F5FE0CDE4E6F4E0FA9306
:10334200EA93E0E4F1E0FA93EA93A5E00E94F9251A
:10335200E0916504F09166046091670470916804DD
:1033620030976040704021F4E0916404EF7E15C014
:10337200E0916404E061E0936404F0E0F695E7957F
:10338200E370F070E330A0E0FA0721F0E130A0E052
:10339200FA0729F4E0916404E860E0936404199167
:1033A2000895BA93AA936D970E945CCCE0E0EE8BED
:1033B200ABA1BCA1EC91E295E1703E2F3030C1F09F
:1033C2001196ED91FD916D917D91ED8FFE8F6F8F35
:1033D20078A3E0915F04F0916004609161047091C0
:1033E2006204AD8DBE8D8F8D98A10E9409CD0CC057
:1033F200ABA1BCA111964D915C91A0915F04B091DB
:103402006004FA010E94F7CCE88FE030A9F1ABA189
:10341200BCA1EC91EF70E13048F0EBA1FCA1A581D9
:10342200A17021F00E94DB270E94347AABA1BCA1DB
:10343200EC91EF70E63000F120E0E1E0EA8FE98FF5
:103442002031D0F4ABA1BCA11596EA8DF0E0AE0F0D
:10345200BF1FEC91A98DEA2319F0A22F0E94886C5C
:10346200E98DEE0FE98FE03029F4EA8DEF5FEA8F04
:10347200E1E0E98F2F5FE4CFE0916404E07109F4A9
:103482003FC0303079F0E0916504F09166046091BC
:10349200670470916804AD8DBE8D8F8D98A10E94D6
:1034A20009CD07C0A0916504B0916604FA010E949B
:1034B200F7CCE88FE03021F1EBA1FCA1A581A1704E
:1034C20071F0E0916404E17021F0E0916404E77F1F
:1034D20003C0E0916404E860E09364040DC0E091ED
:1034E2006404E17021F0E0916404E86003C0E091BB
:1034F2006404E77FE0936404E0915E04E09369046E
:10350200E0916304EF70E23011F4E1E0EE8BA09100
:103512006A04A433A0F0EAEEF1E060E070E00E94F9
:10352200E5CDE0916A04FF27662777270E94E5CD63
:1035320084E00E94E3CB2896E4E3E0936A0420E06F
:10354200E0916A042E1708F04FC5ABE6B4E0E22F13
:10355200F0E0BD01AEE0B0E00E9411CDE60FF71F32
:103562008F01E285E07809F43DC5303061F0D80181
:10357200ED91FD916D917D91AD8DBE8D8F8D98A157
:103582000E9409CD07C0D801ED91FD91DF01FA013A
:103592000E94F7CCE88FE03009F424C5E09163047F
:1035A200E07409F40DC5F801E485E07171F1ABE74F
:1035B200B2E0E22FF0E0BD01AEE0B0E00E9411CD3A
:1035C200DB01AE0FBF1F1C960E9453CEE295EF7037
:1035D200E695E770ABA1BCA11596F0E0AE0FBF1F58
:1035E200EC91EF93ABE7B2E0E22FF0E0BD01AEE089
:1035F200B0E00E9411CDDB01AE0FBF1F1D960E94ED
:1036020053CEAF91EA1709F0DBC4ABE6B4E0E22F88
:10361200F0E0BD01AEE0B0E00E9411CDDB01AE0FE3
:10362200BF1F1D96E0915E04EC93E0E0E9A3EAA3DC
:10363200F801E385EF70E13038F1ABA1BCA115963A
:10364200F801E385F0E0EF70F0703197AE0FBF1F25
:10365200EC91F0E0E9A3FAA3F9A1E0E0E9A3FAA36F
:10366200ABA1BCA11596F801E385F0E00E94E8CC7D
:10367200EF70F0703197AE0FBF1FEC91A9A1BAA104
:10368200F0E0EA2BFB2B0FC0ABA1BCA11596F80111
:10369200E385F0E00E94E8CCEF70F0703197AE0F56
:1036A200BF1FEC91F0E0E9A3FAA3D8011896ED91BF
:1036B200FD91A9A1BAA1EA23FB23E9A3FAA3F80188
:1036C200E485E17059F0F801A085B185FD01F69518
:1036D200E795A9A1BAA1EA17FB0708F00CC0D80127
:1036E2001896ED91FD91E095F095A9A1BAA1EA2B6A
:1036F200FB2BE9A3FAA3F801E485E295EF70E695C6
:10370200E695E170EF8BF801E485E17009F456C2A9
:10371200E9A1FAA1EB8FFC8FF801E285F0E0EF70EE
:10372200F070E630A0E0FA0709F4C7C13097C9F497
:10373200AB8DBC8D00240A160B0624F4EB8DFC8D98
:10374200F29606C0AC8DAA232AF4EB8DFC8DF2977B
:10375200EB8FFC8FAB8DBC8DE4E6F0E00E946ACD6E
:10376200AAC1E130A0E0FA07C9F4AB8DBC8D0024F8
:103772000A160B0624F4EB8DFC8D799606C0AC8DEF
:10378200AA232AF4EB8DFC8D7997EB8FFC8FAB8DFE
:10379200BC8DE2E3F0E00E946ACD8DC1E230A0E090
:1037A200FA07C9F4AB8DBC8D00240A160B0624F46B
:1037B200EB8DFC8D3A9606C0AC8DAA232AF4EB8DD4
:1037C200FC8D3A97EB8FFC8FAB8DBC8DE4E1F0E082
:1037D2000E946ACD70C1E330A0E0FA07C9F4AB8D54
:1037E200BC8D00240A160B0624F4EB8DFC8D359655
:1037F20006C0AC8DAA232AF4EB8DFC8D3597EB8F96
:10380200FC8FAB8DBC8DEAE0F0E00E946ACD53C123
:10381200E430A0E0FA07C9F4AB8DBC8D00240A168F
:103822000B0624F4EB8DFC8D339606C0AC8DAA23D7
:103832002AF4EB8DFC8D3397EB8FFC8FAB8DBC8D17
:10384200E5E0F0E00E946ACD36C1E530A0E0FA077B
:10385200C9F4AB8DBC8D00240A160B0624F4EB8D43
:10386200FC8D329606C0AC8DAA232AF4EB8DFC8D1A
:103872003297EB8FFC8FAB8DBC8DE2E0F0E00E94C3
:103882006ACD19C1E730A0E0FA0741F5AB8DBC8DD6
:1038920000240A160B0674F4AF3FEFE3BE071CF0D8
:1038A200EFEFFFE704C0EB8DFC8DEE0FFF1FEB8FF8
:1038B200FC8F13C0AC8DAA2382F4AB8DBC8DE0E0EB
:1038C200F0ECEA17FB071CF0E0E0F0E804C0EB8D37
:1038D200FC8DEE0FFF1FEB8FFC8FEFC0E830A0E0F6
:1038E200FA0761F5AB8DBC8D00240A160B0684F431
:1038F200A939E9E1BE071CF0EFEFFFE706C0EB8D47
:10390200FC8DA5E0B0E00E943FCDEB8FFC8F15C08F
:10391200AC8DAA2392F4AB8DBC8DE7E6F6EEEA17E6
:10392200FB071CF0E0E0F0E806C0EB8DFC8DA5E0A3
:10393200B0E00E943FCDEB8FFC8FBFC0E930A0E02A
:10394200FA0761F5AB8DBC8D00240A160B0684F4D0
:10395200AC3CECE0BE071CF0EFEFFFE706C0EB8DDE
:10396200FC8DAAE0B0E00E943FCDEB8FFC8F15C02A
:10397200AC8DAA2392F4AB8DBC8DE4E3F3EFEA178E
:10398200FB071CF0E0E0F0E806C0EB8DFC8DAAE03E
:10399200B0E00E943FCDEB8FFC8F8FC0EA30A0E0F9
:1039A200FA0761F5AB8DBC8D00240A160B0684F470
:1039B200A636E6E0BE071CF0EFEFFFE706C0EB8D90
:1039C200FC8DA4E1B0E00E943FCDEB8FFC8F15C0CF
:1039D200AC8DAA2392F4AB8DBC8DEAE9F9EFEA171C
:1039E200FB071CF0E0E0F0E806C0EB8DFC8DA4E1E3
:1039F200B0E00E943FCDEB8FFC8F5FC0EB30A0E0C8
:103A0200FA0761F5AB8DBC8D00240A160B0684F40F
:103A1200AF38E2E0BE071CF0EFEFFFE706C0EB8D28
:103A2200FC8DA2E3B0E00E943FCDEB8FFC8F15C06E
:103A3200AC8DAA2392F4AB8DBC8DE1E7FDEFEA17C2
:103A4200FB071CF0E0E0F0E806C0EB8DFC8DA2E382
:103A5200B0E00E943FCDEB8FFC8F2FC0EC30A0E096
:103A6200FA0759F5AB8DBC8D00240A160B0684F4B7
:103A7200A734E1E0BE071CF0EFEFFFE706C0EB8DD5
:103A8200FC8DA4E6B0E00E943FCDEB8FFC8F15C009
:103A9200AC8DAA2392F4AB8DBC8DE1E7FDEFEA1762
:103AA200FB071CF0E0E0F0E806C0EB8DFC8DA4E61D
:103AB200B0E00E943FCDEB8FFC8FF801E285F0E091
:103AC2000E94E8CCE770F070309769F4F801A481A5
:103AD200B581EB8DFC8DEA17FB0711F4E1E001C023
:103AE200E0E0EF8B6AC0E130A0E0FA0769F4F80188
:103AF200A481B581EB8DFC8DEA17FB0711F4E0E0A0
:103B020001C0E1E0EF8B59C0E230A0E0FA07D9F43E
:103B1200EF89E03061F0D8011696ED91FD91AB8D01
:103B2200BC8DEA17FB0714F0E0E0EF8B0BC0D80165
:103B32001496ED91FD91AB8DBC8DEA17FB0714F441
:103B4200E1E0EF8B3AC0E330A0E0FA07D9F4EF8965
:103B5200E03061F0D8011696ED91FD91AB8DBC8DF0
:103B6200AE17BF0714F0E0E0EF8B0BC0D80114963C
:103B7200ED91FD91AB8DBC8DAE17BF0714F4E1E062
:103B8200EF8B1BC0E430A0E0FA07B9F4D801149619
:103B9200ED91FD91AB8DBC8DAE17BF074CF0D801F6
:103BA2001696ED91FD91AB8DBC8DEA17FB070CF4D7
:103BB20002C0E1E001C0E0E0EF8B75C1F801E285EF
:103BC200F0E0EF70F070E630A0E0FA0709F4CCC044
:103BD200309761F4E9A1FAA1F296E9A3FAA3A9A1A7
:103BE200BAA1E4E6F0E00E9457CDBCC0E130A0E00B
:103BF200FA0761F4E9A1FAA17996E9A3FAA3A9A1C6
:103C0200BAA1E2E3F0E00E9457CDACC0E230A0E0FE
:103C1200FA0761F4E9A1FAA13A96E9A3FAA3A9A1E4
:103C2200BAA1E4E1F0E00E9457CD9CC0E330A0E0ED
:103C3200FA0761F4E9A1FAA13596E9A3FAA3A9A1C9
:103C4200BAA1EAE0F0E00E9457CD8CC0E430A0E0D7
:103C5200FA0761F4E9A1FAA13396E9A3FAA3A9A1AB
:103C6200BAA1E5E0F0E00E9457CD7CC0E530A0E0CB
:103C7200FA0741F4E9A1FAA13196E9A3FAA3F6956C
:103C8200E79570C0E730A0E0FA0781F4A9A1BAA1D4
:103C9200AF3FEFE7BE0728F4E9A1FAA1EE0FFF1F3D
:103CA20002C0EFEFFFEFE9A3FAA35EC0E830A0E0A5
:103CB200FA0779F4A9A1BAA1A333E3E3BE0720F47A
:103CC200E5E00E9439CD02C0EFEFFFEFE9A3FAA3CE
:103CD2004BC0E930A0E0FA0779F4A9A1BAA1A93949
:103CE200E9E1BE0720F4EAE00E9439CD02C0EFEF1D
:103CF200FFEFE9A3FAA338C0EA30A0E0FA0779F4AB
:103D0200A9A1BAA1AC3CECE0BE0720F4E4E10E9418
:103D120039CD02C0EFEFFFEFE9A3FAA325C0EB30E4
:103D2200A0E0FA0779F4A9A1BAA1AE31E5E0BE0795
:103D320020F4E2E30E9439CD02C0EFEFFFEFE9A3E6
:103D4200FAA312C0EC30A0E0FA0771F4A9A1BAA15B
:103D5200AF38E2E0BE0720F4E4E60E9439CD02C0AB
:103D6200EFEFFFEFE9A3FAA3F801E285F0E00E948A
:103D7200E8CCE770F070309769F4F801A481B5815E
:103D8200E9A1FAA1EA17FB0711F4E1E001C0E0E0C2
:103D9200EF8B89C0E130A0E0FA0769F4F801A48151
:103DA200B581E9A1FAA1EA17FB0711F0E0E001C031
:103DB200E1E0EF8B78C0E230A0E0FA07D1F5F8013C
:103DC200E485E170D9F0EF89E03061F0D801169610
:103DD200ED91FD91A9A1BAA1EA17FB0714F0E0E069
:103DE200EF8B0BC0D8011496ED91FD91A9A1BAA158
:103DF200EA17FB0714F4E1E0EF8B1AC0EF89E03019
:103E020061F0D8011696ED91FD91A9A1BAA1EA1728
:103E1200FB0710F0E0E0EF8B0BC0D8011496ED9198
:103E2200FD91A9A1BAA1EA17FB0710F4E1E0EF8B1B
:103E32003AC0E330A0E0FA07D9F4EF89E03061F04C
:103E4200D8011696ED91FD91A9A1BAA1AE17BF07AF
:103E520010F0E0E0EF8B0BC0D8011496ED91FD91CC
:103E6200A9A1BAA1AE17BF0710F4E1E0EF8B1BC006
:103E7200E430A0E0FA07B9F4D8011496ED91FD916F
:103E8200A9A1BAA1AE17BF0748F0D8011696ED91C5
:103E9200FD91A9A1BAA1EA17FB0708F402C0E1E06B
:103EA20001C0E0E0EF8BF801E485E27009F448C05C
:103EB200F801E485E07419F4EF89E03009F43FC0B9
:103EC200F801E485E078F1F0D8011C96EC91EF77E7
:103ED200EC93E0916304E073E03298F0EDEFF1E0EF
:103EE20060E070E00E94E5CDE22FF0E031966F2FA6
:103EF200660F660B762F0E94E5CD84E00E94E3CB2D
:103F020028961DC0D8011C96EC91E068EC93E091D4
:103F12006304E073E03298F0E8E0F2E060E070E021
:103F22000E94E5CDE22FF0E031966F2F660F660B0F
:103F3200762F0E94E5CD84E00E94E3CB289633C021
:103F4200F801E485EE1FE0E0EE1FE170AE2FEF898D
:103F5200EA1749F1D8011C96E170E795E0E0E79590
:103F62000E2EEC91EF77E029EC93E0916304E0737D
:103F7200E032C8F0E3E1F2E060E070E00E94E5CDFB
:103F8200E22FF0E031966F2F660F660B762F0E94BC
:103F9200E5CDEF8DFF27662777270E94E5CD88E0E4
:103FA2000E94E3CB2C96D8011C96EF89E170E29532
:103FB200E07FEE0FEE0F0E2EEC91EF7BE029EC93FB
:103FC200E0916304EF70E13059F0E0916304EF7027
:103FD200AE2FE22FF0E03396B0E0EA17FB0711F4C0
:103FE200E1E0EE8B2F5FACCAE0916304EF70E23048
:103FF20019F0EE89E030A1F1ABA1BCA1EC91EF7018
:10400200ED87AD85A93010F0E8E0ED87ED85E85F3A
:10401200EF83E6E0E887ABA1BCA1EC91E07121F06F
:1040220011960E94CECD07C0ABA1BCA11196ED9115
:10403200FD9166277727E987FA876B877C87FE01E0
:104042003E96FA93EA93EDA1FEA13596FA93EA938E
:10405200A989BB270E9449C5DE0116960E94BA9221
:104062000E9463CCA59608951A930A93AEE6B2E035
:104072000E9453CE0E2F003029F0A02F0E948A3BBF
:10408200E03021F0E0916304E06403C0E091630456
:10409200EF7BE093630410E0E0916A041E1708F0DE
:1040A2007DC0ABE6B4E0E12FF0E0BD01AEE0B0E0F0
:1040B2000E9411CDDB01AE0FBF1F1D96AC91A13046
:1040C20008F46AC0ABE6B4E0E12FF0E0BD01AEE077
:1040D200B0E00E9411CDDB01AE0FBF1F1D96EC9127
:1040E200E150EC93ABE6B4E0E12FF0E0BD01AEE0CD
:1040F200B0E00E9411CDDB01AE0FBF1F1D96EC9107
:10410200E03009F049C0ABE6B4E0E12FF0E0BD01D8
:10411200AEE0B0E00E9411CDDB01AE0FBF1F1C96D6
:10412200EC91F0E00E94ECCCE370F070309781F4F7
:10413200ABE6B4E0E12FF0E0BD01AEE0B0E00E94FA
:1041420011CDDB01AE0FBF1F1C96EC91EF7713C0B0
:10415200E130A0E0FA0701F5ABE6B4E0E12FF0E0D0
:10416200BD01AEE0B0E00E9411CDDB01AE0FBF1F7A
:104172001C96EC91E068EC93ABE6B4E0E12FF0E042
:10418200BD01AEE0B0E00E9411CDDB01AE0FBF1F5A
:104192001C96EC91EF7BEC931F5F7ECFA09169049C
:1041A200A13000F1E0916904E150E0936904EF5F0E
:1041B200E0916904E030B1F4E0916404F0E0F69536
:1041C200E795E370F070309721F4E0916404E77FA3
:1041D20007C0E130A0E0FA0729F4E0916404E86046
:1041E200E09364040C94F625A0971A93A1E4B1E03D
:1041F200E0E0F0E060E070E00E945FCEACE6B2E0AA
:10420200E4EFF1E00E9467CEAEE6B2E0E0E00E94A9
:104212006FCEAFE6B2E00E946FCEA7E7B2E0E0E178
:104222000E946FCEA0E7B2E0E5E00E946FCEA1E768
:10423200B2E0E0E0F0E060E070E00E945FCEA5E76F
:10424200B2E00E9453CEE1600E946FCEFE017196F1
:10425200FA93EA93E0E0EA93A0E1B0E00E945BC542
:10426200FE013196FA93EA93E0E0EA93A0E1B0E02E
:104272000E945BC510E0143308F046C1ABE7B2E020
:10428200E12FF0E0BD01AEE0B0E00E9411CDDB0114
:10429200AE0FBF1FE0E0F0E060E070E00E945FCE92
:1042A200ABE7B2E0E12FF0E0BD01AEE0B0E00E948A
:1042B20011CDDB01AE0FBF1F1496E0E0F0E00E94CB
:1042C20067CEABE7B2E0E12FF0E0BD01AEE0B0E0D7
:1042D2000E9411CDDB01AE0FBF1F1696E0E0F0E0A9
:1042E2000E9467CEABE7B2E0E12FF0E0BD01AEE0A5
:1042F200B0E00E9411CDDB01AE0FBF1F1896EFEFA9
:10430200FFEF0E9467CEABE7B2E0E12FF0E0BD0124
:10431200AEE0B0E00E9411CDDB01AE0FBF1F1A96D6
:104322000E9453CEE07FE6600E946FCEABE7B2E020
:10433200E12FF0E0BD01AEE0B0E00E9411CDDB0163
:10434200AE0FBF1F1A960E9453CEEF78E0620E9412
:104352006FCEABE7B2E0E12FF0E0BD01AEE0B0E03E
:104362000E9411CDDB01AE0FBF1F1A960E9453CEE1
:10437200EF770E946FCEABE7B2E0E12FF0E0BD0134
:10438200AEE0B0E00E9411CDDB01AE0FBF1F1C9664
:104392000E9453CEEE7F0E946FCEABE7B2E0E12FD8
:1043A200F0E0BD01AEE0B0E00E9411CDDB01AE0F46
:1043B200BF1F1B960E9453CEE07F0E946FCEABE7D9
:1043C200B2E0E12FF0E0BD01AEE0B0E00E9411CD1D
:1043D200DB01AE0FBF1F1B960E9453CEEF700E94EF
:1043E2006FCEABE7B2E0E12FF0E0BD01AEE0B0E0AE
:1043F2000E9411CDDB01AE0FBF1F1C960E9453CE4F
:10440200ED7F0E946FCEABE7B2E0E12FF0E0BD019D
:10441200AEE0B0E00E9411CDDB01AE0FBF1F1C96D3
:104422000E9453CEE37F0E946FCEABE7B2E0E12F52
:10443200F0E0BD01AEE0B0E00E9411CDDB01AE0FB5
:10444200BF1F1C960E9453CEEF7E0E946FCEABE739
:10445200B2E0E12FF0E0BD01AEE0B0E00E9411CD8C
:10446200DB01AE0FBF1F1C960E9453CEEF710E945C
:104472006FCEABE7B2E0E12FF0E0BD01AEE0B0E01D
:104482000E9411CDDB01AE0FBF1F1D96E0E00E941E
:104492006FCEFE017196FA93EA93EFE1F2E060E0EB
:1044A20070E00E94E5CDE12FF0E031966F2F660FAC
:1044B200660B762F0E94E5CD84E00E94A8CB2A9657
:1044C200E12FF0E0A0E6BBE30E94D6CCEA0FFB1F8F
:1044D200FA93EA93FE017396FA93EA93A0E10E949B
:1044E200C428E12FF0E0A0EABEE30E94D8CCEA0F94
:1044F200FB1FFA93EA93FE013396FA93EA93A8E03C
:104502000E94C4281F5FB7CE0E942B171881A19664
:1045120008951A93E3E4F7E0FA93EA93E0E0EA936A
:10452200ACE3B0E00E945BC510E0143108F040C07B
:10453200AEEBB6E0E12FF0E0BD01A6E0B0E00E94F4
:1045420011CDDB01AE0FBF1F0E9453CEE03071F1DF
:10455200A3E01A9FF001ED5BF84FDF01EC91E160FF
:10456200EC93A3E01A9FF001ED5BF84FFF93EF93FA
:10457200AEEBB6E0E12FF0E0BD01A6E0B0E00E94B4
:1045820011CDDB01AE0FBF1F12960E944FCEDF018D
:10459200EEE00E9497CCE370AF91BF91E370E29599
:1045A200E07F0E2EEC91EF7CE029EC931F5FBDCFF4
:1045B200199108950E945CCC10E0143108F013C2E6
:1045C200A3E01A9FF001ED5BF84FE081E17009F47E
:1045D20008C2AEEBB6E0E12FF0E0BD01A6E0B0E02C
:1045E2000E9411CDDB01AE0FBF1F0E9453CEAE2F32
:1045F2000E948A3B0E2FA3E01A9FF001ED5BF84F59
:10460200E081F0E00E94E8CCE370F070309709F0AE
:104612007AC0003009F45BC01A9FF001ED5BF84FDD
:10462200E081E47009F052C0AEEBB6E0E12FF0E0B9
:10463200BD01A6E0B0E00E9411CDDB01AE0FBF1FAD
:1046420012960E944FCEFF73AF0100240416050696
:1046520088F4A3E01A9FF001ED5BF84FDF01EC91C3
:10466200E860EC93A3E01A9FF001EC5BF84F408303
:1046720051832CC0A3E01A9FF001ED5BF84FDF01DC
:10468200EC91E77FEC93A3E01A9FF001ED5BF84F0A
:10469200DF01EC91E260EC93A3E01A9FF001EC5B86
:1046A200F84FFF93EF93AEEBB6E0E12FF0E0BD01E0
:1046B200A6E0B0E00E9411CDDB01AE0FBF1F149641
:1046C2000E944FCEAF91BF91ED93FC931BC0A3E02C
:1046D2001A9FF001EC5BF84FA0E0B0E0A083B18339
:1046E200A3E01A9FF001ED5BF84FDF01EC91E77F49
:1046F200EC93A3E01A9FF001ED5BF84FDF01EC9120
:10470200ED7FEC931DC1E130A0E0FA0709F063C030
:10471200A091900DAB3008F413C1003041F4A3E036
:104722001A9FF001ED5BF84FE081E47009F452C08A
:10473200AEEBB6E0E12FF0E0BD01A6E0B0E00E94F2
:1047420011CDDB01AE0FBF1F12960E944FCEFF7339
:10475200AF0100240416050688F4A3E01A9FF001B5
:10476200ED5BF84FDF01EC91E860EC93A3E01A9F58
:10477200F001EC5BF84F408351832CC0A3E01A9FF9
:10478200F001ED5BF84FDF01EC91E860EC93A3E000
:104792001A9FF001ED5BF84FDF01EC91E260EC93C0
:1047A200A3E01A9FF001EC5BF84FFF93EF93AEEB9F
:1047B200B6E0E12FF0E0BD01A6E0B0E00E9411CD2D
:1047C200DB01AE0FBF1F14960E944FCEAF91BF9177
:1047D200ED93FC93B5C0E230A0E0FA0709F05EC0A9
:1047E200003041F0A3E01A9FF001ED5BF84FE08149
:1047F200E47009F052C0AEEBB6E0E12FF0E0BD018B
:10480200A6E0B0E00E9411CDDB01AE0FBF1F1296F1
:104812000E944FCEFF73AF0100240416050688F4F0
:10482200A3E01A9FF001ED5BF84FDF01EC91E86025
:10483200EC93A3E01A9FF001EC5BF84F40835183A5
:104842002CC0A3E01A9FF001ED5BF84FDF01EC9161
:10485200E860EC93A3E01A9FF001ED5BF84FDF01F3
:10486200EC91E260EC93A3E01A9FF001EC5BF84F4D
:10487200FF93EF93AEEBB6E0E12FF0E0BD01A6E0CF
:10488200B0E00E9411CDDB01AE0FBF1F14960E9453
:104892004FCEAF91BF91ED93FC9352C0E330A0E0B5
:1048A200FA0709F04DC0A091900DAB3008F448C052
:1048B200003099F0A3E01A9FF001ED5BF84FDF01A1
:1048C200EC91E260EC93A3E01A9FF001EC5BF84FED
:1048D200A0E0B0E0A083B18333C0A3E01A9FF0014F
:1048E200ED5BF84FE081E47059F11A9FF001ED5B46
:1048F200F84FDF01EC91E77FEC93A3E01A9FF00100
:10490200ED5BF84FDF01EC91E260EC93A3E01A9FBC
:10491200F001EC5BF84FFF93EF93AEEBB6E0E12FC3
:10492200F0E0BD01A6E0B0E00E9411CDDB01AE0FC8
:10493200BF1F14960E944FCEAF91BF91ED93FC938F
:10494200A3E01A9FF001ED5BF84FDF01E02FE17069
:10495200EE0FEE0F0E2EEC91EB7FE029EC93AEEB17
:10496200B6E0E12FF0E0BD01A6E0B0E00E9411CD7B
:10497200DB01AE0FBF1F11960E9453CE3E2F303087
:10498200A1F0A3E01A9FF001ED5BF84FE081E8701F
:1049920039F41A9FF001ED5BF84FE081E27029F0E3
:1049A200A32F0E948A3BE03009F41BC0A3E01A9FA8
:1049B200F001ED5BF84FDF01EC91E77FEC93A3E0B0
:1049C2001A9FF001ED5BF84FDF01EC91ED7FEC9364
:1049D200A3E01A9FF001EC5BF84FA0E0B0E0A083E7
:1049E200B1831F5FEACD0E9463CC49C11A9310E0E4
:1049F200143108F069C0A3E01A9FF001ED5BF84F93
:104A0200E081E17061F01A9FF001EC5BF84FDF0189
:104A1200ED91FC91119700240E160F0608F052C07A
:104A2200A3E01A9FF001EC5BF84FDF01ED91FD91DD
:104A32003197FE93EE93A3E01A9FF001EC5BF84FDF
:104A4200DF01ED91FC9111973097E1F5A3E01A9FF8
:104A5200F001ED5BF84FE081E87059F11A9FF00127
:104A6200ED5BF84FDF01EC91E77FEC93A3E01A9F37
:104A7200F001EC5BF84FFF93EF93AEEBB6E0E12F62
:104A8200F0E0BD01A6E0B0E00E9411CDDB01AE0F67
:104A9200BF1F14960E944FCEAF91BF91ED93FC932E
:104AA200A3E01A9FF001ED5BF84FDF01EC91E260A9
:104AB20008C0A3E01A9FF001ED5BF84FDF01EC9113
:104AC200ED7FEC931F5F94CF0C949F2A60971A930B
:104AD200FE013196FA93EA93E0E0EA93A0E1B0E0B6
:104AE2000E945BC510E0143108F047C0FE01319608
:104AF200FA93EA93E0E0EA93A6E0B0E00E945BC595
:104B0200AEEBB6E0E12FF0E0BD01A6E0B0E00E941E
:104B120011CDE60FF71FFA93EA93FE013396FA934B
:104B2200EA93A6E080D0FE013196FA93EA93E6E298
:104B3200F2E060E070E00E94E5CDE12FF0E0319616
:104B42006F2F660F660B762F0E94E5CD84E00E94E0
:104B5200A8CB2A96E12FF0E0A0E1B1E40E94D6CCE6
:104B6200EA0FFB1FFA93EA93FE013396FA93EA9354
:104B72000E94C428A8951F5FB6CF18816196089538
:104B82001A930A93E6E3F2E060E070E00E94E5CD5A
:104B920080E00E94E3CB24960FE010E0E5E4F1E030
:104BA2000E171F0738F4D801E0E00E946FCE0F5FA6
:104BB2001F4FF4CF0E944B2DA0E0B0E0E0E50E9431
:104BC2006FCEA1E0B0E0E3E40E946FCEA2E0B0E0DD
:104BD200EDE40E946FCEA3E0B0E0E0E50E946FCE6C
:104BE200A4E0B0E0E0E00E946FCE0991199108952F
:104BF2000E945CCC0A2F2E813F814885598510E0A6
:104C0200101778F4E12FF0E0E40FF51F0F01D9013E
:104C1200EE27A10FBE1F0E9453CED001EC931F5F5F
:104C2200EFCF0C94CA290E945CCC0A2F2E813F81BF
:104C32004885598510E0101778F4E12FF0E0E40F71
:104C4200F51F0F01D901EE27A10FBE1FEC91D00174
:104C52000E946FCE1F5FEFCF9CC30E945ECC0A2FD3
:104C62002C813D8110E0101740F4D901EE27A10FED
:104C7200BE1F0E946FCE1F5FF6CF0E9465CC2696A4
:104C820008950E945CCC3A2F4E815F8110E0E32FA1
:104C9200F0E03197A12FB0E0AE17BF078CF4DA0134
:104CA200EE27A10FBE1F0C91003051F0A885B985E7
:104CB200EE27A10FBE1FE02F0E946FCE1F5FE7CF2E
:104CC200A885B985EE27A10FBE1F0E946FCEE12FE6
:104CD20060C30E945CCC3A2F4E815F8110E0E32FCB
:104CE200F0E03197A12FB0E0AE17BF0794F4DA01DC
:104CF200EE27A10FBE1F0E9453CE0E2F003049F0A7
:104D0200E12FA885B985F0E0EA0FFB1F00831F5F42
:104D1200E6CFA885B985EE27A10FBE1FEC93E12F40
:104D220038C32E97D1500E945ECC10E0133030F57C
:104D3200FE01E250FF4FFA93EA93E0E0F0E0FA93CB
:104D4200EA93A4E1B0E06CD1E03089F0E0918B0D00
:104D5200EE7FE0938B0DFE01E250FF4FFA93EA9350
:104D6200ACEBB3E00E946BC5E03041F005C0E091CE
:104D72008B0DE160E0938B0D1F5FD8CF133011F4E0
:104D82002CD194C0E0E0F0E0E093CC03F093CD03AB
:104D920020E030E0283EE3E03E0708F059C0203D25
:104DA200E3E03E0710F409E103C0E8EEE21B0E2F38
:104DB200FE013496FA93EA93E091CA03F091CB0391
:104DC20060E870E0AAE0B0E00E9411CDE60FF71FA4
:104DD200FA93EA93EAE0E09FF001DF0121D1E030AB
:104DE200A1F110E0101788F52F5F3F4FAAE01A9F3C
:104DF200F001DE011496AE0FBF1F1696EC91E03063
:104E020021F1AAE01A9FF001DE011496AE0FBF1F36
:104E1200ED91FD91A091CC03B091CD03AE17BF07E8
:104E220090F4AAE01A9FF001DE011496AE0FBF1FA4
:104E3200ED91FC911197E093CC03F093CD03209375
:104E4200CA033093CB031F5FCDCF101708F0A2CF58
:104E5200ACECB3E0ED91FD913196FE93EE93A0910F
:104E6200CA03B091CB03A83EE3E0BE0728F0E0E01E
:104E7200E093CA03E093CB03EDE4F2E060E070E07C
:104E82000E94E5CDE091CA03F091CB036627772714
:104E92000E94E5CDE091CC03F091CD036627772700
:104EA2000E94E5CD88E00E94E3CB2C960E9465CC5F
:104EB2006296DF5F08951A931A2F1A93E0E0EA933D
:104EC200A0E0B0E001D03AC32A970E945CCC9D01D9
:104ED20008895989E2E6F2E060E070E00E94E5CDDF
:104EE200E52FFF27662777270E94E5CDE02FFF27D2
:104EF200662777270E94E5CD88E00E94E3CB2C96B7
:104F0200543638F0ABE7B9E00E944FCE31960E949A
:104F120067CEE091CC03F091CD03EE83FF83E09165
:104F2200F410F091F5106091F6107091F710E88787
:104F3200F9876A877B875C870D872E873F8710E01A
:104F42001330A0F5E091CA03F091CB0360E870E062
:104F5200AAE0B0E00E9411CDE60FF71FFA93EA93A0
:104F6200FE013896FA93EA93AAE00DD1E030E1F01F
:104F7200ACECB3E0ED91FD913196FE93EE93AAEC89
:104F8200B3E0ED91FD913196FE93EE93A091CA03A9
:104F9200B091CB03A83EE3E0BE0728F0E0E0E09347
:104FA200CA03E093CB0302C01F5FCACF0E9463CC47
:104FB20062960895E1E0F0E0E093CC03F093CD0334
:104FC200E0E0E093CA03E093CB03E0E8F0E0FA9379
:104FD200EA93A0E1B7E2E1D108956497FE01FA9362
:104FE200EA93E0E0EA93A4E1B0E00E945BC5FE012F
:104FF200FA93EA93A6E4B2E080E090E00E94A3C5AF
:10500200E2E0E887EDE0E987E0E0F0E0FA93EA9396
:10501200FE013296FA93EA93A4E1B5D0649608951C
:105022000E945CCCAD0110E01436C0F41298EDB5CC
:10503200E093820DE5E0EEBDEDB5E7FFFDCFE0E0E8
:10504200EEBDEDB5E7FFFDCF0EB5129A00FF06C02B
:1050520080E991E00197F1F71F5FE6CF143659F42A
:10506200E885F985FA93EA93E0E0EA93DA010E948F
:105072005BC5E0E08EC11298EDB5E093820DE3E0EE
:10508200EEBDEDB5E7FFFDCFEF81F070EEBDEDB502
:10509200E7FFFDCFEE81EEBDEDB5E7FFFDCF20E0EE
:1050A20030E02417350788F4EDB5E093820DE0E097
:1050B200EEBDEDB5E7FFFDCFA885B985A20FB31F01
:1050C200EEB5EC932F5F3F4FECCF129A61C10E9475
:1050D2005CCC2A2F4E815F8110E01436C0F4129806
:1050E200EDB5E093820DE5E0EEBDEDB5E7FFFDCF56
:1050F200E0E0EEBDEDB5E7FFFDCF3EB5129A30FF21
:1051020006C080E991E00197F1F71F5FE6CF143600
:1051120029F4A885B985E0E0EC933BC1213008F081
:1051220021501298EDB5E093820DE3E0EEBDEDB5AE
:10513200E7FFFDCFE52FF070EEBDEDB5E7FFFDCF48
:105142004EBDEDB5E7FFFDCF00E00217A0F4EDB5CF
:10515200E093820DE0E0EEBDEDB5E7FFFDCFA8855F
:10516200B985EE27A00FBE1FEEB5EC93EEB5E03089
:1051720011F00F5FEACF129AA885B985EE27A00F2A
:10518200BE1FEC9305C10E945CCC5A2F10E0513037
:1051920008F47AC000E00436C0F41298EDB5E0934A
:1051A200820DE5E0EEBDEDB5E7FFFDCFE0E0EEBD3F
:1051B200EDB5E7FFFDCF3EB5129A30FF06C080E99C
:1051C20091E00197F1F70F5FE6CF043611F4E0E0CA
:1051D200E0C01298EDB5E093820DE6E0EEBDEDB5CC
:1051E200E7FFFDCF129A000000001298EDB5E093A0
:1051F200820DE5E0EEBDEDB5E7FFFDCFE0E0EEBDEF
:10520200EDB5E7FFFDCF3EB5129A31FF3AC0E88512
:10521200EF77A0E8AE1B2A2F521708F4252F129819
:10522200EDB5E093820DE2E0EEBDEDB5E7FFFDCF17
:10523200E985F070EEBDEDB5E7FFFDCFE885EEBD87
:10524200EDB5E7FFFDCF00E0021780F4EDB5E09386
:10525200820DAE81BF81EE27A10FBE1FEC91EEBD84
:10526200EDB5E7FFFDCF0F5F1F5FEECF129A521B26
:10527200E22FF0E0A885B985EA0FFB1FE887F987DE
:1052820002C0E0E086C083CF83C00E945CCC5A2F6C
:1052920010E0513008F47CC000E00436C0F41298EB
:1052A200EDB5E093820DE5E0EEBDEDB5E7FFFDCF94
:1052B200E0E0EEBDEDB5E7FFFDCF3EB5129A30FF5F
:1052C20006C080E991E00197F1F70F5FE6CF04365F
:1052D20011F4E0E05EC01298EDB5E093820DE6E0D5
:1052E200EEBDEDB5E7FFFDCF129A00000000129867
:1052F200EDB5E093820DE5E0EEBDEDB5E7FFFDCF44
:10530200E0E0EEBDEDB5E7FFFDCF3EB5129A31FF0D
:105312003CC0E885EF77A0E8AE1B2A2F521708F4AD
:10532200252F1298EDB5E093820DE2E0EEBDEDB5CA
:10533200E7FFFDCFE985F070EEBDEDB5E7FFFDCFEC
:10534200E885EEBDEDB5E7FFFDCF00E0021780F482
:10535200AE81BF81EE27A10FBE1F3C91EDB5E09358
:10536200820D3EBDEDB5E7FFFDCF0F5F1F5FEECFB4
:10537200129A303069F0521BE22FF0E0A885B9850D
:10538200EA0FFB1FE887F98702C0E0E002C081CF85
:10539200E1E00E9463CC2A9608950E945CCCAD01A4
:1053A20010E000240416050608F07BC000E0043675
:1053B200C0F41298EDB5E093820DE5E0EEBDEDB5D7
:1053C200E7FFFDCFE0E0EEBDEDB5E7FFFDCF3EB577
:1053D200129A30FF06C080E991E00197F1F70F5F62
:1053E200E6CF043611F4E0E05DC01298EDB5E0932B
:1053F200820DE6E0EEBDEDB5E7FFFDCF129A0000AB
:1054020000001298EDB5E093820DE5E0EEBDEDB53A
:10541200E7FFFDCFE0E0EEBDEDB5E7FFFDCF3EB526
:10542200129A31FF3BC0EE81EF77A0E8AE1B2A2F24
:10543200FA01B0E0EA17FB0708F4242F1298EDB541
:10544200E093820DE2E0EEBDEDB5E7FFFDCFEF8127
:10545200F070EEBDEDB5E7FFFDCFEE81EEBDEDB52F
:10546200E7FFFDCF00E0021758F4EDB5E093820D9F
:10547200E0E0EEBDEDB5E7FFFDCF0F5F1F5FF3CFBD
:10548200129AA22FBB274A1B5B0BE22FF0E0AE81E0
:10549200BF81EA0FFB1FEE83FF8302C0E0E002C080
:1054A20080CFE1E00E9463CC289608951A93EFE73B
:1054B200F7E0FA93EA93E0E0EA93A4E1B0E00E9415
:1054C2005BC510E01530D0F5E12FAFE7B7E0F0E0B3
:1054D2000E94DACCEA0FFB1F0F01AAE8B6E0E12F27
:1054E200F0E00E94DACCAE0FBF1F0E9453CED00173
:1054F200EC93E12FAFE7B7E0F0E00E94DACCEA0FDD
:10550200FB1F33960F01AAE8B6E0E12FF0E00E94FC
:10551200DACCAE0FBF1F13960E9453CEEE1FE0E00F
:10552200EE1FE170D001E170EE0FEE0FEE0F0E2EC6
:10553200EC91E77FE029EC931F5FC4CF19910895A6
:105542000E945ECC2A2F10E0153008F0CFC1E12F67
:10555200AFE7B7E0F0E00E94DACCAE0FBF1FAC912C
:10556200A03081F0E12FAFE7B7E0F0E00E94DACCA3
:10557200AE0FBF1F1396EC91E695E695E695E170A6
:105582002E1709F0B1C1E12FAFE7B7E0F0E00E94BA
:10559200DACCAE0FBF1FAC910E948A3BE03009F417
:1055A20079C0E12FAFE7B7E0F0E00E94DACCAE0FAE
:1055B200BF1F1396EC91E47009F06BC0E12FAFE7C7
:1055C200B7E0F0E00E94DACCAE0FBF1F1396EC9169
:1055D200E160EC93E12FAFE7B7E0F0E00E94DACCB4
:1055E200AE0FBF1F1396EC91E460EC93E12FAFE78F
:1055F200B7E0F0E00E94DACCEA0FFB1F33960F010E
:10560200AAE8B6E0E12FF0E00E94DACCAE0FBF1FAD
:1056120013960E9453CEEF77E13010F0E1E001C023
:10562200E0E0D001E170EE0F0E2EEC91ED7FE0296B
:10563200EC93E12FAFE7B7E0F0E00E94DACCEA0F9B
:10564200FB1F32960F01AAE8B6E0E12FF0E00E94BC
:10565200DACCAE0FBF1F13960E9453CEEF77D00164
:10566200EC93E12FAFE7B7E0F0E00E94DACCEA0F6B
:10567200FB1F31960F01AAE8B6E0E12FF0E00E948D
:10568200DACCAE0FBF1F11960E9453CED001EC931D
:105692002BC12FC0E12FAFE7B7E0F0E00E94DACCD8
:1056A200AE0FBF1F1396EC91EB7FEC93E12FAFE7A8
:1056B200B7E0F0E00E94DACCAE0FBF1F1396EC9178
:1056C200E270B9F4E12FAFE7B7E0F0E00E94DACC84
:1056D200AE0FBF1F1396EC91EE7FEC93E12FAFE775
:1056E200B7E0F0E00E94DACCAE0FBF1F1196E0E007
:1056F200EC93E12FAFE7B7E0F0E00E94DACCAE0F17
:10570200BF1F1196AC91A13008F4EEC0E12FAFE7B4
:10571200B7E0F0E00E94DACCAE0FBF1F1196EC9119
:10572200E150EC93E12FAFE7B7E0F0E00E94DACC72
:10573200AE0FBF1F1196EC91E03009F0D5C0E12FFA
:10574200AFE7B7E0F0E00E94DACCAE0FBF1F1396CE
:10575200EC91E17009F48CC0EEE6F2E060E070E0FA
:105762000E94E5CDE12FF0E031966F2F660F660BB8
:10577200762F0E94E5CD84E00E94E3CB2896E12FAC
:10578200AFE7B7E0F0E00E94DACCAE0FBF1F13968E
:10579200EC91EE7FEC93E12FAFE7B7E0F0E00E94EF
:1057A200DACCAE0FBF1F1396EC91E27009F442C03F
:1057B200E12FAFE7B7E0F0E00E94DACCAE0FBF1FF7
:1057C2001296AC91A130A8F1E12FAFE7B7E0F0E07B
:1057D2000E94DACCAE0FBF1F1296EC91E150EC930F
:1057E200E12FAFE7B7E0F0E00E94DACCAE0FBF1FC7
:1057F2001296AC91A130E8F0AAE8B6E0E12FF0E011
:105802000E94DACCAE0FBF1F12960E9453CE0E2F0B
:10581200E295EF70E695E6953E2F031BE6950E1B8B
:10582200E12FAFE7B7E0F0E00E94DACCEA0FFB1F0E
:1058320001831DC0AAE8B6E0E12FF0E00E94DACCB5
:10584200AE0FBF1F12960E9453CE0E2FE295EF703D
:10585200E695E6953E2F031BE6950E1BE12FAFE77B
:10586200B7E0F0E00E94DACCEA0FFB1F01833CC0F4
:10587200E6E7F2E060E070E00E94E5CDE12FF0E0C3
:1058820031966F2F660F660B762F0E94E5CD84E06E
:105892000E94E3CB2896E12FAFE7B7E0F0E00E9449
:1058A200DACCAE0FBF1F1396EC91E160EC93AAE83D
:1058B200B6E0E12FF0E00E94DACCAE0FBF1F1196E6
:1058C2000E9453CE0E2FE295EF70E695E6953E2F9D
:1058D200031BE6950E1BE12FAFE7B7E0F0E00E9455
:1058E200DACCEA0FFB1F01831F5F2ECEC5C1609782
:1058F2001A93FE013196FA93EA93E0E0EA93A0E16B
:10590200B0E00E945BC510E0153008F069C0AAE85B
:10591200B6E0E12FF0E00E94DACCAE0FBF1FE0E06C
:105922000E946FCEAAE8B6E0E12FF0E00E94DACC46
:10593200AE0FBF1F1196E5E00E946FCEAAE8B6E057
:10594200E12FF0E00E94DACCAE0FBF1F1296E5E025
:105952000E946FCEAAE8B6E0E12FF0E00E94DACC16
:10596200AE0FBF1F13960E9453CEE0780E946FCEF7
:10597200AAE8B6E0E12FF0E00E94DACCAE0FBF1F3A
:1059820013960E9453CEEF770E946FCEFE0131969E
:10599200FA93EA93EDE7F2E060E070E00E94E5CD71
:1059A200E12FF0E031966F2F660F660B762F0E9483
:1059B200E5CD84E00E94A8CB2A96E12FF0E0A0E496
:1059C200B0E40E94D6CCEA0FFB1FFA93EA93FE01E1
:1059D2003396FA93EA93A0E10E94C4281F5F94CF02
:1059E20065DD22C1E0E0E2B9EFEFE1B9E1E0E5B95E
:1059F200E7EFE4B9E8E1E8B9EFE9E7B9E5E2EBB9E5
:105A0200E8EBEAB9E2E0EEB9EEE3EDB9E0E0E1BBE2
:105A1200EFE0E0937E00E0EFE0BBE0E0E4BBEFE12B
:105A2200E3BBE1E5ECBDE1E0EDBDE6E0E093C20001
:105A3200E8E9E093C100E0E0E093C500E3E0E09331
:105A4200C400EDE0E4BDE0E0E6BDEFE4E7BDE2E086
:105A5200E0936E000895E0E0E093900D0E94A83577
:105A62000E947A620E94477C0E94B63A0E942B17DB
:105A72000E94070B1BDD0E948A220E948BC20E9499
:105A820005BB0E94F0BC0E94070B0E94D9800E94B5
:105A92000645089560971A9310E01A3048F4A8E179
:105AA200B1E0EE27A10FBE1F0E946FCE1F5FF5CFA0
:105AB200A6E2B1E00E9453CEE07F0E946FCEA6E242
:105AC200B1E00E9453CEEF7E0E946FCEA6E2B1E01B
:105AD2000E9453CEE0620E946FCEA5E2B1E0E0E008
:105AE2000E946FCEA7E2B1E00E946FCEA8E2B1E0C1
:105AF2000E946FCEA9E2B1E00E946FCEAAE2B1E0AD
:105B02000E946FCEABE2B1E00E946FCEACE2B1E098
:105B12000E946FCEADE2B1E0E4E10E946FCEAEE250
:105B2200B1E0E0E00E946FCEAFE2B1E00E946FCE42
:105B3200A0E3B1E00E946FCEA1E3B1E00E946FCE7C
:105B4200FE013196FA93EA93E0E0EA93A0E1B0E035
:105B52000E945BC5FE013196FA93EA93A3ECB3E08F
:105B62000E9496C5E0E0F8E3FA93EA93FE013396C9
:105B7200FA93EA93A0E10E94C428E0E0E983E0E915
:105B8200F4E4FA93EA93FE013396FA93EA93A1E0DE
:105B92000E94C428A2E3B1E0EEE1F0E0FF700F0141
:105BA2000E944FCEE070F07FE029F1290E9467CE7B
:105BB200A4E3B1E0E0E00E946FCEA5E3B1E0EAE049
:105BC2000E946FCEA6E3B1E0E0E80E946FCEA7E3A9
:105BD200B1E00E946FCEE9E3F1E0FA93EA93A7E025
:105BE2000E942E260E94577B0E948A7C0E940E44AD
:105BF2000E94F5200E94A3167ADE0E9467250E9469
:105C02000BC50E9470BC0E9488C10E9425900E9410
:105C1200347A0E9493460E94DB271DDFA8E0B0E0A1
:105C2200E3E00E946FCE6BD11881619608950E94C5
:105C32005ECCA89522E231E000E010E02D37E9E0E9
:105C42003E0748F4D9010E9453CEF0E00E0F1F1F09
:105C52002F5F3F4FF3CFE3E9F2E060E070E00E9494
:105C6200E5CDF801662777270E94E5CD84E00E9402
:105C7200E3CB2896A895F8010E9465CC2496089556
:105C8200EF97EF9726970E945CCCE091910DED7F04
:105C9200E093910DEB7FE093910DE77FE093910DFF
:105CA200E0E0E093930DA8E0B0E00E9453CEE33031
:105CB200B1F5E091910DE260E093910DA2E2B1E0C5
:105CC2000E9453CEE13039F5E091910DE460E0930A
:105CD200910DADDFAF01A3E2B1E00E944FCEE887A4
:105CE200F987E985F0E0F0E04E1B5F0BE885F98566
:105CF200F0E0F0E04E1B5F0BE885F985E417F5074D
:105D020031F4E091910DE860E093910D03C0E4E07D
:105D1200E093930D03C0E2E0E093930D03C0E1E052
:105D2200E093930D30E040E050E0E2E2F1E0EE83F8
:105D3200FF83AE81BF81AD37E9E0BE0708F04BC0FB
:105D4200EDE7F9E0EA1BFB0BE138A0E0FA0710F0FF
:105D520010E804C0AE81EDE7EA1B1E2FFE013A9661
:105D6200FA93EA93E2E2F1E0A0E0B8E20E94F5CD14
:105D7200EA1BFB0BA885B985EA0FFB1FFA93EA938E
:105D8200A12FBB270E941128303071F4AA85A130BF
:105D920031F0E091930DE061E093930D1CC0EB852F
:105DA200FC85E887F98731E000E0011760F4E02F15
:105DB200F0E0DE011A96AE0FBF1FEC91F0E04E0F3D
:105DC2005F1F0F5FF2CFA895EE81FF81E058FF4F72
:105DD200EE83FF83AECF313009F08BC0E985F0E06E
:105DE200F0E04E1B5F0BE885F985F0704E1B5F0BF0
:105DF200E885F985E417F50709F076C0E091910D81
:105E0200E87009F070C0AFEFBFE00E9453CEEF5FC1
:105E12000E946FCEE091930DE064E093930DE2E275
:105E2200F1E0EE83FF83AE81BF81AD37E9E0BE07CB
:105E3200B8F5EDE7F9E0EA1BFB0BE138A0E0FA0761
:105E420010F010E804C0AE81EDE7EA1B1E2FFE0140
:105E52003A96FA93EA93E2E2F1E0A0E0B8E20E9415
:105E6200F5CDEA1BFB0BA885B985EA0FFB1FFA9358
:105E7200EA93A12FBB270E941128EE81FF81FA939A
:105E8200EA93FE013C96FA93EA93A12F0E9414260C
:105E9200A895EE81FF81E058FF4FEE83FF83C3CFC9
:105EA200C6DEAF01A3E2B1E00E944FCEE887F987D8
:105EB200E985F0E0F0E04E1B5F0BE885F985F0E044
:105EC200F0E04E1B5F0BE885F985E417F50731F426
:105ED200E091910DE860E093910D05C0E091930D82
:105EE200E068E093930D05C0E091930DE062E093CA
:105EF200930D0E9463CCEF96EF962C960895EF9740
:105F0200EF9724970E945CCCE0EAF2E060E070E058
:105F12000E94E5CD80E00E94E3CB2496A2E2B1E0AC
:105F2200E1E00E946FCEA3E2B1E0E0E0F0E00E9487
:105F320067CE7DDEAF01A3E2B1E00E944FCEEE83D9
:105F4200FF83EF81F0E0F0E04E1B5F0BEE81FF81FB
:105F5200F0E0F0E04E1B5F0BA3E2B1E0FA010E9419
:105F620067CE22E231E02D37E9E03E0760F5EDE74A
:105F7200F9E0E21BF30BE138A0E0FA0710F010E8B9
:105F820003C0EDE7E21B1E2FFE013896FA93EA9357
:105F92003A932A93A12F0E94F925E2E2F1E0A0E0D0
:105FA200B8E20E94F5CDEA1BFB0BE20FF31FFA9356
:105FB200EA93FE013A96FA93EA93A12F0E94C4282B
:105FC20020583F4FD0CFE091910DE460E093910DC6
:105FD200E860E093910DE0E0E093930DE091910D84
:105FE200E07129F0E091910DE160E093910D0E9442
:105FF20063CCEF96EF962A960895EF97EF97229744
:106002000E945CCC4A2F403039F5A4E1B0E0E3E7CE
:106012000E946FCEA3E2B0E0E1E00E946FCEA4E264
:10602200B0E0E0E0F0E00E9467CE20E030E004E182
:1060320010E0E8E1F1E00E171F0748F4D8010E94D2
:1060420053CEF0E02E0F3F1F0F5F1F4FF2CFA4E29F
:10605200B0E0F9010E9467CE00E010E00430E1E018
:106062001E0748F5E4E0F1E0E01BF10BE138A0E0A7
:10607200FA0710F050E803C0E4E0E01B5E2FFE01D7
:106082003696FA93EA93E4E1F0E0E00FF11FFA9317
:10609200EA93A52F0E94F925F801E058F140FA93FE
:1060A200EA93FE013896FA93EA93A52F0E94C42838
:1060B20000581F4FD3CF0E9463CCEF96EF962896DD
:1060C20008950E945CCC20E030E004E110E0E8E1B9
:1060D200F1E00E171F0748F4D8010E9453CEF0E0FA
:1060E2002E0F3F1F0F5F1F4FF2CFA4E2B0E00E94BE
:1060F2004FCEAF01E52FF0E0F0E02E1B3F0BFA018F
:10610200F0E0F0E02E1B3F0B4217530711F4E1E0E1
:1061120001C0E0E00E9463CC26960895EF97EF97C6
:1061220025970E945CCCE0E0DE01A957BF4FEC93BB
:10613200DE01A957BF4FAC91AA3020F5A8E1B1E02A
:10614200FE01E957FF4FE081F0E0AE0FBF1F0E9452
:1061520053CEDE01A857BF4FEC93DE01A857BF4FC5
:10616200AC91A03210F0AB3730F0A8E1B1E0E0E042
:106172000E946FCE07C0DE01A957BF4FEC91EF5FBF
:10618200EC93D6CFE091910DEF7EE093910DE0E09C
:10619200DE01A957BF4FEC93DE01A957BF4FAC9167
:1061A200A53038F5A0E0B0E00E9453CEE035C1F44E
:1061B200A1E0B0E00E9453CEE33491F4A2E0B0E05B
:1061C2000E9453CEED3461F4A3E0B0E00E9453CEBE
:1061D200E03531F4A4E0B0E00E9453CEE03009F0A3
:1061E20001C007C0DE01A957BF4FEC91EF5FEC93EE
:1061F200D3CFDE01A957BF4FAC91A53039F40E942D
:10620200C125E091920DE160E093920DA3E2B0E02E
:106212000E9453CEE03061F4A4E2B0E00E944FCE7F
:10622200309731F4A2E2B0E00E9453CEEF3109F090
:1062320008C0E091920DE260E093920DA0E0DDDEF5
:106242000EC03FDFE03031F0E091910DE061E0936C
:10625200910D05C0E091920DE460E093920DE0E0B3
:10626200DE01AA57BF4FEC93E0E0F0E08F019F01FF
:106272000430E1E01E0708F061C0E4E0F1E0E01B59
:10628200F10BE138A0E0FA0710F0E0E802C0E4E028
:10629200E01BDE01A857BF4FEC93FE013696FA933E
:1062A200EA93F801E058F140FA93EA93DE01A45729
:1062B200BF4FAC91BB270E941128FE01EA57FF4F46
:1062C200E081E030A9F4AE81A33719F4AD89A130A1
:1062D20009F008C04E895F89E1E0DE01AA57BF4F8D
:1062E200EC9306C0E091920DE860E093920D26C017
:1062F200E0E0DE01A957BF4FEC93FE01E857FF4FE4
:10630200E081DE01A957BF4FAC91AE17A0F4FE01A8
:10631200E957FF4FE081F0E0DE011696AE0FBF1F96
:10632200EC91F0E02E0F3F1FDE01A957BF4FEC9119
:10633200EF5FEC93E2CF00581F4F9ACFE52FF0E0CA
:10634200F0E02E1B3F0BFA01F0E0F0E02E1B3F0BBA
:10635200DE01AA57BF4FAC91A13019F4421753077F
:1063620009F059C0E091910DE07109F053C0E0913C
:10637200920DE061E093920D00E010E00430E1E064
:106382001E0798F5EDE7F9E0E01BF10BE138A0E01C
:10639200FA0710F0E0E802C0EDE7E01BDE01A857C3
:1063A200BF4FEC93FE013696FA93EA93F801E05858
:1063B200F140FA93EA93DE01A457BF4FAC91BB2799
:1063C2000E941128E4E1F0E0E00FF11FFA93EA9352
:1063D200FE013896FA93EA93DE01A457BF4FAC91BF
:1063E2000E94142600581F4FC9CF6BDEE03069F0BF
:1063F200E091910DE061E093910DAEEFBFE00E945C
:1064020053CEEF5F0E946FCE05C0E091920DE06225
:10641200E093920D17C0E091920DE064E093920D2B
:10642200E091910DE07171F0A1E0E7DDADEFBFE029
:106432000E9453CEEF5F0E946FCEE091920DE06812
:10644200E093920D0E9463CCEF96EF962B960895FF
:10645200EAEAF2E060E070E00E94E5CDE2E0F0E01E
:1064620060E070E00E94E5CDEDE0F0E060E070E019
:106472000E94E5CDE0E0F0E060E070E00E94E5CD52
:106482008CE00E94E3CB6096E5EDF2E060E070E024
:106492000E94E5CDA5E1B0E00E944FCE66277727A6
:1064A2000E94E5CD84E00E94E3CB2896E1EEF2E083
:1064B20060E070E00E94E5CDA7E1B0E00E9453CE1B
:1064C200FF27662777270E94E5CDA8E1B0E00E946A
:1064D20053CEFF27662777270E94E5CD88E00E94EA
:1064E200E3CB2C96E9EFF2E060E070E00E94E5CDAC
:1064F200E0918D0DFF27662777270E94E5CDE09179
:106502008E0DFF27662777270E94E5CDAAE1B0E02E
:106512000E9453CEFF27662777270E94E5CD8CE0A5
:106522000E94E3CB6096E7E1F3E060E070E00E9456
:10653200E5CDE091F410F091F5106091F6107091B4
:10654200F7100E94E5CD84E00E94E3CB2896E0910B
:10655200910DE27009F444C0E091910DE47031F1C3
:10656200E5E2F3E060E070E00E94E5CDA3E2B1E095
:106572000E944FCE662777270E94E5CD84E00E94D5
:10658200E3CB2896E091910DE87029F0E6E3F3E081
:1065920060E070E004C0EAE3F3E060E070E00E94D3
:1065A200E5CD80E00E94E3CB249619C0E1E4F3E05C
:1065B20060E070E00E94E5CDA2E2B1E00E9453CE1D
:1065C200FF27662777270E94E5CDE1E0F0E060E053
:1065D20070E00E94E5CD88E00E94E3CB2C9619C0C2
:1065E200E6E5F3E060E070E00E94E5CDA8E0B0E00F
:1065F2000E9453CEFF27662777270E94E5CDE3E06E
:10660200F0E060E070E00E94E5CD88E00E94E3CB1C
:106612002C96EBE6F3E060E070E00E94E5CDAFEF90
:10662200BFE00E9453CEFF27662777270E94E5CD61
:10663200ADEFBFE00E9453CEFF27662777270E9467
:10664200E5CDAEEFBFE00E9453CEFF276627772746
:106652000E94E5CD8CE00E94E3CB6096E0E8F3E097
:1066620060E070E00E94E5CDE091920DFF27662781
:1066720077270E94E5CDE091930DFF2766277727C4
:106682000E94E5CD88E00E94E3CB2C960895ABE012
:10669200B0E00E9453CEE0938D0DACE0B0E00E94DA
:1066A20053CEE0938E0D9ED90E94B2917894A1E0D0
:1066B2000E943D370E949226A89530DDE1DAE091F2
:1066C200910DE07121F0E091910DE87009F405C09F
:1066D200E091910DE160E093910DBDD9A091F01090
:1066E200B091F1108091F2109091F310AA3AE5E581
:1066F200BE07E0E08E07EFEF9E0719F4E4B7E0FF74
:106702001AC0EAEAF5E560E07FEFE093F010F0935B
:10671200F1106093F2107093F310E0E0F0E060E0AB
:1067220070E8E093F410F093F5106093F610709314
:10673200F710E093F810A2E3B1E00E944FCEFF7091
:10674200A4E8BDE0FF700F01ED91FD91E070F07FD4
:10675200E029F129FE93EE93E091840DF091850DED
:10676200FF703A9758F4E091840DF091850DE07036
:10677200F07FEA60E093840DF093850DE4B7E3FFC8
:1067820004C0A091F810A03009F002C0A4E006C035
:10679200E4B7E2FF02C0A5E001C0A2E00E945C27CC
:1067A200E0E0E4BFE093F810E3E9F3E060E070E0DA
:1067B2000E94E5CD80E00E94E3CB2496F09A0ED2AF
:1067C200E091EF08E87FE260E093EF08E091630474
:1067D200EF7CE062E0936304E2E0E093D50CE0E05A
:1067E200E093880DA2E3B1E00E944FCEFF70339791
:1067F20070F4A2E3B1E0E3E0F0E0FF700F010E9469
:106802004FCEE070F07FE029F1290E9467CEE0913F
:10681200920DE03049F0EAE0EA93E0E0EA93A091D9
:10682200920DBB270E946527E091930DE03049F05D
:10683200EBE0EA93E0E0EA93A091930DBB270E947C
:106842006527A091E309A03071F4A091CE0AE091EE
:10685200CF0AEA1741F4A0917A00A03021F4A09166
:10686200880DA03009F005C0E1E0E3BF8895E0E0C3
:10687200E3BFA091950DA13060F0E091950DE1503C
:10688200E093950DEF5FE091910DE07211F40E949B
:10689200B50B0E947C05A0913608A43028F00E9416
:1068A200CA3DE0E0E0933608A091880DA13008F4DB
:1068B20028C1E091880DE150E093880DEF5FE5E09B
:1068C200E093950DA0E0F799A1E0E1E0EA2711F449
:1068D200F79801C0F79AF79BE5C00E9491BF0E940A
:1068E200A1C3E091910DE072D9F4E091AB07F0E021
:1068F200E130A0E0FA0719F40E94514811C0E230D9
:10690200A0E0FA0721F0E330A0E0FA0719F40E94B0
:10691200CA5606C0E430A0E0FA0711F40E943B5DBB
:10692200A1E00E94A12AA0E020FCA1E0E1E0EA2788
:10693200E894EE2309F0689420F820FE0FC00E942C
:1069420064BB0E94DB22E091760DE07439F0E091A5
:10695200760DEF7BE093760D0E94D385A091B50D65
:10696200A43030F4E091B50DEF5FE093B50D91C026
:10697200E0E0E093B50DA0E021FCA1E0E1E0EA2730
:10698200E894EE2309F0689421F821FE82C0A895CC
:10699200A091900DAF3F30F4E091900DEF5FE09346
:1069A200900DE150A091940DA13060F0E091940D12
:1069B200E150E093940DEF5FE091940DE03011F41B
:1069C200A0E01BDBA091830DA13030F0E091830D9C
:1069D200E150E093830D16C0E4E0E093830DA5EE51
:1069E200B8E00A2EEC91E695E170A1E0EA27A02D2D
:1069F200E170EE0F0E2EEC91ED7FE029EC93E0E0DA
:106A0200E093E208A0913508A03131F4E0D00E9471
:106A1200D3850E941A6F11C0E0913308EF70E13004
:106A220060F0A3E3B8E080E0EFE00E9419CEE091CD
:106A32003308E061E093330801C0D0D00E949DBECC
:106A42000E9481420E9435200E94CDC4A0E00E9493
:106A5200A12A0E9474120E94F724E091AB07F0E091
:106A6200E130A0E0FA0711F40E943D510E94BD916D
:106A72000E94F30AA091B60DA93030F4E091B60D50
:106A8200EF5FE093B60D05C0E0E0E093B60D0E9423
:106A920017BFE091760DEF7BE093760D0E94E76CD5
:106AA2000E94A537E091890DF0918A0D7096E093CE
:106AB200890DF0938A0DA091890DB0918A0DA533AD
:106AC200ECE0BE07F0F0E091890DF0918A0DE553FC
:106AD200FC40E093890DF0938A0DA4EFB0E1ED91B3
:106AE200FD916D917D91EF5FFF4F6F4F7F4F7E93D1
:106AF2006E93FE93EE930E94CC7C0E94A5790E9435
:106B0200D438E0913308E07121F0A0913508A0312A
:106B120009F009C0E0913308EF7EE093330857D0C3
:106B22000E941A6F5BD00E941B928BCEFFCFEA931A
:106B3200EFB7EA93E1E0E093870DE091880DEF5F14
:106B4200E093880DE150E991EFBFE99118950E9419
:106B52005ECC10E01031B8F5A2E3B0E0E12FF0E036
:106B6200BD01AAE0B0E00E9411CDDB01AE0FBF1F54
:106B72000E944FCE0E94EACC9F012030E1E03E0706
:106B820088F0ECE9F3E060E070E00E94E5CDF90105
:106B9200662777270E94E5CD84E00E94E3CB289602
:106BA2002FEF30E0ADEAB8E0E12FFF276627772725
:106BB200E054FF4F6F4F6BBFE691F0E0EA0FFB1F0F
:106BC20020831F5FC7CF0E9465CC24960895E6E814
:106BD200E0937A00E0E0E09332080895E6E8E0937B
:106BE2007A00E0E9E8B9E0E0E0937C00E093340861
:106BF200E0933508E1E0E0933208E1E4F8E0FA934B
:106C0200EA93E0E0EA93A4E3B0E00E945BC5E9E71F
:106C1200F8E0FA93EA93E0E0EA93AAE1B0E00E9496
:106C22005BC5E3E9F8E0FA93EA93E0E0EA93AAE1CC
:106C3200B0E00E945BC5E7ECF8E0FA93EA93E0E08B
:106C4200EA93AAE1B0E00E945BC5EEEDE0937A0020
:106C5200E0913308E07FE560E093330808950A92FB
:106C62001A928A93AA93BA93EA93FA93EFB7EA93A2
:106C7200E0913208F0E0E130A0E0FA0739F4EFECFD
:106C8200E0937A00E2E0E0933208ECC0E230A0E068
:106C9200FA0709F0E7C046B0E0913408EF5FE093ED
:106CA2003408E150A0913408A731D0F4E0913408BF
:106CB200E770E869E8B9A83010F443980AC0A091D7
:106CC2003408A03110F4449804C0E3E0E0937C005F
:106CD2004798EEECE0937A00E1E0E093320835C0A9
:106CE200A0913408A73161F4E1E0E0937C00E8E987
:106CF200E8B980E58A95F1F7EFECE0937A0025C0D8
:106D0200A0913408A83151F4E2E0E0937C0080E5E0
:106D12008A95F1F7EFECE0937A0017C0E0E9E8B961
:106D2200E0E0E0933408E0937C00EEECE0937A003C
:106D3200E1E0E0933208A0913508A03130F4E0910F
:106D42003508EF5FE0933508E150A0913408A13097
:106D520010F0A83108F02DC0E0913408E770E093FC
:106D6200B70DA7E3B8E0F0E0EA0FFB1F4082E09125
:106D7200B70DE03031F4E0913608EF5FE09336086A
:106D8200E150A9E7B8E0E0913408F0E0AE0FBF1F90
:106D9200EC91E429EC93A3E9B8E0E0913408F0E047
:106DA200EA0FFB1F0F01A081E42DE095EA2BD00131
:106DB200EC93A0913508A03108F054C0ADEAB8E0D8
:106DC200E0913408F0E0AE0FBF1FEC91E093B70DF5
:106DD200E0917800F0917900A091B70DB0E0AE1784
:106DE200BF0798F4A1E4B8E0E0913408F0E0EE0FB8
:106DF200FF1FEA0FFB1F0F01DF01ED91FD91DF0184
:106E0200E0917800F091790011C0A1E4B8E0E0913E
:106E12003408F0E0EE0FFF1FEA0FFB1F0F01DF0146
:106E2200ED91FD91DF01E091B70DF0E0EA0FFB1F5C
:106E3200D001ED93FC93A0913408A13140F4A091CC
:106E42007800B0917900A03FE3E0BE0708F40AC0E1
:106E5200A7ECB8E0E0913408F0E0AE0FBF1FEC9170
:106E6200EF5FEC93E991EFBFF991E991B991A991A3
:106E720089911990099018951A931A2F103041F0A0
:106E82005C988BE08A95F1F75C9A8BE08A95F1F732
:106E92002898EDB5E093820DE0E4EEBDEDB5E7FF95
:106EA200FDCFE5E0EEBDEDB5E7FFFDCFE8E0EEBDDD
:106EB200EDB5E7FFFDCF289AE091E508EF7BE0937F
:106EC200E508A5E7B2E00E9453CEE170A5EEB8E076
:106ED200E170E795E0E0E7950E2EEC91EF77E0297F
:106EE200EC93E091E508E860E093E508E460E09364
:106EF200E5082898EDB5E093820DE0E4EEBDEDB52E
:106F0200E7FFFDCFEAE0EEBDEDB5E7FFFDCFE09193
:106F1200E508EEBDEDB5E7FFFDCF289A2898EDB55F
:106F2200E093820DE0E4EEBDEDB5E7FFFDCFE0E0DA
:106F3200EEBDEDB5E7FFFDCFE4E0EEBDEDB5E7FF59
:106F4200FDCF289A0C94883BA091E208A13030F042
:106F5200E091E208E150E093E20818C0E3E6E09332
:106F6200E2082898EDB5E093820DE0E4EEBDEDB5C0
:106F7200E7FFFDCFEAE0EEBDEDB5E7FFFDCFE09123
:106F8200E508EEBDEDB5E7FFFDCF289AA091E30835
:106F9200A13038F0E091E308E150E093E308EF5FBD
:106FA2002DC0E3E6E093E3082898EDB5E093820D67
:106FB200E2E4EEBDEDB5E7FFFDCFEAE0EEBDEDB5F3
:106FC200E7FFFDCFE091E708EEBDEDB5E7FFFDCFAE
:106FD200289A2898EDB5E093820DE2E4EEBDEDB576
:106FE200E7FFFDCFE0E0EEBDEDB5E7FFFDCFE091BD
:106FF200E608EEBDEDB5E7FFFDCF289AA091E408C3
:10700200A13038F0E091E408E150E093E408EF5F4A
:107012002DC0E3E6E093E4082898EDB5E093820DF5
:10702200E4E4EEBDEDB5E7FFFDCFEAE0EEBDEDB580
:10703200E7FFFDCFE091E908EEBDEDB5E7FFFDCF3B
:10704200289A2898EDB5E093820DE4E4EEBDEDB503
:10705200E7FFFDCFE0E0EEBDEDB5E7FFFDCFE0914C
:10706200E808EEBDEDB5E7FFFDCF289A08950E942E
:107072005ECC589A509AE091EA08E07CE093EA08E4
:10708200E9B1E370E330A9F0E0E0E093BC0010E086
:10709200E9B1E370E33011F01A3008F00AC05898F1
:1070A2008BE08A95F1F7589A8BE08A95F1F71F5F8A
:1070B200EFCFEFE0E093B800E4EAE093BC0020E019
:1070C20030E0E091BC00E07821F42436E0E03E07B5
:1070D20008F003C02F5F3F4FF4CFE091B900E87F83
:1070E200E83009F052C0E0E9E093BB00E4E8E09345
:1070F200BC0020E030E0E091BC00E07821F42436CE
:10710200E0E03E0708F003C02F5F3F4FF4CFE0916D
:10711200B900E87FE831C9F5E1E0E093BB00E4E8BB
:10712200E093BC0020E030E0E091BC00E07821F484
:107132002436E0E03E0708F003C02F5F3F4FF4CF54
:10714200E091B900E87FE83201F5E1E6E093BB00A7
:10715200E4E9E093BC0020E030E0E091BC00E0789C
:1071620021F42436E0E03E0708F003C02F5F3F4FD2
:10717200F4CFE091B900E87FE83239F4E0E0E0933F
:10718200BC00589850980C94C63DE4E9E093BC00CA
:10719200A2E0B0E00E9427D0E0E0E093BC00589863
:1071A20050980C94C63D0E945CCCE091EA08EF73C3
:1071B200E13030F0AAEEB8E080E0EFE30E9419CEB1
:1071C200589A509AE9B1E370E330A9F0E0E0E09315
:1071D200BC0010E0E9B1E370E33011F01A3008F0BE
:1071E2000AC058988BE08A95F1F7589A8BE08A95F5
:1071F200F1F71F5FEFCFE091EA08EF7309F0D1C01A
:10720200E091EA08E07CE560E093EA08EFE0E093D1
:10721200B800E4EAE093BC0020E030E0E091BC007A
:10722200E07821F42436E0E03E0708F003C02F5F47
:107232003F4FF4CFE091B900E87FE83009F088C110
:10724200E0E9E093BB00E4E8E093BC0020E030E03A
:10725200E091BC00E07821F42436E0E03E0708F03B
:1072620003C02F5F3F4FF4CFE091B900E87FE831D0
:1072720009F06EC1E1E0E093BB00E4E8E093BC00FA
:1072820020E030E0E091BC00E07821F42436E0E038
:107292003E0708F003C02F5F3F4FF4CFE091B900E3
:1072A200E87FE83209F054C1E0E6E093BB00E4E88D
:1072B200E093BC0020E030E0E091BC00E07821F4F3
:1072C2002436E0E03E0708F003C02F5F3F4FF4CFC3
:1072D200E091B900E87FE83209F03AC1E4EAE093CC
:1072E200BC0020E030E0E091BC00E07821F42436DC
:1072F200E0E03E0708F003C02F5F3F4FF4CFE0917C
:10730200B900E87FE03109F023C1E0E9E093BB0076
:10731200E4E8E093BC0020E030E0E091BC00E078DB
:1073220021F42436E0E03E0708F003C02F5F3F4F10
:10733200F4CFE091B900E87FE83109F009C1E0E05B
:10734200E093BB00E4E8E093BC0020E030E0E09191
:10735200BC00E07821F42436E0E03E0708F003C0E8
:107362002F5F3F4FF4CFE091B900E87FE83209F098
:10737200EFC0E4E9E093BC0020E030E0E091BC0023
:10738200E07821F42436E0E03E0708F003C02F5FE6
:107392003F4FF4CFE091EA08E07CEE61E093EA0827
:1073A200D6C0E4EAE093BC0020E030E0E091BC000B
:1073B200E07821F42436E0E03E0708F003C02F5FB6
:1073C2003F4FF4CFE091B900E87FE83009F0C0C048
:1073D200E1E9E093BB00E4E8E093BC0020E030E0A8
:1073E200E091BC00E07821F42436E0E03E0708F0AA
:1073F20003C02F5F3F4FF4CFE091B900E87FE03444
:1074020009F0A6C0E4ECE093BC0020E030E0E0919B
:10741200BC00E07821F42436E0E03E0708F003C027
:107422002F5F3F4FF4CFE091B900E87FE03509F0DC
:107432008FC04091BB005527E4E8E093BC00FA01FD
:107442000E94D6CCAF0120E030E0E091BC00E078B1
:1074520021F42436E0E03E0708F003C02F5F3F4FDF
:10746200F4CFE091B900E87FE83509F071C0E0910E
:10747200BB00F0E00E94DFCC4E2B5F2BE4E9E093EF
:10748200BC0053FD506F20E030E0E091BC00E0789A
:1074920021F42436E0E03E0708F003C02F5F3F4F9F
:1074A200F4CF4093EC085093ED08A091EC08B09112
:1074B200ED08E0E1F0E00E946ACDE0938F0DA6E3D3
:1074C200B1E00E9453CE0E2FE2EEE017E4F4E09119
:1074D2009C0DE03089F0A0918F0DE02FF0E0E7FDE8
:1074E200FFEF3197B0E0A7FDBFEFAE17BF071CF467
:1074F200E0E0E0939C0D07C0A0918F0DA0171CF057
:10750200E1E0E0939C0DA7E3B1E00E9453CE0E2F81
:10751200E2EEE017E4F4E0919D0DE03089F0A091F5
:107522008F0DE02FF0E0E7FDFFEF3197B0E0A7FD10
:10753200BFEFAE17BF071CF4E0E0E0939D0D07C05C
:10754200A0918F0DA0171CF0E1E0E0939D0D09C002
:10755200E091EA08E07CE560E093EA08E4E9E09380
:10756200BC000E9463CC269608951A93F298F39871
:10757200F498F598E0917E00E97FE0937E00E3E9DC
:10758200F7E0FA93EA93E0E0EA93ACE0B0E00E941D
:107592005BC510E01C3008F04EC0E12FF0E0ED5664
:1075A200F84F0F01AAEBB1E0EE27A10FBE1F0E9418
:1075B20053CEE370D001E370EE0FEE0F0E2EEC917E
:1075C200E37FE029EC93E12FF0E0ED56F84F0F0155
:1075D200AAEBB1E0EE27A10FBE1F0E9453CEE695A3
:1075E200E695E170D001E170EE0F0E2EEC91ED7F89
:1075F200E029EC93E12FF0E0ED56F84FE081F0E066
:107602000E94ECCCE370F070309741F4123011F02C
:10761200133011F4F49A01C0F29A0BC0E130A0E0E9
:10762200FA0739F4123011F0133011F4F59A01C04F
:10763200F39A1F5FAFCFE0919507EC70E83031F01D
:10764200AEECB1E00E9453CEE37051F0E0917E00C7
:10765200E260E0937E00E1E0E0933F08F59AF4985F
:10766200E0919607EC70E83031F0AEECB1E00E94A8
:1076720053CEEC7051F0E0917E00E460E0937E0026
:10768200E1E0E0934008F59AF498F29B02C0F39B84
:1076920001C002C0169A01C01698F49B02C0F59B65
:1076A20001C002C0159A01C0159831C01A93E4EBCB
:1076B200F3E060E070E00E94E5CD80E00E94E3CB61
:1076C200249610E01C3000F5ECEBF3E060E070E093
:1076D2000E94E5CDE12FF0E031966F2F660F660B29
:1076E200762F0E94E5CDE12FF0E0ED56F84FE081D4
:1076F200E170FF27662777270E94E5CD88E00E9488
:10770200E3CB2C961F5FDECFAAE00E94F89119917D
:1077120008950E945ECC3A2FE091910DE17009F438
:1077220033C2373310F03C3308F006C0E32FF0E0E9
:10773200F797E957F64F3081313059F4A091990DFE
:10774200B0919A0DA037E7E1BE0710F0E1E01DC24B
:107752001BC2333010F03F3008F008C0E32FF0E0D6
:107762003397ED56F84FE081E1700FC23F3010F0D1
:107772003F3108F020C03F31E8F4E32FF0E03F97BB
:10778200A9E0B0E00E9411CDE950F74FE081E1702D
:1077920079F0E32FF0E03F97A9E0B0E00E9411CD2D
:1077A200E950F74FE081E077E03410F4E1E001C006
:1077B200E0E0EBC1E9C13C3310F0303708F014C00F
:1077C200ABE6B4E0E32FF0E0FC97BD01AEE0B0E041
:1077D2000E9411CDDB01AE0FBF1F1C96EC91EE1F74
:1077E200E0E0EE1FE170D1C1303710F0343808F01C
:1077F20011C0A6EDBCE0E32FF0E0E057F0400E949C
:10780200D8CCAE0FBF1FEC91E295EF70E695E695EE
:10781200E170BBC1343810F0383908F00EC0E32FE4
:10782200F0E0E458F040A3E0B0E00E9411CDED5B3F
:10783200F84FE081E695E170A8C1383910F03D3982
:1078420008F00EC0E32FF0E0E859F040AFE7B7E0F0
:107852000E94DACCAE0FBF1F1396EC91E17095C176
:107862003D39B9F4E091760DEF70E33079F0E091B3
:10787200760DEF70E43051F0E091760DEF70E1306B
:1078820029F0E091760DEF70E63011F4E1E07DC170
:107892007BC13E3969F4E091760DEF70E53029F055
:1078A200E091760DEF70E23011F4E1E06EC16CC14F
:1078B2003F3910F0373B08F06FC0E32FEF591E2F0E
:1078C200FF2766277727E25EFE4F6F4F6BBF069159
:1078D200E12FFF2766277727EA5CFE4F6F4F6BBFCA
:1078E2001691113449F5A3E00A9FF001E453F64FD3
:1078F200E081E07FE03111F4E1E047C1A3E00A9FBB
:10790200F001E453F64FE081E07FE03288F00A9F15
:10791200F001E453F64FE081E770E33041F00A9F53
:10792200F001E453F64FE081E770E43009F401C05E
:1079320002C0E1E02AC12FC0123401F5A3E00A9F80
:10794200F001E453F64FE081E07FE03211F4E1E030
:107952001CC1A3E00A9FF001E453F64FE081E07FEF
:10796200E03340F00A9FF001E453F64FE081E77004
:10797200E43009F002C0E1E008C10DC0133459F44B
:10798200A3E00A9FF001E453F64FE081E07FE03389
:1079920011F4E1E0FAC0F8C03A3B10F0363C08F0CE
:1079A20009C0E32FEA5B0E2FF0E0E156F84FE081C9
:1079B200E170EBC0373C10F03F3D08F0BEC0E091F3
:1079C200AB07F0E0E130A0E0FA0709F04CC03F3C21
:1079D20088F4E32FE75C1E2FA1E0B0E00E9486CC82
:1079E200A091B507B0E0EA23FB23309711F0E1E064
:1079F200CCC038C0333D88F4E32FEF5C1E2FA1E0EA
:107A0200B0E00E9486CCA091B607B0E0EA23FB2347
:107A1200309711F0E1E0B9C025C03B3D88F4E32F77
:107A2200E35D1E2FA1E0B0E00E9486CCA091CE07BC
:107A3200B0E0EA23FB23309711F0E1E0A6C012C0C8
:107A42003F3D80F4E32FEB5D1E2FA1E0B0E00E94EA
:107A520086CCA091CF07B0E0EA23FB23309711F048
:107A6200E1E093C069C0E230A0E0FA0721F0E33020
:107A7200A0E0FA0789F4A2EDB7E0E32FF0E0E75CBB
:107A8200F0400E94DACCAE0FBF1F1296EC91E1706B
:107A920011F0E1E07AC050C0E430A0E0FA0709F04A
:107AA2004BC03F3C88F4E32FE75C1E2FA1E0B0E01F
:107AB2000E9486CCA091B307B0E0EA23FB23309763
:107AC20011F0E1E062C038C0333D88F4E32FEF5C8F
:107AD2001E2FA1E0B0E00E9486CCA091B607B0E0D4
:107AE200EA23FB23309711F0E1E04FC025C03B3D74
:107AF20088F4E32FE35D1E2FA1E0B0E00E9486CC64
:107B0200A091DB07B0E0EA23FB23309711F0E1E01C
:107B12003CC012C03F3D80F4E32FEB5D1E2FA1E07D
:107B2200B0E00E9486CCA091DE07B0E0EA23FB23FE
:107B3200309711F0E1E029C027C03F3D39F4E091D0
:107B42009C0DE03011F0E1E020C01EC0303E39F45F
:107B5200E0919D0DE03011F0E1E017C015C0323028
:107B620059F4A5E3B1E00E9453CEA091900DAE1757
:107B720010F0E1E00AC008C0313E31F4E091640443
:107B8200E87011F0E1E001C0E0E00E9465CC2496CB
:107B9200089523970E945CCCF39904C0F59902C022
:107BA20022FE01C003C0689422F8A6C4F09B10C054
:107BB200E0919307E1704E2FE0919407E170E8871E
:107BC200E0919507E170EF83E0919607E170EE8313
:107BD20022FE4BC0E0919307EC7009F045C0E091A2
:107BE2009307E295EF701E2F669B02C0F19B01C0C6
:107BF2001FC0123010F41F5F1AC01230B9F4E091A6
:107C02009307E27071F0E0919307E17021F0E09147
:107C12009307EE7F03C0E0919307E160E09393073F
:107C220005C0E0919307E160E09393071FE011C064
:107C32001B3010F011500DC0113020F0E09193076D
:107C4200E27009F005C0E0919307EE7FE09393079D
:107C520010E0E12FEF70E295E07F0E2EE0919307A6
:107C6200EF70E029E093930748C0E0919307EC702E
:107C7200E43009F042C0E0919307E295EF701E2FC5
:107C8200669B12C01B3010F011500DC0113020F055
:107C9200E0919307E27009F005C0E0919307EE7F4F
:107CA200E093930710E01EC0123010F41F5F1AC059
:107CB2001230B9F4E0919307E27071F0E09193070A
:107CC200E17021F0E0919307EE7F03C0E09193070A
:107CD200E160E093930705C0E0919307E160E093D0
:107CE20093071FE0E12FEF70E295E07F0E2EE09107
:107CF2009307EF70E029E093930722FE4DC0E091D5
:107D02009407EC7009F047C0E0919407E295EF7098
:107D12001E2F679B02C0F19B01C021C0123010F4DC
:107D22001F5F1CC01230C9F4E0919407E27081F029
:107D3200E0919407E17031F0A4E9B7E0EC91EE7FB5
:107D4200EC9305C0E0919407E160E093940705C0CD
:107D5200E0919407E160E09394071FE011C01B30AB
:107D620010F011500DC0113020F0E0919407E27034
:107D720009F005C0A4E9B7E0EC91EE7FEC9310E0C6
:107D8200A4E9B7E0E12FEF70E295E07F0E2EEC91CF
:107D9200EF70E029EC934AC0E0919407EC70E43074
:107DA20009F044C0E0919407E295EF701E2F679BA3
:107DB20012C01B3010F011500DC0113020F0E091B4
:107DC2009407E27009F005C0A4E9B7E0EC91EE7FF8
:107DD200EC9310E020C0123010F41F5F1CC0123070
:107DE200C9F4E0919407E27081F0E0919407E170A8
:107DF20031F0A4E9B7E0EC91EE7FEC9305C0E0919D
:107E02009407E160E093940705C0E0919407E16074
:107E1200E09394071FE0A4E9B7E0E12FEF70E29549
:107E2200E07F0E2EEC91EF70E029EC93E091950744
:107E3200EC70E83009F03FC0E0917508F0917608E7
:107E420034960E94EACC5E2FE0919507E295EF709E
:107E52001E2FA8ECB1E00E9453CE3E2FA9ECB1E058
:107E62000E9453CE2E2F321728F5E0919507E1702C
:107E720089F0351768F01B3010F0115008C011302E
:107E820028F0A5E9B7E0EC91EE7FEC9310E001C099
:107E92001FE010C0521768F0123010F41F5F08C0C4
:107EA200123029F4E0919507E160E09395071FE015
:107EB20001C010E08BC022FE4AC0E0919507EC7031
:107EC20009F044C0E0919507E295EF701E2F799B6F
:107ED20012C01B3010F011500DC0113020F0E09193
:107EE2009507E27009F005C0A5E9B7E0EC91EE7FD5
:107EF200EC9310E020C0123010F41F5F1CC012304F
:107F0200C9F4E0919507E27081F0E0919507E17084
:107F120031F0A5E9B7E0EC91EE7FEC9305C0E0917A
:107F22009507E160E093950705C0E0919507E16050
:107F3200E09395071FE0A5E9B7E0E12FEF70E29526
:107F4200E07F0E2EEC91EF70E029EC934AC0E091B5
:107F52009507EC70E43009F044C0E0919507E29592
:107F6200EF701E2F799B21C0123010F41F5F1CC0CE
:107F72001230C9F4E0919507E27081F0E091950723
:107F8200E17031F0A5E9B7E0EC91EE7FEC9305C02A
:107F9200E0919507E160E093950705C0E0919507B0
:107FA200E160E09395071FE011C01B3010F0115003
:107FB2000DC0113020F0E0919507E27009F005C084
:107FC200A5E9B7E0EC91EE7FEC9310E0A5E9B7E00C
:107FD200E12FEF70E295E07F0E2EEC91EF70E02939
:107FE200EC93E0919607EC70E83009F03FC0E09125
:107FF2007708F091780834960E94EACC5E2FE091DF
:108002009607E295EF701E2FACECB1E00E9453CEC2
:108012003E2FADECB1E00E9453CE2E2F321728F541
:10802200E0919607E17089F0351768F01B3010F087
:10803200115008C0113028F0A6E9B7E0EC91EE7FAC
:10804200EC9310E001C01FE010C0521768F012302C
:1080520010F41F5F08C0123029F4E0919607E16026
:10806200E09396071FE001C010E085C022FE47C0E2
:10807200E0919607EC7009F041C0E0919607E29515
:10808200EF701E2F7A9B0FC01B3010F011500AC0E8
:10809200E0919607E27029F4A6E9B7E0EC91EE7F51
:1080A200EC9310E020C0123010F41F5F1CC012309D
:1080B200C9F4E0919607E27081F0E0919607E170D1
:1080C20031F0A6E9B7E0EC91EE7FEC9305C0E091C8
:1080D2009607E160E093960705C0E0919607E1609C
:1080E200E09396071FE0A6E9B7E0E12FEF70E29573
:1080F200E07F0E2EEC91EF70E029EC9347C0E09107
:108102009607EC70E43009F041C0E0919607E295E1
:10811200EF701E2F7A9B21C0123010F41F5F1CC01B
:108122001230C9F4E0919607E27081F0E09196076F
:10813200E17031F0A6E9B7E0EC91EE7FEC9305C077
:10814200E0919607E160E093960705C0E0919607FB
:10815200E160E09396071FE00EC01B3010F0115053
:108162000AC0E0919607E27029F4A6E9B7E0EC9123
:10817200EE7FEC9310E0A6E9B7E0E12FEF70E29515
:10818200E07F0E2EEC91EF70E029EC93F09B5FC044
:10819200E0919307E170E41791F0E3ECF3E060E023
:1081A20070E00E94E5CDE0919307E170FF2766271A
:1081B20077270E94E5CD84E00E94E3CB2896E091E8
:1081C2009407E170A885EA1791F0EDECF3E060E026
:1081D20070E00E94E5CDE0919407E170FF276627E9
:1081E20077270E94E5CD84E00E94E3CB2896E091B8
:1081F2009507E170AF81EA1791F0E7EDF3E060E0F7
:1082020070E00E94E5CDE0919507E170FF276627B7
:1082120077270E94E5CD84E00E94E3CB2896E09187
:108222009607E170AE81EA1791F0E1EEF3E060E0CB
:1082320070E00E94E5CDE0919607E170FF27662786
:1082420077270E94E5CD84E00E94E3CB289654E094
:108252005C3008F01DC1E52FF0E0ED56F84FE081EB
:10826200E1704E2F22FE77C0E52FF0E0ED56F84F79
:10827200E081EC7009F06EC0F19B02C000E011C019
:10828200A7E3B8E0E52FFF2766277727EC56FF4FD5
:108292006F4F6BBFE691F0E0AE0FBF1FEC91E07243
:1082A2000E2FE52FF0E0ED56F84FE081E295EF70EA
:1082B2001E2F003061F1123010F41F5F27C0123000
:1082C20021F5E52FF0E0ED56F84FE081E270B1F0D4
:1082D200E52FF0E0ED56F84FE081E17039F0A52F7F
:1082E200B0E0AD56B84FEC91EE7F06C0A52FB0E0DE
:1082F200AD56B84FEC91E160EC9307C0A52FB0E00A
:10830200AD56B84FEC91E160EC931FE016C01B3004
:1083120010F0115012C0113038F0E52FF0E0ED5698
:10832200F84FE081E27009F007C0A52FB0E0AD562A
:10833200B84FEC91EE7FEC9310E0A52FB0E0AD5674
:10834200B84FE12FEF70E295E07F0E2EEC91EF70C7
:10835200E029EC9373C0E52FF0E0ED56F84FE08191
:10836200EC70E43009F06AC0A7E3B8E0E52FFF271C
:1083720066277727EC56FF4F6F4F6BBFE691F0E011
:10838200AE0FBF1FEC91E0720E2FE52FF0E0ED561D
:10839200F84FE081E295EF701E2F0030B9F01B30EC
:1083A20010F0115012C0113038F0E52FF0E0ED5608
:1083B200F84FE081E27009F007C0A52FB0E0AD569A
:1083C200B84FEC91EE7FEC9310E02BC0123010F41A
:1083D2001F5F27C0123021F5E52FF0E0ED56F84F70
:1083E200E081E270B1F0E52FF0E0ED56F84FE08168
:1083F200E17039F0A52FB0E0AD56B84FEC91EE7FA9
:1084020006C0A52FB0E0AD56B84FEC91E160EC93F9
:1084120007C0A52FB0E0AD56B84FEC91E160EC93E8
:108422001FE0A52FB0E0AD56B84FE12FEF70E295F7
:10843200E07F0E2EEC91EF70E029EC93F09B26C0CA
:10844200E52FF0E0ED56F84FE081E170E417F1F02E
:10845200EBEEF3E060E070E00E94E5CDE52FF0E0A6
:1084620031966F2F660F660B762F0E94E5CDE52FB2
:10847200F0E0ED56F84FE081E170FF27662777279D
:108482000E94E5CD88E00E94E3CB2C965F5FE0CEB0
:10849200F39B06C0F29904C0F59B02C0F49B01C095
:1084A20002C0E89414C0F39906C0F29B04C0F59987
:1084B20002C0F49901C002C0689409C0A0E022FC85
:1084C200A1E0E1E0EA27E894EE2309F0689422F8BB
:1084D200F39B02C0F29901C005C022FE02C0169AA7
:1084E20001C01698F59B02C0F49901C005C022FE96
:1084F20002C0159A01C015980E9463CC299608956E
:1085020024970E945CCCAEECB1E00E9453CEE370A3
:108512003E2F303009F4B9C0AFECB1E00E9453CE27
:108522002E2FA0EDB1E00E9453CE5E2F313029F400
:10853200E0917508F091760804C0E0917708F09117
:10854200780834960E94ECCCE887F98710E0163060
:1085520008F09BC0A1EDB1E0EE27A10FBE1F0E9463
:1085620053CE0E2F013008F48EC0F0E0EE83FF836D
:10857200EE0FFF1FEE83FF83E12FF0E0E156F84F8D
:10858200E081E17009F443C0E22FF0E0A885B985EB
:10859200AE0FBF1FEE27A50FBE1FEE81FF81AE17E4
:1085A200BF0778F0E22FF0E0AE81BF81AE0FBF1FB0
:1085B200E52FF0E0EA0FFB1FA885B985EA17FB0754
:1085C20028F5F09B1CC0E6EFF3E060E070E00E944B
:1085D200E5CDE12FF0E031966F2F660F660B762F17
:1085E2000E94E5CDA889B989EAE00E9439CD6627C3
:1085F20077270E94E5CD88E00E94E3CB2C96A12F3D
:10860200B0E0A156B84FEC91EE7FEC933CC0E22F64
:10861200F0E0A885B985AE0FBF1FEE81FF81AE17CE
:10862200BF0758F0E22FF0E0AE81BF81EA0FFB1FD7
:10863200A885B985EA17FB0708F425C0F09B1CC082
:10864200EAE0F4E060E070E00E94E5CDE12FF0E0C6
:1086520031966F2F660F660B762F0E94E5CDA889A3
:10866200B989EAE00E9439CD662777270E94E5CDD5
:1086720088E00E94E3CB2C96A12FB0E0A156B84F20
:10868200EC91E160EC931F5F62CFAEECB1E00E942F
:1086920053CEE695E695E3703E2F303009F4B9C02B
:1086A200AFECB1E00E9453CE2E2FA0EDB1E00E94BC
:1086B20053CE5E2F313029F4E0917508F09176089F
:1086C20004C0E0917708F091780834960E94ECCCCF
:1086D200E887F98716E01C3008F09BC0A1EDB1E0F5
:1086E200EE27A10FBE1F0E9453CE0E2F013008F4B9
:1086F2008EC0F0E0EE83FF83EE0FFF1FEE83FF8359
:10870200E12FF0E0E156F84FE081E17009F443C057
:10871200E22FF0E0A885B985AE0FBF1FEE27A50FA7
:10872200BE1FEE81FF81AE17BF0778F0E22FF0E0A7
:10873200AE81BF81AE0FBF1FE52FF0E0EA0FFB1F36
:10874200A885B985EA17FB0728F5F09B1CC0E6EF60
:10875200F3E060E070E00E94E5CDE12FF0E03196B9
:108762006F2F660F660B762F0E94E5CDA889B98917
:10877200EAE00E9439CD662777270E94E5CD88E09E
:108782000E94E3CB2C96A12FB0E0A156B84FEC91FA
:10879200EE7FEC933CC0E22FF0E0A885B985AE0FE6
:1087A200BF1FEE81FF81AE17BF0758F0E22FF0E046
:1087B200AE81BF81EA0FFB1FA885B985EA17FB07C7
:1087C20008F425C0F09B1CC0EAE0F4E060E070E031
:1087D2000E94E5CDE12FF0E031966F2F660F660B18
:1087E200762F0E94E5CDA889B989EAE00E9439CDA9
:1087F200662777270E94E5CD88E00E94E3CB2C967E
:10880200A12FB0E0A156B84FEC91E160EC931F5F4D
:1088120062CF0E9463CC2A96089560971A93FE0154
:108822003196FA93EA93E0E0EA93A0E1B0E00E9485
:108832005BC510E01C3008F03FC0AAEBB1E0EE27A8
:10884200A10FBE1F0E9453CEEC7F0E946FCEAAEBF7
:10885200B1E0EE27A10FBE1F0E9453CEEB7F0E9414
:108862006FCEFE013196FA93EA93EDE1F4E060E017
:1088720070E00E94E5CDE12FF0E031966F2F660F98
:10888200660B762F0E94E5CD84E00E94A8CB2A9643
:10889200E12FF0E0A0E6B9E30E94D6CCEA0FFB1F7D
:1088A200FA93EA93FE013396FA93EA93A0E10E94C7
:1088B200C428A8951F5FBECFA6ECB1E0E0E00E94FD
:1088C2006FCEA7ECB1E0EAEF0E946FCEA8ECB1E068
:1088D200E4E60E946FCEA9ECB1E0E6E90E946FCE19
:1088E200AAECB1E0E0E00E946FCEABECB1E0EAEFBF
:1088F2000E946FCEACECB1E0E4E60E946FCEADEC2C
:10890200B1E0E6E90E946FCEAEECB1E00E9453CE38
:10891200EC7F0E946FCEAEECB1E00E9453CEE37FBB
:108922000E946FCEAEECB1E00E9453CEEF700E9477
:108932006FCEAFECB1E0E8E10E946FCEA0EDB1E006
:10894200E2E00E946FCEE1EDF1E0FA93EA93ACE04F
:108952000E942E2610E0163008F054C0FE01319617
:10896200FA93EA93E7E2F4E060E070E00E94E5CD7A
:10897200E12FF0E031966F2F660F660B762F0E9483
:10898200E5CD84E00E94A8CB2A96E12FF0E0A0ED8D
:10899200B3E40E94D6CCEA0FFB1FFA93EA93FE01DE
:1089A2003396FA93EA93A0E10E94C428FE0131961D
:1089B200FA93EA93E3E3F4E060E070E00E94E5CD2D
:1089C200E12FF0E031966F2F660F660B762F0E9433
:1089D200E5CD84E00E94A8CB2A96E12FF0E03696FE
:1089E200A0EDB3E40E94D6CCEA0FFB1FFA93EA9300
:1089F200FE013396FA93EA93A0E10E94C428A89557
:108A02001F5FA9CF1881619608950E945CCCEBEAA2
:108A1200F7E0FA93EA93E0E0EA93A7E8B0E00E9475
:108A22005BC5A8E3B1E00E9453CEE093AB07E0E45C
:108A3200F4E060E070E00E94E5CD80E00E94E3CBCC
:108A42002496E091AB07F0E0E130A0E0FA0709F0EC
:108A520028C100E0023008F007C1A9E2B8E0E02F27
:108A6200F0E0BD01A1E7B0E00E9411CDDB01AE0F45
:108A7200BF1F0E9453CEE03009F4F4C0ACEAB7E065
:108A8200E02FF0E0BD01A9E1B0E00E9411CDE60FB8
:108A9200F71FFF93EF93A9E2B8E0E02FF0E0BD01EA
:108AA200A1E7B0E00E9411CDDB01AE0FBF1F11960E
:108AB2000E9453CEE295EF70AF91BF91EF770E2EE9
:108AC200EC91E078E029EC93ACEAB7E0E02FF0E03B
:108AD200BD01A9E1B0E00E9411CDDB01AE0FBF1FC5
:108AE2001296E5E0EC9331E0E0E01E2F5E2F2E2F90
:108AF200183008F040C0A9E2B8E0E02FF0E0BD0174
:108B0200A1E7B0E00E9411CDDB01AE0FBF1F1E96A0
:108B1200E12FF0E00E94D8CCAE0FBF1F16960E9444
:108B220053CEF0E0F695E795E370F070E130A0E007
:108B3200FA0721F0E330A0E0FA0709F4232BA9E2B7
:108B4200B8E0E02FF0E0BD01A1E7B0E00E9411CD56
:108B5200DB01AE0FBF1F1E96E12FF0E00E94D8CCC2
:108B6200AE0FBF1F16960E9453CEE17009F0532B31
:108B72001F5F330FBDCFACEAB7E0E02FF0E0BD01DD
:108B8200A9E1B0E00E9411CDE60FF71F2187ACEA00
:108B9200B7E0E02FF0E0BD01A9E1B0E00E9411CD05
:108BA200E60FF71F558331E0E0E05E2F2E2F1C30D9
:108BB20008F040C0A9E2B8E0E02FF0E0BD01A1E773
:108BC200B0E00E9411CDDB01AE0FBF1F1E96E12F58
:108BD200F0E00E94D8CCAE0FBF1F16960E9453CE73
:108BE200F0E0F695E795E370F070E130A0E0FA0767
:108BF20021F0E330A0E0FA0709F4232BA9E2B8E060
:108C0200E02FF0E0BD01A1E7B0E00E9411CDDB0151
:108C1200AE0FBF1F1E96E12FF0E00E94D8CCAE0F20
:108C2200BF1F16960E9453CEE17009F0532B1F5FAF
:108C3200330FBDCFACEAB7E0E02FF0E0BD01A9E110
:108C4200B0E00E9411CDE60FF71F2287ACEAB7E031
:108C5200E02FF0E0BD01A9E1B0E00E9411CDE60FE6
:108C6200F71F56830F5FF6CEE8E4F4E060E070E0B1
:108C72000E94E5CDA9E2B8E00E9453CEFF27662705
:108C820077270E94E5CDAAE9B8E00E9453CEFF27DC
:108C9200662777270E94E5CD88E00E94E3CB2C96D9
:108CA2003DC0E230A0E0FA0769F4E9E5F4E060E0F3
:108CB20070E00E94E5CD80E00E94E3CB24960E9402
:108CC200F1522CC0E330A0E0FA0769F4EBE6F4E0DD
:108CD20060E070E00E94E5CD80E00E94E3CB249644
:108CE2000E94F1521BC0E430A0E0FA0769F4EBE7FE
:108CF200F4E060E070E00E94E5CD80E00E94E3CB0A
:108D020024960E94515B0AC0E3E8F4E060E070E060
:108D12000E94E5CD80E00E94E3CB24960E9463CCC2
:108D220026960895E0E0E093AB07A8E3B1E00E9445
:108D32006FCE0895BA93AA9323970E945CCCA9851B
:108D4200BA85EC91E07109F0A7C1E985FA85A181A4
:108D5200EFE7EA233E2F303009F49EC100E00230F3
:108D620008F09AC1A9E2B8E0E02FF0E0BD01A1E766
:108D7200B0E00E9411CDDB01AE0FBF1F0E9453CEA7
:108D82003E1709F087C1ACEAB7E0E02FF0E0BD0181
:108D9200A9E1B0E00E9411CDDB01AE0FBF1F129618
:108DA200EAE0EC93E985FA85A181B281E7E00E94CD
:108DB20097CCEE83F0E0EE30A0E0FA0709F46AC146
:108DC200E330A0E0FA0709F065C1ACEAB7E0E02FB2
:108DD200F0E0BD01A9E1B0E00E9411CDDB01AE0FD0
:108DE200BF1FEC91E07889F5ACEAB7E0E02FF0E044
:108DF200BD01A9E1B0E00E9411CDDB01AE0FBF1FA2
:108E0200EC91E068EC93ACEAB7E0E02FF0E0BD0152
:108E1200A9E1B0E00E9411CDDB01AE0FBF1F119698
:108E2200E0E0EC93EAE8F4E060E070E00E94E5CD77
:108E3200E02FF0E031966F2F660F660B762F0E94BF
:108E4200E5CD84E00E94E3CB2896ACEAB7E0E02FC0
:108E5200F0E0BD01A9E1B0E00E9411CDDB01AE0F4F
:108E6200BF1F1296E1E1EC93ACEAB7E0E02FF0E02D
:108E7200BD01A9E1B0E00E9411CDE60FF71F4185C7
:108E8200ACEAB7E0E02FF0E0BD01A9E1B0E00E945A
:108E920011CDDB01AE0FBF1F1796EC91E887ACEA4C
:108EA200B7E0E02FF0E0BD01A9E1B0E00E9411CDF2
:108EB200DB01AE0FBF1F1596EC91EF83E985FA85B2
:108EC200258110E051E0183008F5E52FAF81EA2343
:108ED20091F0E52FE22349F0E52FA885EA2321F45A
:108EE2004527E52FEA2BE88705C0E52FE095A88501
:108EF200EA23E88708C0E52FE22311F0452B03C0DF
:108F0200E52FE0954E231F5F550FDDCFACEAB7E0AA
:108F1200E02FF0E0BD01A9E1B0E00E9411CDDB013C
:108F2200AE0FBF1F1996AC914A17D9F0ACEAB7E061
:108F3200E02FF0E0BD01A9E1B0E00E9411CDE60F03
:108F4200F71F4187ACEAB7E0E02FF0E0BD01A9E1ED
:108F5200B0E00E9411CDDB01AE0FBF1F1396E0E01F
:108F6200EC93ACEAB7E0E02FF0E0BD01A9E1B0E09C
:108F72000E9411CDE60FF71F3796A885A083ACEAB1
:108F8200B7E0E02FF0E0BD01A9E1B0E00E9411CD11
:108F9200E60FF71F4285ACEAB7E0E02FF0E0BD0133
:108FA200A9E1B0E00E9411CDDB01AE0FBF1F189600
:108FB200EC91E887ACEAB7E0E02FF0E0BD01A9E16F
:108FC200B0E00E9411CDDB01AE0FBF1F1696EC91EF
:108FD200EF83E985FA85268110E051E0143008F527
:108FE200E52FAF81EA2391F0E52FE22349F0E52F47
:108FF200A885EA2321F44527E52FEA2BE88705C057
:10900200E52FE095A885EA23E88708C0E52FE2234B
:1090120011F0452B03C0E52FE0954E231F5F550F3E
:10902200DDCFACEAB7E0E02FF0E0BD01A9E1B0E0AE
:109032000E9411CDDB01AE0FBF1F1A96AC914A17E9
:10904200D9F0ACEAB7E0E02FF0E0BD01A9E1B0E071
:109052000E9411CDE60FF71F4287ACEAB7E0E02F7E
:10906200F0E0BD01A9E1B0E00E9411CDDB01AE0F3D
:10907200BF1F1396E0E0EC93ACEAB7E0E02FF0E01C
:10908200BD01A9E1B0E00E9411CDE60FF71F3896AD
:10909200A885A0830F5F63CE0E9463CC2B960895B0
:1090A2006F970E945CCCE0916304E07421F40E940B
:1090B20063CCA596089540E0423010F00C943951EB
:1090C200ACEAB7E0E42FF0E0BD01A9E1B0E00E9414
:1090D20011CDDB01AE0FBF1F1296AC91A13010F47F
:1090E2000C943651ACEAB7E0E42FF0E0BD01A9E1FF
:1090F200B0E00E9411CDDB01AE0FBF1FEC91EF7704
:109102005E2FACEAB7E0E42FF0E0BD01A9E1B0E0E8
:109112000E9411CDDB01AE0FBF1F1396AC91A1309F
:1091220080F0ACEAB7E0E42FF0E0BD01A9E1B0E0E5
:109132000E9411CDDB01AE0FBF1F1396EC91E150DF
:1091420089C6ACEAB7E0E42FF0E0BD01A9E1B0E0E6
:109152000E9411CDDB01AE0FBF1F1396E4E0EC932A
:10916200FE013C96FA93EA93E0E0EA93A6E0B0E0CF
:109172000E945BC5FE013696FA93EA93E0E0EA9319
:10918200A6E0B0E00E945BC520E0E1E0EE8BE0E10A
:10919200ED8B251708F0E5C500E030E0A9E2B8E064
:1091A200E42FF0E0BD01A1E7B0E00E9411CDDB01A8
:1091B200AE0FBF1F1E96E22FF0E00E94D8CCAE0F7A
:1091C200BF1F15960E9453CE1E2FA12F0E949E7A7A
:1091D2003E2F3030E9F4A9E2B8E0E42FF0E0BD011F
:1091E200A1E7B0E00E9411CDDB01AE0FBF1F1E96BA
:1091F200E22FF0E00E94D8CCAE0FBF1F14960E945F
:1092020053CE1E2F103021F0A12F0E949E7A3E2FA6
:109212003030E9F4A9E2B8E0E42FF0E0BD01A1E7C3
:10922200B0E00E9411CDDB01AE0FBF1F1E96E22FF0
:10923200F0E00E94D8CCAE0FBF1F13960E9453CE0F
:109242001E2F103021F0A12F0E949E7A3E2F303027
:1092520009F4C4C0E32FF0E0E130A0E0FA0729F5F9
:10926200A9E2B8E0E42FF0E0BD01A1E7B0E00E947E
:1092720011CDDB01AE0FBF1F1C960E9453CEE295AB
:10928200E7700E2FA9E2B8E0E42FF0E0BD01A1E7FC
:10929200B0E00E9411CDDB01AE0FBF1F1C960E94F1
:1092A20053CEEE1FE0E0EE1F96C0E230A0E0FA07D8
:1092B200F9F4A9E2B8E0E42FF0E0BD01A1E7B0E0E3
:1092C2000E9411CDDB01AE0FBF1F1C960E9453CE30
:1092D200E7700E2FA9E2B8E0E42FF0E0BD01A1E7AC
:1092E200B0E00E9411CDDB01AE0FBF1F1C966EC015
:1092F200E330A0E0FA0729F5A9E2B8E0E42FF0E0B4
:10930200BD01A1E7B0E00E9411CDDB01AE0FBF1F8E
:109312001B960E9453CEE295E7700E2FA9E2B8E0A9
:10932200E42FF0E0BD01A1E7B0E00E9411CDDB0126
:10933200AE0FBF1F1B960E9453CEEE1FE0E0EE1F42
:109342004AC0E430A0E0FA07F9F4A9E2B8E0E42F59
:10935200F0E0BD01A1E7B0E00E9411CDDB01AE0F4C
:10936200BF1F1B960E9453CEE7700E2FA9E2B8E0F2
:10937200E42FF0E0BD01A1E7B0E00E9411CDDB01D6
:10938200AE0FBF1F1B9622C0E530A0E0FA0729F5F9
:10939200A9E2B8E0E42FF0E0BD01A1E7B0E00E944D
:1093A20011CDDB01AE0FBF1F1D960E9453CEE77099
:1093B2000E2FA9E2B8E0E42FF0E0BD01A1E7B0E092
:1093C2000E9411CDDB01AE0FBF1F1D960E9453CE2E
:1093D200E695E695E695E170EF8BF0C0A9E2B8E07C
:1093E200E42FF0E0BD01A1E7B0E00E9411CDDB0166
:1093F200AE0FBF1F1E96E22FF0E00E94D8CCAE0F38
:10940200BF1F12960E9453CE1E2F103029F0A12F9B
:109412000E948A3BE03009F42EC0A9E2B8E0E42FB2
:10942200F0E0BD01A1E7B0E00E9411CDDB01AE0F7B
:10943200BF1F1E96E22FF0E00E94D8CCAE0FBF1FD6
:1094420017960E9453CEE295E7700E2FA9E2B8E07C
:10945200E42FF0E0BD01A1E7B0E00E9411CDDB01F5
:10946200AE0FBF1F1E96E22FF0E00E94D8CCAE0FC7
:10947200BF1F17969CC0A9E2B8E0E42FF0E0BD013F
:10948200A1E7B0E00E9411CDDB01AE0FBF1F1E9617
:10949200E22FF0E00E94D8CCAE0FBF1F11960E94BF
:1094A20053CE1E2F103029F0A12F0E948A3BE030AC
:1094B20009F432C0A9E2B8E0E42FF0E0BD01A1E76F
:1094C200B0E00E9411CDDB01AE0FBF1F1E96E22F4E
:1094D200F0E00E94D8CCAE0FBF1F17960E9453CE69
:1094E200E7700E2FA9E2B8E0E42FF0E0BD01A1E79A
:1094F200B0E00E9411CDDB01AE0FBF1F1E96E22F1E
:10950200F0E00E94D8CCAE0FBF1F17960E9453CE38
:10951200E695E695E69550C0A9E2B8E0E42FF0E0C2
:10952200BD01A1E7B0E00E9411CDDB01AE0FBF1F6C
:109532001E96E22FF0E00E94D8CCAE0FBF1F0E9411
:1095420053CE1E2F103029F0A12F0E948A3BE0300B
:1095520009F434C0A9E2B8E0E42FF0E0BD01A1E7CC
:10956200B0E00E9411CDDB01AE0FBF1F1E96E22FAD
:10957200F0E00E94D8CCAE0FBF1F16960E9453CEC9
:10958200E295E7700E2FA9E2B8E0E42FF0E0BD010A
:10959200A1E7B0E00E9411CDDB01AE0FBF1F1E9606
:1095A200E22FF0E00E94D8CCAE0FBF1F16960E94A9
:1095B20053CEEE1FE0E0EE1FE170EF8BEF89E0305B
:1095C20009F4DFC1593008F047C0E02FF0E0E13084
:1095D200A0E0FA0729F4EE89AE81EA2BEE833BC0C4
:1095E200E230A0E0FA0719F4FE0137962EC0E3300C
:1095F200A0E0FA0741F1E430A0E0FA0739F4EE897D
:10960200AE81EA2BEE83FE0137961FC0E530A0E063
:10961200FA0789F0E630A0E0FA0729F4EE89AE8174
:10962200EA2BEE8310C0E730A0E0FA07A1F4EE893E
:10963200AE81EA2BEE83FE0137960F01E081AE89FF
:10964200EA2BD001EC93FE0138960F01E081AE893E
:10965200EA2BD001EC9394C15A3009F0C9C0E02F33
:10966200F0E0E130A0E0FA0781F4283028F4EE8936
:10967200AE81EA2BEE8308C0FE0137960F01E0812E
:10968200AE89EA2BD001EC93B2C0E230A0E0FA0737
:1096920071F4283018F4FE01389602C0FE013996A2
:1096A2000F01E081AE89EA2BD001EC93A0C0E33038
:1096B200A0E0FA0771F4283018F4FE013A9602C0CD
:1096C200FE013B960F01E081AE89EA2BD001EC93BB
:1096D2008EC0E430A0E0FA07E9F4283028F4EE89DD
:1096E200AE81EA2BEE8308C0FE0137960F01E081BE
:1096F200AE89EA2BD001EC93283018F4FE0138969B
:1097020002C0FE0139960F01E081AE89EA2BD00139
:10971200EC936DC0E530A0E0FA07D9F4283018F4D4
:10972200FE01389602C0FE0139960F01E081AE8932
:10973200EA2BD001EC93283018F4FE013A9602C0CD
:10974200FE013B960F01E081AE89EA2BD001EC933A
:109752004EC0E630A0E0FA07E9F4283028F4EE899A
:10976200AE81EA2BEE8308C0FE0137960F01E0813D
:10977200AE89EA2BD001EC93283018F4FE013A9618
:1097820002C0FE013B960F01E081AE89EA2BD001B7
:10979200EC932DC0E730A0E0FA0749F5283018F421
:1097A200FE01389602C0FE0139960F01E081AE89B2
:1097B200EA2BD001EC93283028F4EE89AE81EA2B13
:1097C200EE8308C0FE0137960F01E081AE89EA2BD5
:1097D200D001EC93283018F4FE013A9602C0FE0143
:1097E2003B960F01E081AE89EA2BD001EC93C8C011
:1097F200E02FF0E0E130A0E0FA0781F4283028F40D
:10980200EE89AE81EA2BEE8308C0FE0137960F0186
:10981200E081AE89EA2BD001EC93B2C0E230A0E045
:10982200FA0771F4243018F4FE01379602C0FE01E3
:1098320038960F01E081AD89EA2BD001EC93A0C0EC
:10984200E330A0E0FA0771F4283018F4FE013996EB
:1098520002C0FE013A960F01E081AE89EA2BD001E7
:10986200EC938EC0E430A0E0FA07E9F4283028F443
:10987200EE89AE81EA2BEE8308C0FE0137960F0116
:10988200E081AE89EA2BD001EC93243018F4FE017A
:10989200379602C0FE0138960F01E081AD89EA2BAE
:1098A200D001EC936DC0E530A0E0FA07D9F4243082
:1098B20018F4FE01379602C0FE0138960F01E081CE
:1098C200AD89EA2BD001EC93283018F4FE013996C9
:1098D20002C0FE013A960F01E081AE89EA2BD00167
:1098E200EC934EC0E630A0E0FA07E9F4283028F401
:1098F200EE89AE81EA2BEE8308C0FE0137960F0196
:10990200E081AE89EA2BD001EC93283018F4FE01F5
:10991200399602C0FE013A960F01E081AE89EA2B28
:10992200D001EC932DC0E730A0E0FA0749F52830CA
:1099320028F4EE89AE81EA2BEE8308C0FE01379649
:109942000F01E081AE89EA2BD001EC93243018F4A8
:10995200FE01379602C0FE0138960F01E081AD8903
:10996200EA2BD001EC93283018F4FE01399602C09C
:10997200FE013A960F01E081AE89EA2BD001EC9309
:10998200DEC1593008F047C0E02FF0E0E130A0E03E
:10999200FA0729F4EE89AC85EA2BEC873BC0E2306A
:1099A200A0E0FA0719F4FE013D962EC0E330A0E0D4
:1099B200FA0741F1E430A0E0FA0739F4EE89AC8508
:1099C200EA2BEC87FE013D961FC0E530A0E0FA07C6
:1099D20089F0E630A0E0FA0729F4EE89AC85EA2B9B
:1099E200EC8710C0E730A0E0FA07A1F4EE89AC855D
:1099F200EA2BEC87FE013D960F01E081AE89EA2B4E
:109A0200D001EC93FE013E960F01E081AE89EA2B74
:109A1200D001EC9394C15A3009F0C9C0E02FF0E0B4
:109A2200E130A0E0FA0781F4283028F4EE89AC8511
:109A3200EA2BEC8708C0FE013D960F01E081AE895A
:109A4200EA2BD001EC93B2C0E230A0E0FA0771F445
:109A5200283018F4FE013E9602C0FE013F960F0127
:109A6200E081AE89EA2BD001EC93A0C0E330A0E004
:109A7200FA0771F4283018F4FE01709602C0FE0154
:109A820071960F01E081AE89EA2BD001EC938EC072
:109A9200E430A0E0FA07E9F4283028F4EE89AC8536
:109AA200EA2BEC8708C0FE013D960F01E081AE89EA
:109AB200EA2BD001EC93283018F4FE013E9602C046
:109AC200FE013F960F01E081AE89EA2BD001EC93B3
:109AD2006DC0E530A0E0FA07D9F4283018F4FE0191
:109AE2003E9602C0FE013F960F01E081AE89EA2B4D
:109AF200D001EC93283018F4FE01709602C0FE01EA
:109B020071960F01E081AE89EA2BD001EC934EC031
:109B1200E630A0E0FA07E9F4283028F4EE89AC85B3
:109B2200EA2BEC8708C0FE013D960F01E081AE8969
:109B3200EA2BD001EC93283018F4FE01709602C093
:109B4200FE0171960F01E081AE89EA2BD001EC9300
:109B52002DC0E730A0E0FA0749F5283018F4FE01DD
:109B62003E9602C0FE013F960F01E081AE89EA2BCC
:109B7200D001EC93283028F4EE89AC85EA2BEC87EF
:109B820008C0FE013D960F01E081AE89EA2BD001AB
:109B9200EC93283018F4FE01709602C0FE01719613
:109BA2000F01E081AE89EA2BD001EC93C8C0E02F0F
:109BB200F0E0E130A0E0FA0781F4283028F4EE89E1
:109BC200AC85EA2BEC8708C0FE013D960F01E081CF
:109BD200AE89EA2BD001EC93B2C0E230A0E0FA07E2
:109BE20071F4243018F4FE013D9602C0FE013E9647
:109BF2000F01E081AD89EA2BD001EC93A0C0E330E4
:109C0200A0E0FA0771F4283018F4FE013F9602C072
:109C1200FE0170960F01E081AE89EA2BD001EC9330
:109C22008EC0E430A0E0FA07E9F4283028F4EE8987
:109C3200AC85EA2BEC8708C0FE013D960F01E0815E
:109C4200AE89EA2BD001EC93243018F4FE013D9644
:109C520002C0FE013E960F01E081AD89EA2BD001E0
:109C6200EC936DC0E530A0E0FA07D9F4243018F483
:109C7200FE013D9602C0FE013E960F01E081AD89D4
:109C8200EA2BD001EC93283018F4FE013F9602C073
:109C9200FE0170960F01E081AE89EA2BD001EC93B0
:109CA2004EC0E630A0E0FA07E9F4283028F4EE8945
:109CB200AC85EA2BEC8708C0FE013D960F01E081DE
:109CC200AE89EA2BD001EC93283018F4FE013F96BE
:109CD20002C0FE0170960F01E081AE89EA2BD0012D
:109CE200EC932DC0E730A0E0FA0749F5283028F4BC
:109CF200EE89AC85EA2BEC8708C0FE013D960F0188
:109D0200E081AE89EA2BD001EC93243018F4FE01F5
:109D12003D9602C0FE013E960F01E081AD89EA2B1D
:109D2200D001EC93283018F4FE013F9602C0FE01E8
:109D320070960F01E081AE89EA2BD001EC93EE8997
:109D4200EE0FEE8BED89EE0FED8BEE89E03011F424
:109D5200E1E0EE8BED89E03011F4E1E0ED8B2F5F75
:109D620018CAACEAB7E0E42FF0E0BD01A9E1B0E027
:109D72000E9411CDE60FF71F3B96FA93EA93FE017C
:109D82003E96FA93EA93A6E0B0E00E9430C5E03036
:109D920029F1ACEAB7E0E42FF0E0BD01A9E1B0E0BF
:109DA2000E9411CDE60FF71F3B96FA93EA93FE014C
:109DB2003E96FA93EA93A6E0B0E00E9449C5ACEA67
:109DC200B7E0E42FF0E0BD01A9E1B0E00E9411CDBF
:109DD200DB01AE0FBF1F5796E0E0EC93ACEAB7E0B1
:109DE200E42FF0E0BD01A9E1B0E00E9411CDE60F41
:109DF200F71F7196FA93EA93FE013896FA93EA9363
:109E0200A6E0B0E00E9430C5E03029F1ACEAB7E04C
:109E1200E42FF0E0BD01A9E1B0E00E9411CDE60F10
:109E2200F71F7196FA93EA93FE013896FA93EA9332
:109E3200A6E0B0E00E9449C5ACEAB7E0E42FF0E04A
:109E4200BD01A9E1B0E00E9411CDDB01AE0FBF1F41
:109E52005896E0E0EC93ACEAB7E0E42FF0E0BD0105
:109E6200A9E1B0E00E9411CDDB01AE0FBF1F149635
:109E7200AC91A13088F0ACEAB7E0E42FF0E0BD018C
:109E8200A9E1B0E00E9411CDDB01AE0FBF1F149615
:109E9200EC91E150EC9324C1ACEAB7E0E42FF0E09E
:109EA200BD01A9E1B0E00E9411CDDB01AE0FBF1FE1
:109EB2005796AC91A13080F0ACEAB7E0E42FF0E025
:109EC200BD01A9E1B0E00E9411CDDB01AE0FBF1FC1
:109ED2005896AC91A13008F403C1ACEAB7E0E42F84
:109EE200F0E0BD01A9E1B0E00E9411CDDB01AE0FAF
:109EF200BF1F1496E4E6EC93A9E2B8E0E42FF0E089
:109F0200BD01A1E7B0E00E9411CDDB01AE0FBF1F82
:109F120017960E9453CEAE2F0E948A3BE03081F109
:109F2200A9E2B8E0E42FF0E0BD01A1E7B0E00E94B1
:109F320011CDDB01AE0FBF1F18960E9453CEEC8BE2
:109F4200A9E2B8E0E42FF0E0BD01A1E7B0E00E9491
:109F520011CDDB01AE0FBF1F1A960E9453CEE295C0
:109F6200EF70EB8BA9E2B8E0E42FF0E0BD01A1E7CE
:109F7200B0E00E9411CDDB01AE0FBF1F199671C078
:109F8200A9E2B8E0E42FF0E0BD01A1E7B0E00E9451
:109F920011CDDB01AE0FBF1F14960E9453CEAE2F20
:109FA2000E948A3BE03079F1A9E2B8E0E42FF0E0C8
:109FB200BD01A1E7B0E00E9411CDDB01AE0FBF1FD2
:109FC20015960E9453CEEC8BA9E2B8E0E42FF0E0A4
:109FD200BD01A1E7B0E00E9411CDDB01AE0FBF1FB2
:109FE2001A960E9453CEEF70EB8BA9E2B8E0E42FF1
:109FF200F0E0BD01A1E7B0E00E9411CDDB01AE0FA0
:10A00200BF1F16962EC0A9E2B8E0E42FF0E0BD0112
:10A01200A1E7B0E00E9411CDDB01AE0FBF1F129687
:10A022000E9453CEEC8BA9E2B8E0E42FF0E0BD0130
:10A03200A1E7B0E00E9411CDDB01AE0FBF1F119668
:10A042000E9453CEEF70EB8BA9E2B8E0E42FF0E070
:10A05200BD01A1E7B0E00E9411CDDB01AE0FBF1F31
:10A0620013960E9453CEEA8BE88DE07FE160E88F81
:10A07200EF7EE88FA9E2B8E0E42FF0E0BD01A1E7AE
:10A08200B0E00E9411CDDB01AE0FBF1F0E9453CE84
:10A09200F0E0F460E98FFA8FEA89ED8FDE015896DD
:10A0A2000E943C09E88DE07FE260E88FA9E2B8E017
:10A0B200E42FF0E0BD01A1E7B0E00E9411CDDB0189
:10A0C200AE0FBF1F0E9453CEF0E0F560E98FFA8F0A
:10A0D200EC89ED8FEB89EE8FDE0158960E943C09E8
:10A0E200593010F0E6E001C0E3E0EF700E2EE88D8B
:10A0F200E07FE029E88FEF7EE88FACEAB7E0E42F5B
:10A10200F0E0BD01A9E1B0E00E9411CDDB01AE0F8C
:10A11200BF1F5796AC91A13088F0ACEAB7E0E42FAC
:10A12200F0E0BD01A9E1B0E00E9411CDDB01AE0F6C
:10A13200BF1F5796EC91E150EC933BC0ACEAB7E0FD
:10A14200E42FF0E0BD01A9E1B0E00E9411CDDB01F6
:10A15200AE0FBF1F5796EAEFEC93A9E2B8E0E42FE7
:10A16200F0E0BD01A1E7B0E00E9411CDDB01AE0F2E
:10A17200BF1F0E9453CEF0E0F260E98FFA8FFE011A
:10A182007D96FA93EA93ACEAB7E0E42FF0E0BD01E2
:10A19200A9E1B0E00E9411CDE60FF71F3B96FA93BA
:10A1A200EA93A6E0B0E00E9449C5DE0158960E94FB
:10A1B2003C09ACEAB7E0E42FF0E0BD01A9E1B0E070
:10A1C2000E9411CDDB01AE0FBF1F5896AC91A1309A
:10A1D20088F0ACEAB7E0E42FF0E0BD01A9E1B0E01D
:10A1E2000E9411CDDB01AE0FBF1F5896EC91E150DA
:10A1F200EC933BC0ACEAB7E0E42FF0E0BD01A9E18B
:10A20200B0E00E9411CDDB01AE0FBF1F5896EAEFFE
:10A21200EC93A9E2B8E0E42FF0E0BD01A1E7B0E0E1
:10A222000E9411CDDB01AE0FBF1F0E9453CEF0E0A2
:10A23200F360E98FFA8FFE017D96FA93EA93ACEA16
:10A24200B7E0E42FF0E0BD01A9E1B0E00E9411CD3A
:10A25200E60FF71F7196FA93EA93A6E0B0E00E9428
:10A2620049C5DE0158960E943C094F5F0C945D4837
:10A272000E9463CCA59608952D970E945ECCE09132
:10A282006304E07409F4A8C100E0023008F0A4C13C
:10A29200A9E2B8E0E02FF0E0BD01A1E7B0E00E9442
:10A2A20011CDDB01AE0FBF1F0E9453CEE03081F40F
:10A2B200ACEAB7E0E02FF0E0BD01A9E1B0E00E9416
:10A2C20011CDDB01AE0FBF1F1296E0E0EC9382C10D
:10A2D200ACEAB7E0E02FF0E0BD01A9E1B0E00E94F6
:10A2E20011CDDB01AE0FBF1F1296AC91A13008F465
:10A2F2006CC0ACEAB7E0E02FF0E0BD01A9E1B0E04C
:10A302000E9411CDDB01AE0FBF1F1296EC91E150FE
:10A31200EC93ACEAB7E0E02FF0E0BD01A9E1B0E0D8
:10A322000E9411CDDB01AE0FBF1F1196AC91A1307F
:10A3320088F0ACEAB7E0E02FF0E0BD01A9E1B0E0BF
:10A342000E9411CDDB01AE0FBF1F1196EC91E150BF
:10A35200EC933AC0ACEAB7E0E02FF0E0BD01A9E12E
:10A36200B0E00E9411CDDB01AE0FBF1F1196E2E3F8
:10A37200EC93EC81E07FE860EC83EF7EEC83A9E272
:10A38200B8E0E02FF0E0BD01A1E7B0E00E9411CDFE
:10A39200DB01AE0FBF1F0E9453CEF0E0F660ED83EB
:10A3A200FE83EBE2E987E0E0EA87E8E1EB87E5E0BC
:10A3B200EC87E4EFED87E1E0EE87E0E0EF87E88B02
:10A3C200DE0114960E943C0905C1ACEAB7E0E02F19
:10A3D200F0E0BD01A9E1B0E00E9411CDDB01AE0FBA
:10A3E200BF1FEC91E07809F4C8C0ACEAB7E0E02FF7
:10A3F200F0E0BD01A9E1B0E00E9411CDDB01AE0F9A
:10A40200BF1FEC91EF773E2FACEAB7E0E02FF0E010
:10A41200BD01A9E1B0E00E9411CDDB01AE0FBF1F6B
:10A42200EC91EF77EC93EAE9F4E060E070E00E94EF
:10A43200E5CDE02FF0E031966F2F660F660B762F99
:10A442000E94E5CD84E00E94E3CB289621E010E053
:10A45200131708F047C0A9E2B8E0E02FF0E0BD0111
:10A46200A1E7B0E00E9411CDDB01AE0FBF1F1E9627
:10A47200E12FF0E00E94D8CCAE0FBF1F16960E94CB
:10A4820053CEF0E0F695E795E370F070309799F4CB
:10A49200ACEAB7E0E02FF0E0BD01A9E1B0E00E9434
:10A4A20011CDE60FF71F39960F01A081E22FE0953B
:10A4B200EA23D00113C0E130A0E0FA0781F4ACEA4C
:10A4C200B7E0E02FF0E0BD01A9E1B0E00E9411CDBC
:10A4D200DB01AE0FBF1F1996EC91E22BEC931F5FCD
:10A4E200220FB6CF21E0131708F047C0A9E2B8E067
:10A4F200E02FF0E0BD01A1E7B0E00E9411CDDB0149
:10A50200AE0FBF1F1E96E12FF0E00E94D8CCAE0F17
:10A51200BF1F16960E9453CEF0E0F695E795E370C2
:10A52200F070309799F4ACEAB7E0E02FF0E0BD01AB
:10A53200A9E1B0E00E9411CDE60FF71F3A960F0194
:10A54200A081E22FE095EA23D00113C0E130A0E020
:10A55200FA0781F4ACEAB7E0E02FF0E0BD01A9E12F
:10A56200B0E00E9411CDDB01AE0FBF1F1A96EC9135
:10A57200E22BEC931F5F220FB6CFACEAB7E0E02FDD
:10A58200F0E0BD01A9E1B0E00E9411CDDB01AE0F08
:10A59200BF1F1296EAE0EC93EC81E07FE260EC836D
:10A5A200EF7EEC83E0E0ED83EE83E1E0E987A9E270
:10A5B200B8E0E02FF0E0BD01A1E7B0E00E9411CDCC
:10A5C200DB01AE0FBF1F0E9453CEEA87DE01149655
:10A5D2000E943C090F5F59CE0E9465CC6196089596
:10A5E2000E945ECC10E0133008F081C0AEEAB7E002
:10A5F200E12FF0E0BD01ACE0B0E00E9411CDE60F2A
:10A60200F71F3196FF93EF93A9E2B8E0E12FF0E054
:10A61200BD01AAE0B0E00E9411CDDB01AE0FBF1F69
:10A622000E9453CEAF91BF91EC93AEEAB7E0E12F17
:10A63200F0E0BD01ACE0B0E00E9411CDE60FF71FE3
:10A642003296FF93EF93A9E2B8E0E12FF0E0BD016B
:10A65200AAE0B0E00E9411CDDB01AE0FBF1F119640
:10A662000E9453CEAF91BF91EC93AEEAB7E0E12FD7
:10A67200F0E0BD01ACE0B0E00E9411CDE60FF71FA3
:10A682003596FF93EF93A9E2B8E0E12FF0E0BD0128
:10A69200AAE0B0E00E9411CDDB01AE0FBF1F1296FF
:10A6A2000E9453CEAF91BF91EC93AEEAB7E0E12F97
:10A6B200F0E0BD01ACE0B0E00E9411CDE60FF71F63
:10A6C2003696FF93EF93A9E2B8E0E12FF0E0BD01E7
:10A6D200AAE0B0E00E9411CDDB01AE0FBF1F1596BC
:10A6E2000E9453CEAF91BF91EC931F5F7CCFE0915C
:10A6F200B007E093BD07A091B007E091BC07EA0F55
:10A70200E093C907A091C907E091C807EA0FE09357
:10A71200AD0710E0183108F0E1C0E0E03E2F0E2F47
:10A72200A7E4B8E0E12FF0E0BD01ACE0B0E00E94A8
:10A7320011CDDB01AE0FBF1F11960E9453CEE03048
:10A7420009F031E0A7E4B8E0E12FF0E0BD01ACE0B0
:10A75200B0E00E9411CDDB01AE0FBF1F12960E9426
:10A7620053CEE03009F03260A7E4B8E0E12FF0E028
:10A77200BD01ACE0B0E00E9411CDDB01AE0FBF1F06
:10A7820015960E9453CEE03009F03460A7E4B8E099
:10A79200E12FF0E0BD01ACE0B0E00E9411CDDB01A1
:10A7A200AE0FBF1F16960E9453CEE03009F03860FC
:10A7B200A7E4B8E0E12FF0E0BD01ACE0B0E00E9418
:10A7C20011CDDB01AE0FBF1F19960E9453CEE030B0
:10A7D20009F03061A7E4B8E0E12FF0E0BD01ACE0A0
:10A7E200B0E00E9411CDDB01AE0FBF1F1A960E948E
:10A7F20053CEE03009F03062A7E4B8E0E12FF0E098
:10A80200BD01ACE0B0E00E9411CDDB01AE0FBF1F75
:10A8120013960E9453CEE03009F000E1A7E4B8E0BD
:10A82200E12FF0E0BD01ACE0B0E00E9411CDDB0110
:10A83200AE0FBF1F17960E9453CEE03009F00062A0
:10A84200A7E4B8E0E12FF0E0BD01ACE0B0E00E9487
:10A8520011CDDB01AE0FBF1F1B960E9453CEE0301D
:10A8620009F00064A2EDB7E0E12FF0E00E94DACC3B
:10A87200EA0FFB1F0283A2EDB7E0E12FF0E00E9496
:10A88200DACCEA0FFB1F3383A2EDB7E0E12FF0E051
:10A892000E94DACCEA0FFB1F3296FF93EF93A7E4F4
:10A8A200B8E0E12FF0E0BD01ACE0B0E00E9411CDD4
:10A8B200DB01AE0FBF1F0E9453CEE295EF70E6950B
:10A8C200E695E170AF91BF91E170EE0FEE0F0E2EA3
:10A8D200EC91EB7FE029EC931F5F1CCF0E9465CCCB
:10A8E20024960895BA93AA9325970E945CCCE0918E
:10A8F200AB07F0E0E230A0E0FA0739F4AB85BC85A3
:10A90200EC91E07109F02AC10AC0E330A0E0FA0735
:10A9120031F4AB85BC85EC91E07109F41FC1E09183
:10A92200AB07F0E0E230A0E0FA0729F0E330A0E064
:10A93200FA0709F013C110E0133008F00FC1AEEAB4
:10A94200B7E0E12FF0E0BD01ACE0B0E00E9411CD34
:10A95200E60FF71F2281213008F4FDC0AEEAB7E00E
:10A96200E12FF0E0BD01ACE0B0E00E9411CDE60FB6
:10A97200F71F3181A091AB07A23089F4E32FF0E0F9
:10A98200E058FE4F0F01AB85BC851196ED91FC910D
:10A992001197E015F10509F0DFC0E1E007C0EB8592
:10A9A200FC85E181E31709F0D7C0E3E0EA87AEEA6C
:10A9B200B7E0E12FF0E0BD01ACE0B0E00E9411CDC4
:10A9C200DB01AE0FBF1FEC91E03079F4AEEAB7E0E5
:10A9D200E12FF0E0BD01ACE0B0E00E9411CDDB015F
:10A9E200AE0FBF1F1496EFEFEC93AEEAB7E0E12F84
:10A9F200F0E0BD01ACE0B0E00E9411CDDB01AE0F92
:10AA0200BF1FECE0EC93AEEAB7E0E12FF0E0BD014E
:10AA1200ACE0B0E00E9411CDE60FF71F5381E0E0F9
:10AA22004E2FE8870E2F421708F094C0A091AB0773
:10AA3200A230A1F4003069F407E0AB85BC8515961D
:10AA4200E885EF5FE887E150F0E0AE0FBF1FEC91C1
:10AA520003C00150E985E695E98714C0003069F426
:10AA620003E0AB85BC851596E885EF5FE887E1508A
:10AA7200F0E0AE0FBF1FEC9104C00150E985E695EE
:10AA8200E695E987A2EDB7E0E52FF0E00E94DACC87
:10AA9200AE0FBF1F1296EC91E47009F43FC0A2ED15
:10AAA200B7E0E52FF0E00E94DACCAE0FBF1F12969E
:10AAB200EC91E170EF83A2EDB7E0E52FF0E00E94A8
:10AAC200DACCAE0FBF1F1296EC91E695E170EE83E1
:10AAD200EA85A985EA23E13069F4EE81E03049F4A0
:10AAE200E1E0EE83EF81E03011F0E0E001C0E1E06F
:10AAF200EF8302C0E0E0EE83A2EDB7E0E52FF0E0E5
:10AB02000E94DACCAE0FBF1F1296EE81E170EE0FFB
:10AB12000E2EEC91ED7FE029EC9309C0EA85A98520
:10AB2200EA23E13011F4E1E001C0E0E0EF83A2EDBD
:10AB3200B7E0E52FF0E00E94DACCAE0FBF1F12960D
:10AB4200EF81E1700E2EEC91EE7FE029EC934F5FE6
:10AB52005F5F69CF03C002C01F5FEECE0E9463CC6D
:10AB62002D9608952D970E945ECC1A2F09893A8955
:10AB7200EC81E061EC83E07FE860EC83F32FE0E0BE
:10AB820066277727E060F0606F6E7861DF01CB01A6
:10AB9200E0915C04FF2766277727EA2BFB2B682BC3
:10ABA200792BED83FE836F837887E02FEF5FE98750
:10ABB200A2EDB7E0E12FF0E00E94DACCAE0FBF1FAA
:10ABC200EC91EA87A2EDB7E0E12FF0E00E94DACC47
:10ABD200AE0FBF1F1196EC91EB87C9C02D970E9453
:10ABE2005CCC4A2FEE81EF7EEE83E07FE860EE835D
:10ABF200EC89F0E0E050FE4FEF83F887FE013B96D0
:10AC0200FA93EA93E0E0EA93A8E0B0E00E945BC521
:10AC120051E020E031E0E0E00E2F1E2F141708F083
:10AC22004BC030E0333008F042C0503051F4E02FD6
:10AC32000F5FF0E0DE011B96EA0FFB1F208351E05D
:10AC420020E0E32FF0E0309769F4A2EDB7E0EB8962
:10AC5200F0E00E94DACCAE0FBF1FEC91EF7009F06A
:10AC6200252B22C0E130A0E0FA0769F4A2EDB7E09B
:10AC7200EB89F0E00E94DACCAE0FBF1FEC91E07FCF
:10AC820009F0252B11C0E230A0E0FA0769F4A2ED29
:10AC9200B7E0EB89F0E00E94DACCAE0FBF1F11964D
:10ACA200EC91E03009F0252B550F3F5FBBCF1F5FC2
:10ACB200EB89EF5FEB8BB2CFE02FF0E0DE011B966A
:10ACC200EA0FFB1F2083DE0116960E943C090E94B8
:10ACD20063CC659608952D970E945ECC1A2F098940
:10ACE2003A89FE013996FA93EA93E0E0EA93A0E00A
:10ACF200B0E00E945BC5EC81EF7EEC83E07FE86010
:10AD0200EC83E32FF0E0E050FD4FED83FE831987E3
:10AD1200FE013B96008335C02D970E945ECC1A2F10
:10AD220009893A89EC81E061EC83E07FE860EC8399
:10AD3200F32FE0E066277727E060F060606D7861CE
:10AD4200DF01CB01E0915C04FF2766277727EA2B1E
:10AD5200FB2B682B792BED83FE836F837887E0E0F2
:10AD6200E987FE013A960083FE013B961083FE01BD
:10AD72003C96FA93EA93EFEFEA93A5E0B0E00E94E3
:10AD82005BC5DE0114960E943C090E9465CC639665
:10AD9200089562970E945CCCE0916304E07409F428
:10ADA2007BC4A091AC07A43038F4E091AC07EF5F0C
:10ADB200E093AC07E15003C0E0E0E093AC07A09160
:10ADC200AC07A33008F068C4AEEAB7E0E091AC0784
:10ADD200F0E0BD01ACE0B0E00E9411CDE60FF71F3C
:10ADE2005181AEEAB7E0E091AC07F0E0BD01ACE022
:10ADF200B0E00E9411CDE60FF71F1281AEEAB7E074
:10AE0200E091AC07F0E0BD01ACE0B0E00E9411CDF2
:10AE1200E60FF71F3381113010F0103108F03CC4F7
:10AE2200E091AB07F0E0E230A0E0FA0729F0E3306E
:10AE3200A0E0FA0709F030C4AEEAB7E0E091AC074F
:10AE4200F0E0BD01ACE0B0E00E9411CDDB01AE0F3D
:10AE5200BF1FAC91A13008F440C0AEEAB7E0E09168
:10AE6200AC07F0E0BD01ACE0B0E00E9411CDDB0127
:10AE7200AE0FBF1FEC91E150EC93AEEAB7E0E09168
:10AE8200AC07F0E0BD01ACE0B0E00E9411CDDB0107
:10AE9200AE0FBF1FEC91E030F9F400E0232F011751
:10AEA200D8F4A2EDB7E0E22FF0E00E94DACCAE0FC8
:10AEB200BF1F1296EC91EE7FEC93A2EDB7E0E22F6A
:10AEC200F0E00E94DACCAE0FBF1F1296EC91E26066
:10AED200EC930F5F2F5FE3CF48C0A091AB07A23086
:10AEE20009F043C0AEEAB7E0E091AC07F0E0BD0183
:10AEF200ACE0B0E00E9411CDDB01AE0FBF1F1A968D
:10AF0200AC91A13088F0AEEAB7E0E091AC07F0E096
:10AF1200BD01ACE0B0E00E9411CDDB01AE0FBF1F5E
:10AF22001A96EC91E15020C0EE81E07FE260EE8360
:10AF3200EF7EEE83E0E0EF83E887E1E0EB87E0E09D
:10AF4200EC87DE0116960E943C09AEEAB7E0E0917A
:10AF5200AC07F0E0BD01ACE0B0E00E9411CDDB0136
:10AF6200AE0FBF1F1A96E4E1EC93AEEAB7E0E091B0
:10AF7200AC07F0E0BD01ACE0B0E00E9411CDDB0116
:10AF8200AE0FBF1F1696AC910E948A3BE03011F1C2
:10AF9200A9E2B8E0E091AC07F0E0BD01AAE0B0E0C0
:10AFA2000E9411CDDB01AE0FBF1F16960E9453CE39
:10AFB2004E2FA9E2B8E0E091AC07F0E0BD01AAE0B3
:10AFC200B0E00E9411CDDB01AE0FBF1F17960E94A9
:10AFD20053CE37C0AEEAB7E0E091AC07F0E0BD0176
:10AFE200ACE0B0E00E9411CDDB01AE0FBF1F1596A1
:10AFF200AC910E948A3BE03011F1A9E2B8E0E09105
:10B00200AC07F0E0BD01AAE0B0E00E9411CDDB0187
:10B01200AE0FBF1F13960E9453CE4E2FA9E2B8E087
:10B02200E091AC07F0E0BD01AAE0B0E00E9411CDD2
:10B03200DB01AE0FBF1F14960E9453CE02C040E048
:10B04200E0E0EF8BAEEAB7E0E091AC07F0E0BD01E3
:10B05200ACE0B0E00E9411CDDB01AE0FBF1F17962E
:10B06200AC914A1799F4AEEAB7E0E091AC07F0E090
:10B07200BD01ACE0B0E00E9411CDDB01AE0FBF1FFD
:10B082001896AC91EF89EA1709F447C0AEEAB7E027
:10B09200E091AC07F0E0BD01ACE0B0E00E9411CD60
:10B0A200E60FF71F4783AEEAB7E0E091AC07F0E0A6
:10B0B200BD01ACE0B0E00E9411CDE60FF71F38965B
:10B0C200AF89A083A091AB07A23011F55A93AEEAE3
:10B0D200B7E0E091AC07F0E0BD01ACE0B0E00E9467
:10B0E20011CDDB01AE0FBF1F1896EC91EA93AEEAC9
:10B0F200B7E0E091AC07F0E0BD01ACE0B0E00E9447
:10B1020011CDDB01AE0FBF1F1796AC91E4DD05C078
:10B112005A93E88DEA93A42FFFDD00E0232F011755
:10B1220008F0E8C1A2EDB7E0E22FF0E00E94DACC2D
:10B13200AE0FBF1F1296EC91EE8BA2EDB7E0E22F9D
:10B14200F0E00E94DACCAE0FBF1F1396EC91ED8BAC
:10B15200EE89E071A1F0A7E4B8E0E22FF0E0BD01D2
:10B16200ACE0B0E00E9411CDDB01AE0FBF1F139621
:10B172000E9453CEAE2F0E945062E03009F412C0FA
:10B18200A7E4B8E0E22FF0E0BD01ACE0B0E00E943D
:10B1920011CDDB01AE0FBF1F0E9453CEE295E370CB
:10B1A200EF5F55C0ED89E270A1F0A7E4B8E0E22FAD
:10B1B200F0E0BD01ACE0B0E00E9411CDDB01AE0FCA
:10B1C200BF1F12960E9453CEAE2F0E948A3BE030E0
:10B1D20009F413C0A7E4B8E0E22FF0E0BD01ACE04F
:10B1E200B0E00E9411CDDB01AE0FBF1F0E9453CE13
:10B1F200E695E695E370EF5F2AC0ED89E170A1F074
:10B20200A7E4B8E0E22FF0E0BD01ACE0B0E00E94BC
:10B2120011CDDB01AE0FBF1F11960E9453CEAE2F90
:10B222000E948A3BE03009F411C0A7E4B8E0E22FA3
:10B23200F0E0BD01ACE0B0E00E9411CDDB01AE0F49
:10B24200BF1F0E9453CEE370EF5F01C0E0E0EC8BC2
:10B25200EE89E072A1F0A7E4B8E0E22FF0E0BD01D0
:10B26200ACE0B0E00E9411CDDB01AE0FBF1F17961C
:10B272000E9453CEAE2F0E945062E03009F411C0FA
:10B28200A7E4B8E0E22FF0E0BD01ACE0B0E00E943C
:10B2920011CDDB01AE0FBF1F14960E9453CEE29573
:10B2A20051C0ED89E870A1F0A7E4B8E0E22FF0E028
:10B2B200BD01ACE0B0E00E9411CDDB01AE0FBF1FBB
:10B2C20016960E9453CEAE2F0E948A3BE03009F4BC
:10B2D20012C0A7E4B8E0E22FF0E0BD01ACE0B0E0BC
:10B2E2000E9411CDDB01AE0FBF1F14960E9453CEF8
:10B2F200E695E69527C0ED89E470A1F0A7E4B8E0F1
:10B30200E22FF0E0BD01ACE0B0E00E9411CDDB0124
:10B31200AE0FBF1F15960E9453CEAE2F0E948A3BDE
:10B32200E03009F416C0A7E4B8E0E22FF0E0BD0176
:10B33200ACE0B0E00E9411CDDB01AE0FBF1F14964E
:10B342000E9453CEE370EF5FE295E07FAC89EA2B77
:10B35200EC8BEE89E074A1F0A7E4B8E0E22FF0E014
:10B36200BD01ACE0B0E00E9411CDDB01AE0FBF1F0A
:10B372001B960E9453CEAE2F0E945062E03009F419
:10B3820013C0A7E4B8E0E22FF0E0BD01ACE0B0E00A
:10B392000E9411CDDB01AE0FBF1F18960E9453CE43
:10B3A200E295E370EF5F57C0ED89E072A1F0A7E488
:10B3B200B8E0E22FF0E0BD01ACE0B0E00E9411CDB8
:10B3C200DB01AE0FBF1F1A960E9453CEAE2F0E9412
:10B3D2008A3BE03009F414C0A7E4B8E0E22FF0E0C1
:10B3E200BD01ACE0B0E00E9411CDDB01AE0FBF1F8A
:10B3F20018960E9453CEE695E695E370EF5F2BC058
:10B40200ED89E071A1F0A7E4B8E0E22FF0E0BD0120
:10B41200ACE0B0E00E9411CDDB01AE0FBF1F199668
:10B422000E9453CEAE2F0E948A3BE03009F412C034
:10B43200A7E4B8E0E22FF0E0BD01ACE0B0E00E948A
:10B4420011CDDB01AE0FBF1F18960E9453CEE370E1
:10B45200EF5F01C0E0E0EB8BA2EDB7E0E22FF0E09E
:10B462000E94DACCAE0FBF1FAC91EC89EA1769F4E7
:10B47200A2EDB7E0E22FF0E00E94DACCAE0FBF1FE0
:10B482001196AC91EB89EA1791F1A2EDB7E0E22FA8
:10B49200F0E00E94DACCEA0FFB1FAC89A083A2ED98
:10B4A200B7E0E22FF0E00E94DACCEA0FFB1F319600
:10B4B200AB89A083AEEAB7E0E091AC07F0E0BD0152
:10B4C200ACE0B0E00E9411CDDB01AE0FBF1F1996B8
:10B4D200E4E1EC93A091AB07A23029F45A933A939A
:10B4E200A12F7CDB04C05A930A93A22F3BDB0F5F90
:10B4F2002F5F15CEAEEAB7E0E091AC07F0E0BD01F8
:10B50200ACE0B0E00E9411CDDB01AE0FBF1F199677
:10B51200AC91A13088F0AEEAB7E0E091AC07F0E080
:10B52200BD01ACE0B0E00E9411CDDB01AE0FBF1F48
:10B532001996EC91E150AFC0A091AB07A230B1F5E2
:10B54200AEEAB7E0E091AC07F0E0BD01ACE0B0E0FC
:10B552000E9411CDDB01AE0FBF1F1996E9E0EC93FB
:10B562005A933A93A12F3ADB5A93AEEAB7E0E091AD
:10B57200AC07F0E0BD01ACE0B0E00E9411CDDB0110
:10B58200AE0FBF1F1896EC91EA93AEEAB7E0E091D6
:10B59200AC07F0E0BD01ACE0B0E00E9411CDDB01F0
:10B5A200AE0FBF1F1796AC9196DB76C0AEEAB7E03E
:10B5B200E091AC07F0E0BD01ACE0B0E00E9411CD3B
:10B5C200DB01AE0FBF1F1996EAE0EC93AEEAB7E0DB
:10B5D200E091AC07F0E0BD01ACE0B0E00E9411CD1B
:10B5E200DB01AE0FBF1F1496AC91A11790F1AEEA2A
:10B5F200B7E0E091AC07F0E0BD01ACE0B0E00E9442
:10B6020011CDDB01AE0FBF1F1496E0E0EC935A930D
:10B61200AEEAB7E0E091AC07F0E0BD01ACE0B0E02B
:10B622000E9411CDDB01AE0FBF1F1896EC91EA9379
:10B63200AEEAB7E0E091AC07F0E0BD01ACE0B0E00B
:10B642000E9411CDDB01AE0FBF1F1796AC9164DBD8
:10B6520023C0AEEAB7E0E091AC07F0E0BD01ACE098
:10B66200B0E00E9411CDE60FF71F04815A930A93AE
:10B67200A02FA30F77DAAEEAB7E0E091AC07F0E0D3
:10B68200BD01ACE0B0E00E9411CDDB01AE0FBF1FE7
:10B692001496EC91EF5FEC930E9463CC6896089548
:10B6A2000E945ECCECEAF7E0FA93EA93E0E0EA93D8
:10B6B200A9E6B0E00E945BC5A9E2B8E00E9453CEC1
:10B6C200E093AD07AAE2B8E00E9453CEE093D5071B
:10B6D20010E0123008F0A2C0ABE2B8E0E12FF0E0D7
:10B6E200BD01AAE0B0E00E9411CDDB01AE0FBF1F89
:10B6F2000E944FCE9F01ADEAB7E0E12FF0E0BD011D
:10B70200A8E2B0E00E9411CDE60FF71F3496FF9336
:10B71200EF93ABE2B8E0E12FF0E0BD01AAE0B0E0C8
:10B722000E9411CDDB01AE0FBF1F12960E9453CEB5
:10B73200AF91BF91EC93ADEAB7E0E12FF0E0BD012C
:10B74200A8E2B0E00E9411CDE60FF71F3596FF93F5
:10B75200EF93ABE2B8E0E12FF0E0BD01AAE0B0E088
:10B762000E9411CDDB01AE0FBF1F16960E9453CE71
:10B77200AF91BF91EC93ADEAB7E0E12FF0E0BD01EC
:10B78200A8E2B0E00E9411CDE60FF71F2787308BA9
:10B79200ADEAB7E0E12FF0E0BD01A8E2B0E00E941F
:10B7A20011CDDB01AE0FBF1F1E96EC91E07FE4606E
:10B7B200EC93ADEAB7E0E12FF0E0BD01A8E2B0E022
:10B7C2000E9411CDDB01AE0FBF1F1196F901319618
:10B7D200ED93FC93ADEAB7E0E12FF0E0BD01A8E202
:10B7E200B0E00E9411CDDB01AE0FBF1F5C96F901E4
:10B7F2003496ED93FC93ADEAB7E0E12FF0E0BD01A2
:10B80200A8E2B0E00E9411CDDB01AE0FBF1F5B9634
:10B81200EC91E07FE860EC931F5F5BCFAFE3B8E0B1
:10B822000E9453CEE093B507A0E4B8E00E9453CE45
:10B83200E093B807A1E4B8E00E9453CEE093DD079D
:10B84200A2E4B8E00E9453CEE093E00710E0183182
:10B85200A0F500E0A3E4B8E0E12FF0E00E94DACC2A
:10B86200AE0FBF1F11960E9453CEE03009F001E0E7
:10B87200A3E4B8E0E12FF0E00E94DACCAE0FBF1FE4
:10B8820012960E9453CEE03009F00260A3E4B8E0C1
:10B89200E12FF0E00E94DACCAE0FBF1F13960E9498
:10B8A20053CEE03009F00460ADEFB7E0E12FF0E0F5
:10B8B200EA0FFB1F00831F5FCACF0E9465CC24964C
:10B8C2000895BA93AA930E945CCC10E0123008F05B
:10B8D200CDC0ADEAB7E0E12FF0E0BD01A8E2B0E0F3
:10B8E2000E9411CDDB01AE0FBF1FEC91E030B1F031
:10B8F200ADEAB7E0E12FF0E0BD01A8E2B0E00E94BE
:10B9020011CDE60FF71F01801280AE81BF81119623
:10B91200ED91FC911197E015F10509F0A5C0EE81BA
:10B92200FF810581ADEAB7E0E12FF0E0BD01A8E2B9
:10B93200B0E00E9411CDE60FF71F2681ADEAB7E015
:10B94200E12FF0E0BD01A8E2B0E00E9411CDE60FC8
:10B95200F71F5085ADEAB7E0E12FF0E0BD01A8E2A4
:10B96200B0E00E9411CDE60FF71F37812523A02FEB
:10B97200A523EFEFE327EA232E27E52FE095E02327
:10B982002E2BADEAB7E0E12FF0E0BD01A8E2B0E076
:10B992000E9411CDE60FF71F2683ADEAB7E0E12F33
:10B9A200F0E0BD01A8E2B0E00E9411CDE60FF71F62
:10B9B2000783EE81FF81E681EF700E2FADEAB7E0DB
:10B9C200E12FF0E0BD01A8E2B0E00E9411CDE60F48
:10B9D200F71F2185ADEAB7E0E12FF0E0BD01A8E253
:10B9E200B0E00E9411CDE60FF71F5385ADEAB7E034
:10B9F200E12FF0E0BD01A8E2B0E00E9411CDE60F18
:10BA0200F71F32852523A02FA523EFEFE327EA2393
:10BA12002E27E52FE095E0232E2BADEAB7E0E12FAC
:10BA2200F0E0BD01A8E2B0E00E9411CDE60FF71FE1
:10BA32002187ADEAB7E0E12FF0E0BD01A8E2B0E076
:10BA42000E9411CDE60FF71F0287ADEAB7E0E12FA2
:10BA5200F0E0BD01A8E2B0E00E9411CDDB01AE0F23
:10BA6200BF1F1396EAE0EC931F5F30CF0E9463CCB6
:10BA72002896089524970E945CCCE0916304E074B8
:10BA820009F4BBC3A091AC07A43038F4E091AC0731
:10BA9200EF5FE093AC07E15003C0E0E0E093AC0756
:10BAA200A091AC07A23008F0A8C3ADEAB7E0E091DC
:10BAB200AC07F0E0BD01A8E2B0E00E9411CDDB01CD
:10BAC200AE0FBF1FEC91E03009F497C3ADEAB7E0C7
:10BAD200E091AC07F0E0BD01A8E2B0E00E9411CD18
:10BAE200DB01AE0FBF1F1396AC91A13008F463C007
:10BAF200ADEAB7E0E091AC07F0E0BD01A8E2B0E04A
:10BB02000E9411CDDB01AE0FBF1F1396EC91E150E5
:10BB1200EC93ADEAB7E0E091AC07F0E0BD01A8E23A
:10BB2200B0E00E9411CDDB01AE0FBF1F1396EC9166
:10BB3200E03009F040C0ADEAB7E0E091AC07F0E0D8
:10BB4200BD01A8E2B0E00E9411CDDB01AE0FBF1F24
:10BB52001696E0E0EC93ADEAB7E0E091AC07F0E0D6
:10BB6200BD01A8E2B0E00E9411CDDB01AE0FBF1F04
:10BB72001796E0E0EC93ADEAB7E0E091AC07F0E0B5
:10BB8200BD01A8E2B0E00E9411CDDB01AE0FBF1FE4
:10BB92001996E0E0EC93ADEAB7E0E091AC07F0E093
:10BBA200BD01A8E2B0E00E9411CDDB01AE0FBF1FC4
:10BBB2001A96E0E0EC93E0E02E2F3E2FE091AC07E6
:10BBC200E03011F450E001C05CE040E011E01030E0
:10BBD20009F47DC0ADEFB7E0EE27A50FBE1F0C91B3
:10BBE20002FF10C0A3E4B8E0E52FF0E00E94DACC37
:10BBF200AE0FBF1F13960E9453CEAE2F0E9450620B
:10BC0200E03009F40EC0A3E4B8E0E52FF0E00E94B2
:10BC1200DACCAE0FBF1F0E9453CEE295E370EE83E3
:10BC220043C001FF10C0A3E4B8E0E52FF0E00E949A
:10BC3200DACCAE0FBF1F12960E9453CEAE2F0E94D7
:10BC42008A3BE03009F40FC0A3E4B8E0E52FF0E04E
:10BC52000E94DACCAE0FBF1F0E9453CEE695E69546
:10BC6200E370EE8321C000FF10C0A3E4B8E0E52F2B
:10BC7200F0E00E94DACCAE0FBF1F11960E9453CEA5
:10BC8200AE2F0E948A3BE03009F40DC0A3E4B8E075
:10BC9200E52FF0E00E94DACCAE0FBF1F0E9453CE18
:10BCA200E370EE8301C010C0EE81F0E0309711F432
:10BCB200312B0AC0E130A0E0FA0729F0E230A0E01F
:10BCC200FA0711F4312B212B5F5F110F80CFADEA00
:10BCD200B7E0E091AC07F0E0BD01A8E2B0E00E945D
:10BCE20011CDE60FF71FA0A13A1771F0ADEAB7E048
:10BCF200E091AC07F0E0BD01A8E2B0E00E9411CDF6
:10BD0200E60FF71F30A341E0ADEAB7E0E091AC07E0
:10BD1200F0E0BD01A8E2B0E00E9411CDE60FF71FEE
:10BD2200A2A12A1771F0ADEAB7E0E091AC07F0E00A
:10BD3200BD01A8E2B0E00E9411CDE60FF71F22A3D9
:10BD420041E0E0E02E2F3E2F11E0103109F47CC0DB
:10BD5200ADEFB7E0EE27A50FBE1F0C9102FF0FC09B
:10BD6200A3E4B8E0E52FF0E00E94DACCAE0FBF1FEB
:10BD720013960E9453CEAE2F92D3E03009F40EC038
:10BD8200A3E4B8E0E52FF0E00E94DACCAE0FBF1FCB
:10BD92000E9453CEE295E370EE8343C001FF10C0D0
:10BDA200A3E4B8E0E52FF0E00E94DACCAE0FBF1FAB
:10BDB20012960E9453CEAE2F0E948A3BE03009F4C5
:10BDC2000FC0A3E4B8E0E52FF0E00E94DACCAE0F9A
:10BDD200BF1F0E9453CEE695E695E370EE8321C025
:10BDE20000FF10C0A3E4B8E0E52FF0E00E94DACC37
:10BDF200AE0FBF1F11960E9453CEAE2F0E948A3BF8
:10BE0200E03009F40DC0A3E4B8E0E52FF0E00E94B1
:10BE1200DACCAE0FBF1F0E9453CEE370EE8301C097
:10BE220010C0EE81F0E0309711F4312B0AC0E130FE
:10BE3200A0E0FA0729F0E230A0E0FA0711F4312B72
:10BE4200212B5F5F110F81CFADEAB7E0E091AC0724
:10BE5200F0E0BD01A8E2B0E00E9411CDE60FF71FAD
:10BE6200A1A13A1771F0ADEAB7E0E091AC07F0E0BA
:10BE7200BD01A8E2B0E00E9411CDE60FF71F31A389
:10BE820041E0ADEAB7E0E091AC07F0E0BD01A8E225
:10BE9200B0E00E9411CDE60FF71FA3A12A1771F09F
:10BEA200ADEAB7E0E091AC07F0E0BD01A8E2B0E096
:10BEB2000E9411CDE60FF71F23A341E0403089F421
:10BEC200ADEAB7E0E091AC07F0E0BD01A8E2B0E076
:10BED2000E9411CDDB01AE0FBF1F1D96AC91A130A8
:10BEE20008F412C0ADEAB7E0E091AC07F0E0BD01A2
:10BEF200A8E2B0E00E9411CDDB01AE0FBF1F1D967C
:10BF0200EC91E150EC9320C0ADEAB7E0E091AC07D0
:10BF1200F0E0BD01A8E2B0E00E9411CDDB01AE0F5E
:10BF2200BF1F1D96E0E1EC93ADEAB7E0E091AC07EC
:10BF3200F0E0BD01A8E2B0E00E9411CDDB01AE0F3E
:10BF4200BF1F5B960E943C09ADEAB7E0E091AC07E7
:10BF5200F0E0BD01A8E2B0E00E9411CDDB01AE0F1E
:10BF6200BF1F1496AC91A03091F4ADEAB7E0E09116
:10BF7200AC07F0E0BD01A8E2B0E00E9411CDDB0108
:10BF8200AE0FBF1F1596AC91A03009F436C140E048
:10BF9200E1E0E987EFE0E887EF83ADEAB7E0E0911F
:10BFA200AC07F0E0BD01A8E2B0E00E9411CDDB01D8
:10BFB200AE0FBF1F1596AC910E948A3BE03089F10B
:10BFC200ABE2B8E0E091AC07F0E0BD01AAE0B0E07E
:10BFD2000E9411CDDB01AE0FBF1F17960E9453CEF8
:10BFE200E987ABE2B8E0E091AC07F0E0BD01AAE07E
:10BFF200B0E00E9411CDDB01AE0FBF1F18960E9468
:10C0020053CEE887ABE2B8E0E091AC07F0E0BD01C7
:10C01200AAE0B0E00E9411CDDB01AE0FBF1F19965E
:10C0220043C0ADEAB7E0E091AC07F0E0BD01A8E2A1
:10C03200B0E00E9411CDDB01AE0FBF1F1496AC9190
:10C042000E948A3BE03099F1ABE2B8E0E091AC07A4
:10C05200F0E0BD01AAE0B0E00E9411CDDB01AE0F1D
:10C06200BF1F13960E9453CEE987ABE2B8E0E0917E
:10C07200AC07F0E0BD01AAE0B0E00E9411CDDB0107
:10C08200AE0FBF1F14960E9453CEE887ABE2B8E012
:10C09200E091AC07F0E0BD01AAE0B0E00E9411CD52
:10C0A200DB01AE0FBF1F15960E9453CEEF83ADEAA0
:10C0B200B7E0E091AC07F0E0BD01A8E2B0E00E9479
:10C0C20011CDE60FF71FA489E985EA1781F0ADEAE1
:10C0D200B7E0E091AC07F0E0BD01A8E2B0E00E9459
:10C0E20011CDE60FF71F7496A985A08341E0ADEA52
:10C0F200B7E0E091AC07F0E0BD01A8E2B0E00E9439
:10C1020011CDE60FF71FA589E885EA1781F0ADEAA0
:10C11200B7E0E091AC07F0E0BD01A8E2B0E00E9418
:10C1220011CDE60FF71F7596A885A08341E0ADEA11
:10C13200B7E0E091AC07F0E0BD01A8E2B0E00E94F8
:10C1420011CDE60FF71FA689EF81EA1781F0ADEA5C
:10C15200B7E0E091AC07F0E0BD01A8E2B0E00E94D8
:10C1620011CDE60FF71F7696AF81A08341E04030F4
:10C1720089F4ADEAB7E0E091AC07F0E0BD01A8E2D6
:10C18200B0E00E9411CDDB01AE0FBF1F1C96AC9137
:10C19200A13008F412C0ADEAB7E0E091AC07F0E0DC
:10C1A200BD01A8E2B0E00E9411CDDB01AE0FBF1FBE
:10C1B2001C96EC91E150EC9320C0ADEAB7E0E0911F
:10C1C200AC07F0E0BD01A8E2B0E00E9411CDDB01B6
:10C1D200AE0FBF1F1C96E0E1EC93ADEAB7E0E09131
:10C1E200AC07F0E0BD01A8E2B0E00E9411CDDB0196
:10C1F200AE0FBF1F1E960E943C090E9463CC2A9676
:10C20200089508951A931A2FA9E01A9FF001E65093
:10C21200F74FA081A73B21F4A12F0E9417833DC1B4
:10C222001730D0F4103011F42D9815C0113011F4DC
:10C23200109811C0123011F42E980DC0133011F461
:10C24200A19809C0143011F4739805C0153011F487
:10C25200A29801C0A09825C01D30B0F4173011F487
:10C262005F9811C0183011F42F980DC0193011F4D5
:10C27200139809C01A3011F4749805C01B3011F4D8
:10C28200149801C075980DC0123158F41D3011F484
:10C292008C9807C01E3011F42C9803C01F3009F48B
:10C2A2008D98FBC01A931A2F1730D0F4103011F466
:10C2B2002D9A15C0113011F4109A11C0123011F4D8
:10C2C2002E9A0DC0133011F4A19A09C0143011F442
:10C2D200739A05C0153011F4A29A01C0A09A25C024
:10C2E2001D30B0F4173011F45F9A11C0183011F4F8
:10C2F2002F9A0DC0193011F4139A09C01A3011F493
:10C30200749A05C01B3011F4149A01C0759A0DC0BD
:10C31200123158F41D3011F48C9A07C01E3011F4FA
:10C322002C9A03C01F3009F48D9AB7C01A931A2FA2
:10C332001730D0F4103011F42D9815C0113011F4CB
:10C34200109811C0123011F42E980DC0133011F450
:10C35200A19809C0143011F4739805C0153011F476
:10C36200A29801C0A09825C01D30B0F4173011F476
:10C372005F9811C0183011F42F980DC0193011F4C4
:10C38200139809C01A3011F4749805C01B3011F4C7
:10C39200149801C075980DC0123158F41D3011F473
:10C3A2008C9807C01E3011F42C9803C01F3009F47A
:10C3B2008D9873C01A931A2FEEEAF4E060E070E0F1
:10C3C2000E94E5CDE12FFF27662777270E94E5CD62
:10C3D20084E00E94E3CB289611501730A0F4E12F9D
:10C3E200A1E00E947ECC1E2FA091E608E095EA23F0
:10C3F200E093E608E091E708E12BE093E708E0E04C
:10C40200E093E30816C01830A0F41850E12FA1E021
:10C412000E947ECC1E2FA091E808E095EA23E093CB
:10C42200E808E091E908E12BE093E908E0E0E09315
:10C43200E40833C01A931A2FEFEBF4E060E070E0E7
:10C442000E94E5CDE12FFF27662777270E94E5CDE1
:10C4520084E00E94E3CB28961150173070F4E12F4C
:10C46200A1E00E947ECC1E2FE091E608E12BE09332
:10C47200E608E0E0E093E30810C0183070F41850CA
:10C48200E12FA1E00E947ECC1E2FE091E808E12B73
:10C49200E093E808E0E0E093E408199108950E942F
:10C4A2005ECC3A2F3F3010F03F3108F01EC0E32F30
:10C4B200EF501E2FA9E01A9FF001E950F74FE081DB
:10C4C200E47011F0E1E074C2A9E01A9FF001E950B2
:10C4D200F74FE081E295E7700E2F013021F0043032
:10C4E20011F0053011F4E1E063C2A32F0E945D7CDC
:10C4F2005FC20E945ECCE091EF08EF7EE093EF080E
:10C50200EF7DE093EF08E4E1E093F308E091EF08B8
:10C51200EF7BE093EF08E091F008EE7FE093F00804
:10C52200ED7FE093F008E7EFF8E0FA93EA93E0E0BA
:10C53200EA93A0E9B0E00E945BC5089A999A9A9A98
:10C54200989A0B9A6C9A859AE2B1E67EE2B9E5B1C5
:10C55200EF70E5B95F98EEB1E77CEEB9E1B3EF7C3D
:10C56200E1BBE4B3E87FE4BBEFEFE093E608E093DE
:10C57200E80810E0103108F008C2A9E01A9FF001A3
:10C58200E650F74FFF93EF93A5E4B1E0E12FF0E01F
:10C59200BD01A7E0B0E00E9411CDDB01AE0FBF1FCD
:10C5A2000E9453CEAF91BF91EC93A9E01A9FF00184
:10C5B200E950F74FFF93EF93A5E4B1E0E12FF0E0EC
:10C5C200BD01A7E0B0E00E9411CDDB01AE0FBF1F9D
:10C5D20012960E9453CEE07121F5A5E4B1E0E12F5D
:10C5E200F0E0BD01A7E0B0E00E9411CDDB01AE0F8B
:10C5F200BF1F12960E9453CEE07299F4A5E4B1E0F7
:10C60200E12FF0E0BD01A7E0B0E00E9411CDDB0117
:10C61200AE0FBF1F12960E9453CEE07411F4E0E0F9
:10C6220001C0E1E0AF91BF91E170EE0F0E2EEC91EF
:10C63200ED7FE029EC93A5E4B1E0E12FF0E0BD014C
:10C64200A7E0B0E00E9411CDDB01AE0FBF1F15962F
:10C652000E9453CEE07249F0A9E01A9FF001E8501F
:10C66200F74FDF01EC91E061EC93A5E4B1E0E12F3B
:10C67200F0E0BD01A7E0B0E00E9411CDDB01AE0FFA
:10C68200BF1F15960E9453CEE07449F0A9E01A9F8D
:10C69200F001E850F74FDF01EC91E062EC93A5E482
:10C6A200B1E0E12FF0E0BD01A7E0B0E00E9411CDC2
:10C6B200DB01AE0FBF1F12960E9453CEE07859F0F5
:10C6C200183020F4E091EF08E06103C0E091EF0838
:10C6D200E062E093EF08A7E6B9E0E12FF0E0F5951C
:10C6E200E795AE0FBF1F0E9453CE0E2F10FF0DC055
:10C6F200E02FE07F49F0A9E01A9FF001E950F74FDF
:10C70200DF01EC91E068EC930CC0E02FEF7049F090
:10C71200A9E01A9FF001E950F74FDF01EC91E068C0
:10C72200EC93A9E01A9FF001E650F74FA081A633DF
:10C7320009F03FC0E12FFF2766277727E056FF4F1A
:10C742006F4F6BBF3691303148F4A9E03A9FF00148
:10C75200E850F74FDF01EC91E064EC93E12FF0E059
:10C76200E130A0E0FA0711F4089823C0E330A0E01A
:10C77200FA0711F499981DC0E530A0E0FA0711F408
:10C782009A9817C0E630A0E0FA0711F4989811C001
:10C79200E930A0E0FA0711F40B980BC0EA30A0E0F0
:10C7A200FA0711F46C9805C0EF30A0E0FA0709F41B
:10C7B2008598A5E4B1E0E12FF0E0BD01A7E0B0E08B
:10C7C2000E9411CDDB01AE0FBF1F15960E9453CE02
:10C7D200E07409F4D8C0183008F06AC0E12FF0E024
:10C7E200309749F4E091E608EE7FE093E608E091A5
:10C7F200E708E1605AC0E130A0E0FA0749F4E091AD
:10C80200E608ED7FE093E608E091E708E2604DC0BC
:10C81200E230A0E0FA0749F4E091E608EF7EE09307
:10C82200E608E091E708E06140C0E330A0E0FA07E3
:10C8320049F4E091E608EF77E093E608E091E70833
:10C84200E06833C0E430A0E0FA0749F4E091E6087A
:10C85200EB7FE093E608E091E708E46026C0E5306C
:10C86200A0E0FA0749F4E091E608EF7DE093E608DC
:10C87200E091E708E06219C0E630A0E0FA0749F467
:10C88200E091E608EF7BE093E608E091E708E064D8
:10C892000CC0E730A0E0FA0751F4E091E608E77F28
:10C8A200E093E608E091E708E860E093E7086BC0F0
:10C8B200E12FF0E0E830A0E0FA0749F4E091E8085F
:10C8C200EE7FE093E808E091E908E1605AC0E930C0
:10C8D200A0E0FA0749F4E091E808EF77E093E8086E
:10C8E200E091E908E0684DC0EA30A0E0FA0749F4B7
:10C8F200E091E808EF7BE093E808E091E908E06462
:10C9020040C0EB30A0E0FA0749F4E091E808EF7D7F
:10C91200E093E808E091E908E06233C0EC30A0E07F
:10C92200FA0749F4E091E808EF7EE093E808E09125
:10C93200E908E06126C0ED30A0E0FA0749F4E09191
:10C94200E808E77FE093E808E091E908E86019C0A9
:10C95200EE30A0E0FA0749F4E091E808EB7FE093BB
:10C96200E808E091E908E4600CC0EF30A0E0FA07C3
:10C9720051F4E091E808ED7FE093E808E091E908DE
:10C98200E260E093E9081F5FF5CDE0E0E093E308A1
:10C99200E093E408E091EF08E07111F0A39A01C07E
:10C9A200A398E091EF08E07211F0A49A01C0A49854
:10C9B2000E9465CC2496089527970E945CCCE09152
:10C9C200F108EF73E03100F1A398A498E091F10827
:10C9D200E07CE093F108E091EE08E770E063E09319
:10C9E200EE08E2B1E67EE2B9E5B1EF70E5B95F9833
:10C9F200EEB1E77CEEB9E1B3EF7CE1BBE4B3E87FF3
:10CA0200E4BBA0E04FDCB6C2E091EE08E87FE8307C
:10CA120008F4B0C2AEEEB8E083E0EFE10E9419CEB6
:10CA2200E091EE08E87FE830D1F4A1E4B8E0E091CB
:10CA3200F108EF73FF2766277727E054FF4F6F4F08
:10CA42006BBFE691F0E0EE0FFF1FAE0FBF1FED913F
:10CA5200FC911197E093F508F093F6088BC2E091F0
:10CA6200EE08E87F09F086C2A1E4B8E0E091F1089F
:10CA7200EF73FF2766277727E054FF4F6F4F6BBF97
:10CA8200E691F0E0EE0FFF1FAE0FBF1FED91FD919B
:10CA9200A091F508B091F608EA0FFB1FE093F508A4
:10CAA200F093F608A091F508B091F608E091F60827
:10CAB200F070EA0FFB1FE093F508F093F6080E946E
:10CAC200ECCCE093F508F093F608E091EE08F0E084
:10CAD200E770F070E230A0E0FA07E1F5A2E3B0E01F
:10CAE200E091F108EF73F0E0BD01AAE0B0E00E942E
:10CAF20011CDDB01AE0FBF1FE091F508F091F608F2
:10CB02000E9467CEE091F108EF73FF27662777272F
:10CB1200E053FF4F6F4F6BBFE691E03061F4EEE4FC
:10CB2200F1E060E070E00E94D4CD9F01EEE6F1E01A
:10CB320060E070E00BC0EEE8F1E060E070E00E94BF
:10CB4200D4CD9F01EEEAF1E060E070E00E94D4CD26
:10CB5200AF0103C1E330A0E0FA07E9F5A2E3B0E0D8
:10CB6200E091F108EF73F0E0BD01AAE0B0E00E94AD
:10CB720011CDDB01AE0FBF1F1296E091F508F091C7
:10CB8200F6080E9467CEE091F108EF73FF2766274F
:10CB92007727E053FF4F6F4F6BBFE691E03061F4B0
:10CBA200E0E5F1E060E070E00E94D4CD9F01E0E7B3
:10CBB200F1E060E070E00BC0E0E9F1E060E070E01D
:10CBC2000E94D4CD9F01E0EBF1E060E070E00E94B2
:10CBD200D4CDAF01C2C0E430A0E0FA07E9F5A2E388
:10CBE200B0E0E091F108EF73F0E0BD01AAE0B0E03F
:10CBF2000E9411CDDB01AE0FBF1F1496E091F50824
:10CC0200F091F6080E9467CEE091F108EF73FF27DA
:10CC120066277727E053FF4F6F4F6BBFE691E030F7
:10CC220061F4E2E5F1E060E070E00E94D4CD9F01A2
:10CC3200E2E7F1E060E070E00BC0E2E9F1E060E021
:10CC420070E00E94D4CD9F01E2EBF1E060E070E081
:10CC52000E94D4CDAF0181C0E530A0E0FA07E9F52A
:10CC6200A2E3B0E0E091F108EF73F0E0BD01AAE0C9
:10CC7200B0E00E9411CDDB01AE0FBF1F1696E0910E
:10CC8200F508F091F6080E9467CEE091F108EF7383
:10CC9200FF2766277727E053FF4F6F4F6BBFE69161
:10CCA200E03061F4E4E5F1E060E070E00E94D4CDB0
:10CCB2009F01E4E7F1E060E070E00BC0E4E9F1E03D
:10CCC20060E070E00E94D4CD9F01E4EBF1E060E00F
:10CCD20070E00E94D4CDAF0140C0E630A0E0FA0778
:10CCE200E1F5A2E3B0E0E091F108EF73F0E0BD01FD
:10CCF200AAE0B0E00E9411CDDB01AE0FBF1F189673
:10CD0200E091F508F091F6080E9467CEE091F108F3
:10CD1200EF73FF2766277727E053FF4F6F4F6BBFF5
:10CD2200E691E03061F4E6E5F1E060E070E00E9457
:10CD3200D4CD9F01E6E7F1E060E070E00BC0E6E9E8
:10CD4200F1E060E070E00E94D4CD9F01E6EBF1E0FB
:10CD520060E070E00E94D4CDAF01E4EDF4E060E069
:10CD620070E00E94E5CDE091F108EF73F0E03196BA
:10CD72006F2F660F660B762F0E94E5CDE091F508C6
:10CD8200F091F608662777270E94E5CD88E00E9499
:10CD9200E3CB2C96A091F508B091F608A217B30741
:10CDA20018F04A175B0708F402C011E013C010E044
:10CDB200E091F208EC7771F4A2EFB8E0E091F108AB
:10CDC200EF73EF5FEF71EE0FEE0F0E2EEC91E37843
:10CDD200E029EC93A12F0E94DBBCE7E0EF83E9EFAF
:10CDE200E887E985E160E987E12FE170EE0F0E2E19
:10CDF200E985ED7FE029E987E091F108EF73EF5FC4
:10CE0200EF73EE0FEE0F0E2EE985E370E029E9874E
:10CE1200E091F508F091F608EB87FC87E091EE08C7
:10CE2200F0E0E770F070E230A0E0FA0711F4E1E020
:10CE320019C0E330A0E0FA0711F4E2E013C0E430D5
:10CE4200A0E0FA0711F4E3E00DC0E530A0E0FA0734
:10CE520011F4E4E007C0E630A0E0FA0711F4E5E0DF
:10CE620001C0E0E0EA87E2B1E67EE2B9E5B1EF7047
:10CE7200E5B95F98EEB1E77CEEB9E1B3EF7CE1BBD7
:10CE8200E4B3E87FE4BBDE0116960E94BA92E09119
:10CE9200F108EF73EF3090F4A1EFB8E080E0EFE338
:10CEA2000E9415CEE091EE08E770E062E093EE0892
:10CEB200E091F108EF73AE2FF5D95CC0A2E2B0E0C9
:10CEC2000E9453CE1E2EE091EE08E770E250A1E0E0
:10CED2000E947ECCE129A2E2B0E00E946FCEEFED8B
:10CEE200F4E060E070E00E94E5CD80E00E94E3CBD8
:10CEF2002496E091F208EC7791F4EAEEF4E060E037
:10CF020070E00E94E5CD80E00E94E3CB2496E091A0
:10CF1200EE08E770E23011F40E94A83514C0EEEE7C
:10CF2200F4E060E070E00E94E5CDE091F208E69561
:10CF3200E695EF71FF27662777270E94E5CD84E00B
:10CF42000E94E3CB2896E091EF08E07111F0A39ADA
:10CF520001C0A398E091EF08E07211F0A49A01C019
:10CF6200A498E091EE08E87FE160E093EE08E6E045
:10CF7200E093940D0E9463CC2D9608952F970E9402
:10CF82005CCCE091F108EF73E03100F1E091F1083F
:10CF9200E07CE093F108E091EE08E770E062E09354
:10CFA200EE08A398A498E2B1E67EE2B9E5B1EF708B
:10CFB200E5B95F98EEB1E77CEEB9E1B3EF7CE1BB96
:10CFC200E4B3E87FE4BBA0E06DD938C2E091EE089B
:10CFD200E87FE83008F432C2E091F108EF730E2FD7
:10CFE200AEEEB8E083E0EFE10E9419CEE091EE08E8
:10CFF200E87FE830D1F40031B8F4A1E4B8E0E02FE2
:10D00200FF2766277727E054FF4F6F4F6BBFE691EC
:10D01200F0E0EE0FFF1FAE0FBF1FED91FC911197D5
:10D02200E093F508F093F60809C2E091EE08E87F74
:10D0320009F004C2E7E0EF83E9EFE887E6E0EA8778
:10D04200E985E160E987E260E987E091F108EF7341
:10D05200EF5FEF73EE0FEE0F0E2EE985E370E0291E
:10D06200E987E0E0EB87EC87003108F0AAC1A1E490
:10D07200B8E0E02FFF2766277727E054FF4F6F4F76
:10D082006BBFE691F0E0EE0FFF1FAE0FBF1FED91F9
:10D09200FD91A091F508B091F608AE0FBF1FFD01FA
:10D0A2000E94ECCC9F01A2E3B0E0E02FF0E0BD01D2
:10D0B200AAE0B0E00E9411CDDB01AE0FBF1F0E94BB
:10D0C2004FCEAF014217530718F020E030E0E1C025
:10D0D200A2E3B0E0E02FF0E0BD01AAE0B0E00E94E0
:10D0E20011CDDB01AE0FBF1F12960E944FCEEB8B0C
:10D0F200FC8BE217F30708F1241B350BF9016627B5
:10D1020077276E2F7F2FE0E0F0E07F936F93FF93FE
:10D11200EF93EB89FC89E41BF50B66277727AFE8D1
:10D12200B2E080E090E00E9419CDAF91BF918F9163
:10D132009F910E946FCD9F01ACC0A2E3B0E0E02FAF
:10D14200F0E0BD01AAE0B0E00E9411CDDB01AE0F1C
:10D15200BF1F14960E944FCEE98BFA8BE217F3079A
:10D1620030F1AB89BC892A1B3B0BD901882799274F
:10D17200E1E10E94A8CC7F936F93FF93EF93AB8979
:10D18200BC89E989FA89EA1BFB0B66277727AFE896
:10D19200B2E080E090E00E9419CDAF91BF918F91F3
:10D1A2009F910E946FCD9F012C593F4F72C0A2E305
:10D1B200B0E0E02FF0E0BD01AAE0B0E00E9411CDA6
:10D1C200DB01AE0FBF1F16960E944FCEEF87F88B82
:10D1D200E217F30730F1A989BA892A1B3B0BD9015F
:10D1E20088279927E1E10E94A8CC7F936F93FF9350
:10D1F200EF93A989BA89EF85F889EA1BFB0B6627A9
:10D202007727A4EBB1E080E090E00E9419CDAF91C6
:10D21200BF918F919F910E946FCD9F01245D3E4FE0
:10D2220038C0A2E3B0E0E02FF0E0BD01AAE0B0E038
:10D232000E9411CDDB01AE0FBF1F18960E944FCE88
:10D24200ED87FE87AF85B8892A1B3B0BD90188275A
:10D252009927E3E10E94A8CC7F936F93FF93EF930A
:10D26200AF85B889ED85FE85EA1BFB0BF695E79540
:10D2720066277727ACEEB2E080E090E00E9419CDFD
:10D28200AF91BF918F919F910E946FCD9F01285ABC
:10D292003D4FE3E0F5E060E070E00E94E5CDE02F75
:10D2A200F0E031966F2F660F660B762F0E94E5CD68
:10D2B200F901662777270E94ECCEDF01CB01E0E07F
:10D2C200F0E068EC72E40E94C3CF0E94E5CD88E0F2
:10D2D2000E94E3CB2C96F6982B873C8710E0103106
:10D2E20008F06FC00117B1F5A3E9B8E0E12FFF27FD
:10D2F20066277727E055FF4F6F4F6BBFE691F0E04F
:10D30200AE0FBF1FEC91E07421F5E2E1F5E060E0C1
:10D3120070E00E94E5CDE02FF0E031966F2F660FAE
:10D32200660B762F0E94E5CDE12FF0E031966F2F4C
:10D33200660F660B762F0E94E5CD88E00E94E3CB54
:10D342002C96E091F208E260E093F208E985ED7F25
:10D35200E98735C0A3E9B8E0E12FFF2766277727E1
:10D36200E055FF4F6F4F6BBFE691F0E0AE0FBF1F6E
:10D37200EC91E07421F1ECE2F5E060E070E00E94F3
:10D38200E5CDE02FF0E031966F2F660F660B762F1A
:10D392000E94E5CDE12FF0E031966F2F660F660B0C
:10D3A200762F0E94E5CD88E00E94E3CB2C96E09197
:10D3B200F208E260E093F208E985ED7FE9871F5FFA
:10D3C2008ECFE091F108EF730E2FA02F0E9497618C
:10D3D200DE0116960E94BA920F3098F4A1EFB8E0DF
:10D3E20080E0EFE30E9415CEE091F108EF73AE2FDB
:10D3F2000E945361E091EE08E770E062E093EE086C
:10D402001DC0E9E4F5E060E070E00E94E5CD80E057
:10D412000E94E3CB2496E091F208E695E170A0E049
:10D42200EA17E1E009F0EE27AE2F0E94DBBCE091A3
:10D43200EE08E87FE093EE08A398A4980E9463CCDC
:10D442006596089526970E945CCCE5E5F5E060E0DC
:10D4520070E00E94E5CDABE1B0E00E944FCE6627BE
:10D4620077270E94E5CD84E00E94E3CB2896ABE1CA
:10D47200B0E00E944FCEE03CA3E3FA0740F0ABE1FC
:10D48200B0E00E944FCEE134AFE3FA0708F002C0E9
:10D4920021E001C020E0A22F0E94DBBCE6E6F5E01D
:10D4A20060E070E00E94E5CDADE1B0E00E944FCEB9
:10D4B200662777270E94E5CDAFE1B0E00E944FCE0C
:10D4C200662777270E94E5CD88E00E94E3CB2C9661
:10D4D200ADE1B0E00E944FCEE53AA7E1FA07C0F015
:10D4E200ADE1B0E00E944FCEE73EACE1FA0780F436
:10D4F200AFE1B0E00E944FCEE53AA7E1FA0740F073
:10D50200AFE1B0E00E944FCEE73EACE1FA0708F08F
:10D5120002C051E001C050E0A52F0E94DBBCEFE742
:10D52200F5E060E070E00E94E5CDA2E2B0E00E948A
:10D5320053CEFF27662777270E94E5CD84E00E941D
:10D54200E3CB2896E0E01E2F3E2F103108F03EC1BB
:10D55200E4E9F5E060E070E00E94E5CDE12FF0E063
:10D5620031966F2F660F660B762F0E94E5CDA2E3F0
:10D57200B0E0E12FF0E0BD01AAE0B0E00E9411CDE1
:10D58200DB01AE0FBF1F0E944FCE662777270E9496
:10D59200E5CDA2E3B0E0E12FF0E0BD01AAE0B0E00A
:10D5A2000E9411CDDB01AE0FBF1F12960E944FCE1B
:10D5B200662777270E94E5CDA2E3B0E0E12FF0E0F5
:10D5C200BD01AAE0B0E00E9411CDDB01AE0FBF1F8A
:10D5D20014960E944FCE662777270E94E5CDA2E3DC
:10D5E200B0E0E12FF0E0BD01AAE0B0E00E9411CD71
:10D5F200DB01AE0FBF1F16960E944FCE662777271C
:10D602000E94E5CDA2E3B0E0E12FF0E0BD01AAE087
:10D61200B0E00E9411CDDB01AE0FBF1F18960E9431
:10D622004FCE662777270E94E5CD88E10E94E3CBA3
:10D632006C9600E0053008F0B6C0E02FF0E03097BD
:10D6420069F4A2E3B0E0E12FF0E0BD01AAE0B0E0AE
:10D652000E9411CDDB01AE0FBF1F47C0E130A0E039
:10D66200FA0771F4A2E3B0E0E12FF0E0BD01AAE015
:10D67200B0E00E9411CDDB01AE0FBF1F129635C084
:10D68200E230A0E0FA0771F4A2E3B0E0E12FF0E0AB
:10D69200BD01AAE0B0E00E9411CDDB01AE0FBF1FB9
:10D6A200149623C0E330A0E0FA0771F4A2E3B0E0DD
:10D6B200E12FF0E0BD01AAE0B0E00E9411CDDB0154
:10D6C200AE0FBF1F169611C0E430A0E0FA0789F42E
:10D6D200A2E3B0E0E12FF0E0BD01AAE0B0E00E94D9
:10D6E20011CDDB01AE0FBF1F18960E944FCEEE8305
:10D6F200FF83E12FFF2766277727E053FF4F6F4F06
:10D702006BBFE691E030C1F4E02FAEE4B1E080E01F
:10D71200FF2766277727EE0FFF1F661F771FEA0F87
:10D72200FB1F681F791F0E94D4CDEA87FB87E02F79
:10D73200AEE6B1E080E017C0E02FAEE8B1E080E0F5
:10D74200FF2766277727EE0FFF1F661F771FEA0F57
:10D75200FB1F681F791F0E94D4CDEA87FB87E02F49
:10D76200AEEAB1E080E0FF2766277727EE0FFF1FC2
:10D77200661F771FEA0FFB1F681F791F0E94D4CD17
:10D78200E887F987EE81FF81AA85BB85EA17FB0747
:10D7920038F0E885F985AE81BF81EA17FB0708F406
:10D7A20002C00F5F47CFA02FE5E0EA17E1E009F0E2
:10D7B200EE27AE2F0E94DBBC053010F4303009F0AA
:10D7C20003C0E12FEF5F3E2F1F5FBFCEEFEDF4E00E
:10D7D20060E070E00E94E5CD80E00E94E3CB2496F9
:10D7E200A2E2B0E00E9453CEEF3181F5203029F45D
:10D7F200EEEAF5E060E070E022C0503029F4E1EC9E
:10D80200F5E060E070E01BC03130A8F0EEEEF4E02D
:10D8120060E070E00E94E5CDE091F208E695E695C1
:10D82200EF71FF27662777270E94E5CD84E00E94EB
:10D83200E3CB28960AC0EAEEF4E060E070E00E94D2
:10D84200E5CD80E00E94E3CB24960AC0E3EDF5E04B
:10D8520060E070E00E94E5CD80E00E94E3CB249678
:10D862000E9463CC2C9608950E945ECC0A2F3C81C4
:10D87200303108F048C0A9E03A9FF001E950F74F73
:10D88200DF01EC91E068EC93A9E03A9FF001E750E8
:10D89200F74FDF01EC91E061EC9330FF1CC036954D
:10D8A200A7E6B9E0EE27A30FBE1F0E9453CE1E2F9C
:10D8B200023019F4E07FE03169F01F70E02FE29549
:10D8C200E07F1E2BA7E6B9E0EE27A30FBE1FE12FD4
:10D8D2000E946FCE18C03695A7E6B9E0EE27A30FD7
:10D8E200BE1F0E9453CE1E2F023019F4EF70E1309A
:10D8F20051F0107F102BA7E6B9E0EE27A30FBE1F51
:10D90200E12F0E946FCE0E9465CC259608951A934E
:10D912000A930A2FE6EEF5E060E070E00E94E5CDA2
:10D92200E02FFF27662777270E94E5CD84E00E943B
:10D93200E3CB2896003108F046C0A9E00A9FF00127
:10D94200E950F74FDF01EC91EF77EC93A9E00A9FE2
:10D95200F001E750F74FDF01EC91E07FEC9300FF1D
:10D9620002C01FE001C010EFA7E6B9E0E02FF0E02F
:10D97200F595E795AE0FBF1F0E9453CEE1230E949B
:10D982006FCEA9E00A9FF001E950F74FE081E17004
:10D9920089F00A9FF001E950F74FE081E077E03427
:10D9A20040F00A9FF001E950F74FDF01EC91EF7868
:10D9B200EC9309C0A9E00A9FF001E950F74FDF019B
:10D9C200EC91EF78EC930991199108950E945CCC47
:10D9D200E091EE08E770E23008F0F6C1A7E2B1E0AC
:10D9E2000E9453CEE03079F0A7E2B1E00E9453CE1C
:10D9F200AE2F0E948A3BA0EFB8E0E1700E2EEC91B0
:10DA0200EE7FE029EC93A8E2B1E00E9453CEE03031
:10DA120081F0A8E2B1E00E9453CEAE2F0E948A3B71
:10DA2200A0EFB8E0E170EE0F0E2EEC91ED7FE02951
:10DA3200EC931FE0103108F0C7C1A9E01A9FF00172
:10DA4200E650F74F2081263309F4BCC1A9E01A9FA2
:10DA5200F001E950F74FE081E295E7705E2F40E078
:10DA6200E091EE08E770E13041F41A9FF001E950CD
:10DA7200F74FE081E1703E2F73C0273B09F4A2C14A
:10DA8200A9E01A9FF001E950F74FE081E27009F432
:10DA920041C0A5E4B1E0E12FF0E0BD01A7E0B0E0B4
:10DAA2000E9411CDDB01AE0FBF1F12960E9453CE12
:10DAB200E07121F0E091F008E17059F5A5E4B1E0E0
:10DAC200E12FF0E0BD01A7E0B0E00E9411CDDB0143
:10DAD200AE0FBF1F12960E9453CEE07221F0E0916A
:10DAE200F008E270B1F4A5E4B1E0E12FF0E0BD018D
:10DAF200A7E0B0E00E9411CDDB01AE0FBF1F12966E
:10DB02000E9453CEE07421F0E091EF08E07809F42E
:10DB120001C001C002C030E016C0A22F0E948A3BA1
:10DB22003E2FA9E01A9FF001E850F74FE081E07123
:10DB320021F0E091910DE17009F405C0303011F04F
:10DB420030E001C031E0A9E01A9FF001E950F74F3F
:10DB5200DF01E32FE1700E2EEC91EE7FE029EC93D2
:10DB6200303069F1E52FF0E0309721F0E130A0E0AC
:10DB7200FA07D9F4E091EF08E770E23098F0E5EFA8
:10DB8200F5E060E070E00E94E5CDE12FF0E0319633
:10DB92006F2F660F660B762F0E94E5CD84E00E9400
:10DBA200E3CB289641E052E009C0E430A0E0FA0756
:10DBB20021F0E530A0E0FA0709F442E029C0503034
:10DBC20011F0513009F424C042E050E0A9E01A9F5C
:10DBD200F001E950F74FDF01EC91EB7FEC93A9E004
:10DBE2001A9FF001E250F74FA0E0B0E0A083B183AA
:10DBF200A9E01A9FF001E550F74FA0E0A083A9E049
:10DC02001A9FF001E750F74FDF01EC91E07FEC93B0
:10DC1200E42FF0E0309709F484C0E130A0E0FA0785
:10DC220009F05CC0A12F0E945361A9E01A9FF00184
:10DC3200E850F74FDF01EC91E068EC93A9E01A9FFE
:10DC4200F001E550F74FA0E0A083A9E01A9FF00190
:10DC5200E750F74FDF01EC91E07FEC93A9E01A9FC8
:10DC6200F001E850F74FE081E074B9F1E12FFF27AE
:10DC720066277727E056FF4F6F4F6BBF06910A9FCB
:10DC8200F001E950F74FDF01EC91E160EC93A9E07C
:10DC92000A9FF001E950F74FDF01EC91EF78E06263
:10DCA200EC93A9E00A9FF001E850F74FDF01EC91F5
:10DCB200E068EC93A9E00A9FF001E550F74FA0E07D
:10DCC200A083A9E00A9FF001E750F74FDF01EC9132
:10DCD200E07FEC93A02F0E94536123C0E230A0E0CA
:10DCE200FA07F9F4A12F0E940361A9E01A9FF0013B
:10DCF200E850F74FE081E074A1F0E12FFF2766279B
:10DD02007727E056FF4F6F4F6BBF06910A9FF001D6
:10DD1200E950F74FDF01EC91EE7FEC93A02F0E94C8
:10DD22000361E091EF08E770E23050F0A9E01A9F3A
:10DD3200F001E950F74FE081E295E7705E1709F4D0
:10DD420032C0E1E0F6E060E070E00E94E5CDE12F54
:10DD5200F0E031966F2F660F660B762F0E94E5CDAD
:10DD6200A9E01A9FF001E950F74FE081E295E770D0
:10DD7200FF27662777270E94E5CDE52FFF27662735
:10DD820077270E94E5CDE32FFF27662777270E949A
:10DD9200E5CDE42FFF27662777270E94E5CD84E1B2
:10DDA2000E94E3CB6896A9E01A9FF001E950F74F71
:10DDB200DF01E52FE770E295E07F0E2EEC91EF7820
:10DDC200E029EC93115036CE0E9463CC269608953A
:10DDD20027970E945ECC8D013B852C85E7E0ED8381
:10DDE200E9EFEE83EF81E160EF83E32FE170EE0F65
:10DDF2000E2EEF81ED7FE029EF83203011F4E7E072
:10DE020001C0E8E0E887E22FEF73EE0FEE0F0E2E6F
:10DE1200EF81E370E029EF8309871A87DE01149608
:10DE22000E94BA92A32F0E94DBBC0E9465CC2D9661
:10DE3200089562970E945CCCE091EE08E770E230B0
:10DE420080F0E091EE08E770E73011F497D802C055
:10DE52000E94DD64E4E1E093F3080E9463CC6896DB
:10DE62000895E0E0F0E0E093F508F093F608E09121
:10DE7200F208E170C9F1E091F208EE7FE093F20856
:10DE8200E1E2F6E060E070E00E94E5CD80E00E9411
:10DE9200E3CB2496E0E0EB8BAB89A03210F5E6E20F
:10DEA200F6E060E070E00E94E5CDEF89FF2766278B
:10DEB20077270E94E5CDA1E4B8E0EB8DF0E0EE0F0C
:10DEC200FF1FAE0FBF1FED91FD91662777270E94BE
:10DED200E5CD88E00E94E3CB2C96EB89EF5FEB8BDC
:10DEE200DBCFAAE00E94F891ABE1B0E00E944FCEF6
:10DEF200ED87FE87A091970DB091980DE091630890
:10DF0200F09164080E94ECCCEA0FFB1FE093970D9E
:10DF1200F093980DE091960DEF70E93038F4A6E990
:10DF2200BDE080E0EFE00E9415CE6BC0E091960D5F
:10DF3200E071D1F1E091960DEF7EE093960DABE1A9
:10DF4200B0E0E091970DF091980D0E9467CEE6E067
:10DF5200E093940DEDE2F6E060E070E00E94E5CD22
:10DF6200E091970DF091980D662777270E94E5CDF5
:10DF720084E00E94E3CB2896E0E0EA93A091970D1B
:10DF8200B091980DA03CE3E3BE0730F0A134EFE37B
:10DF9200BE0710F4E1E001C0E0E0EA93A091970D22
:10DFA200B091980D15DF22C0E091970DF091980D78
:10DFB20066277727E987FA876B877C87A0EEBEE220
:10DFC20080E090E00E9419CDE987FA876B877C8711
:10DFD200ED85FE85A985BA858B859C856627772781
:10DFE2000E946FCDE093990DF0939A0DE091960DFA
:10DFF200E07FE093960DE0E0F0E0E093970DF09380
:10E00200980DE0916308F091640866277727E98705
:10E01200FA876B877C87ACE2B1E080E090E00E94F7
:10E0220019CDE987FA876B877C87ED85FE85F695A2
:10E03200E795A985BA858B859C8566277727EA0FA0
:10E04200FB1F681F791FE987FA876B877C87ED853D
:10E05200FE85A985BA858B859C85662777270E94D0
:10E062006FCDE0939B0DAAE2B1E00E9453CEE13066
:10E0720008F4A1C0E091EF08E07809F443C0A09150
:10E08200990DB0919A0DE4E6F0E00E9457CD0F0190
:10E09200ACE2B1E00E9453CED001F0E0AE17BF0770
:10E0A20068F1ADE2B1E00E9453CEA091F408AE1740
:10E0B20038F4E091F408EF5FE093F408E1501DC0FA
:10E0C200E7E3F6E060E070E00E94E5CDE091990DB3
:10E0D200F0919A0D662777270E94E5CD84E00E9491
:10E0E200E3CB2896A9E00E945C27E091EF08EF7746
:10E0F200E093EF08E0E0E093F40803C0E0E0E0938F
:10E10200F40859C0E0E0EA8BABE2B1E00E9453CEE2
:10E11200EA3058F4AAE2B1E00E9453CEA0919B0DDE
:10E12200AE1710F4E1E0EA8B14C0A091990DB09102
:10E132009A0DE4E6F0E00E9457CD0F01AAE2B1E0A9
:10E142000E9453CED001F0E0AE17BF0710F4E1E019
:10E15200EA8BEA89E03061F1ABE2B1E00E9453CE92
:10E16200A091F408AE1738F4E091F408EF5FE09361
:10E17200F408E1501CC0E7E4F6E060E070E00E94C1
:10E18200E5CDE0919B0DFF27662777270E94E5CD1D
:10E1920084E00E94E3CB2896A8E00E945C27E091ED
:10E1A200EF08E068E093EF08E0E0E093F40803C0D2
:10E1B200E0E0E093F408A0919B0DA83330F5E091E4
:10E1C200F308E030E9F4E8E5F6E060E070E00E9490
:10E1D200E5CDE0919B0DF0E06F2F660F660B762F79
:10E1E2000E94ECCEDF01CB01E0E0F0E060E271E4FE
:10E1F2000E94C3CF0E94E5CD84E00E94E3CB289623
:10E20200EAE0E093F308F19A35C0A091F308A13057
:10E2120088F1E091F308E150E093F308EF5FE091B9
:10E22200F308E03039F5E091EF08E07411F1E09184
:10E23200EF08EF7BE093EF08E0E7F6E060E070E0E4
:10E242000E94E5CDE0919B0DF0E06F2F660F660B0B
:10E25200762F0E94ECCEDF01CB01E0E0F0E060E23D
:10E2620071E40E94C3CF0E94E5CD84E00E94E3CB1B
:10E272002896F198A091F308E0E0EA17E1E008F0AF
:10E28200EE27E88BA0913F08A13008F490C0E091FE
:10E292003F08F0E0E130A0E0FA07C1F5E091710833
:10E2A200F091720866277727A8EEB3E080E090E04D
:10E2B2000E9419CD7F936F93FF93EF93ADE1B0E08E
:10E2C2000E944FCEAF91BF918F919F916627772782
:10E2D2000E946FCDE0937508F0937608A0917508BF
:10E2E200B0917608139718F4E0E0F0E00AC0A0912C
:10E2F2007508B0917608A93FE7E0BE0730F0E8EF75
:10E30200F7E0E0937508F093760851C0E230A0E0A0
:10E31200FA0721F4E3E0E0933F0849C0E330A0E0CC
:10E32200FA0709F044C0E1E0E0933F08E091710888
:10E33200F0917208F695E795ED87FE87ADE1B0E0C2
:10E342000E9467CEE7E8F6E060E070E00E94E5CD6B
:10E35200E989FA89662777270E94E5CD84E00E9441
:10E36200E3CB2896E3E0EA93EE85FF85E53AA7E161
:10E37200FA0740F0AE85BF85A73EECE1BE0710F478
:10E38200E1E001C0E0E0EA93AF85B88921DDE1E098
:10E39200E0933F08E6E0E093940DA0914008A2309C
:10E3A20020F4F49B02C0F59B01C001C0159AA09114
:10E3B2004008A13008F490C0E0914008F0E0E1305C
:10E3C200A0E0FA07C1F5A0914108B0914208882760
:10E3D2009927E8EEF3E060E070E00E9419CD7F93A8
:10E3E2006F93FF93EF93AFE1B0E00E944FCEAF91F6
:10E3F200BF918F919F91662777270E946FCDE093FF
:10E402007708F0937808A0917708B091780813976D
:10E4120018F4E0E0F0E00AC0A0917708B091780823
:10E42200A93FE7E0BE0730F0E8EFF7E0E0937708B6
:10E43200F093780851C0E230A0E0FA0721F4E3E05B
:10E44200E093400849C0E330A0E0FA0709F044C075
:10E45200E1E0E0934008E0914108F0914208F6952E
:10E46200E795ED87FE87AFE1B0E00E9467CEE6E078
:10E47200E093940DE3E9F6E060E070E00E94E5CD00
:10E48200E989FA89662777270E94E5CD84E00E9410
:10E49200E3CB2896E4E0EA93EE85FF85E53AA7E12F
:10E4A200FA0740F0AE85BF85A73EECE1BE0710F447
:10E4B200E1E001C0E0E0EA93AF85B88989DCE1E000
:10E4C200E0934008A0913F08A23020F4F49B02C0E0
:10E4D200F59B01C001C0159AEFE0EB8BAB89A0312F
:10E4E20008F0B4C6EB89A9E0EA9FF001E850F74FC3
:10E4F200E081E07849F0EB89EA9FF001E850F74FBC
:10E50200DF01EC91EF779DC6EB89A9E0EA9FF0016C
:10E51200E650F74FE081E887E0E0EE83EF87A885D9
:10E52200A633D9F4EB89FF2766277727E056FF4FFA
:10E532006F4F6BBFE691A9E0EA9FF001E950F74FF8
:10E54200E081E170E98BEB89FF2766277727E056A8
:10E55200FF4F6F4F6BBFE6910AC0EB89A9E0EA9FBC
:10E56200F001E950F74FE081E170E98BEB89A9E016
:10E57200EA9FF001E950F74FE081E295E770EF83FF
:10E58200E989E03009F4FFC4A1E4B8E0EB89FF2790
:10E5920066277727E054FF4F6F4F6BBFE691F0E09D
:10E5A200EE0FFF1FAE0FBF1FED91FD91F695E795A0
:10E5B200ED87FE87A2E3B0E0EB89F0E0BD01AAE0BF
:10E5C200B0E00E9411CDDB01AE0FBF1F0E944FCE03
:10E5D2008F01AD85BE850A171B0720F0E0E0ED87AD
:10E5E200EE87F1C0A2E3B0E0EB89F0E0BD01AAE062
:10E5F200B0E00E9411CDDB01AE0FBF1F12960E9448
:10E602004FCE9F01AD85BE852A173B0710F1ED85E0
:10E61200FE85E01BF10BED87FE87662777276E2FBD
:10E622007F2FE0E0F0E07F936F93FF93EF93F90188
:10E63200E01BF10B66277727AFE8B2E080E090E0BD
:10E642000E9419CDAF91BF918F919F910E946FCD82
:10E65200B8C0A2E3B0E0EB89F0E0BD01AAE0B0E00F
:10E662000E9411CDDB01AE0FBF1F14960E944FCE48
:10E67200AF01AD85BE854A175B0738F1ED85FE8592
:10E68200E21BF30BED87FE87AD85BE8588279927B0
:10E69200E1E10E94A8CC7F936F93FF93EF93FA017D
:10E6A200E21BF30B66277727AFE8B2E080E090E049
:10E6B2000E9419CDAF91BF918F919F910E946FCD12
:10E6C200ED87FE87EC59FF4F7CC0A2E3B0E0EB89F7
:10E6D200F0E0BD01AAE0B0E00E9411CDDB01AE0F77
:10E6E200BF1F16960E944FCEEE8BFF8BAD85BE8567
:10E6F200EA17FB0740F1ED85FE85E41BF50BED877C
:10E70200FE87AD85BE8588279927E1E10E94A8CCC6
:10E712007F936F93FF93EF93EE89FF89E41BF50BD1
:10E7220066277727A4EBB1E080E090E00E9419CD44
:10E73200AF91BF918F919F910E946FCDED87FE8720
:10E74200E45DFE4F3EC0A2E3B0E0EB89F0E0BD0124
:10E75200AAE0B0E00E9411CDDB01AE0FBF1F1896F8
:10E762000E944FCEEC8BFD8BAE89BF89ED85FE8575
:10E77200EA1BFB0BED87FE87AD85BE8588279927AF
:10E78200E3E10E94A8CC7F936F93FF93EF93AE894E
:10E79200BF89EC89FD89EA1BFB0BF695E795662795
:10E7A2007727ACEEB2E080E090E00E9419CDAF9105
:10E7B200BF918F919F910E946FCDED87FE87E85A9E
:10E7C200FD4FED87FE87A885A73BA1F0A63389F40C
:10E7D200EB89FF2766277727E056FF4F6F4F6BBF06
:10E7E200E691A9E0EA9FF001E650F74FA081A73B2E
:10E7F20009F06EC0A885A73B19F4EB89EA8B0AC021
:10E80200EB89FF2766277727E056FF4F6F4F6BBFD5
:10E8120006900A8AA2E9B9E0EA89FF2766277727E4
:10E82200E052FF4F6F4F6BBFE691F0E00E94D8CCF1
:10E83200AE0FBF1F1196AC91A83C11F4E0E001C0ED
:10E84200E1E0EF87AD85BE85A130E0E4BE0720F0B0
:10E85200E0E0F0E4ED87FE87EB89A9E0EA9FF001B2
:10E86200E450F74FCF0160817181EB89A9E0EA9F03
:10E87200F001E450F74FDF01ED91FD910E94E8CCE9
:10E88200DF01FB01EA1BFB0BDC01ED93FC93EB893F
:10E89200A9E0EA9FF001E450F74F0F01DF01ED918B
:10E8A200FD91DF01ED85FE850E94ECCCEA0FFB1F96
:10E8B200D001ED93FC93EB89A9E0EA9FF001E450CB
:10E8C200F74FDF01ED91FD910E94ECCCED87FE87C1
:10E8D200E091F508F091F608AD85BE85EA0FFB1FC1
:10E8E200E093F508F093F608EB89A9E0EA9FF001BE
:10E8F200E850F74FE081E074B1F0EB89FF2766271B
:10E902007727E056FF4F6F4F6BBFE691EA9FF0010A
:10E91200E250F74FDF01ED91FD91AD85BE85EA0F23
:10E92200FB1FED87FE87AD85BE85A73FE7E2BE07E9
:10E9320020F0E6EFF7E2ED87FE87EB89A9E0EA9F98
:10E94200F001E250F74FAD85BE85A083B183E0911F
:10E95200EF08E870C9F0EFE9F6E060E070E00E94CD
:10E96200E5CDEF89F0E031966F2F660F660B762FBB
:10E972000E94E5CDED89FE89662777270E94E5CDC5
:10E9820088E00E94E3CB2C96EF81F0E0E230A0E039
:10E99200FA0709F0ADC0EB89A9E0EA9FF001E75060
:10E9A200F74FDF01EC91EF7EEC93A889A03039F5A7
:10E9B200A7ECB8E0EB89FF2766277727E054FF4FE3
:10E9C2006F4F6BBFE691F0E0AE0FBF1FAC91A2306C
:10E9D200A8F4AF85A03089F4A9E7B8E0EB89FF2756
:10E9E20066277727E055FF4F6F4F6BBFE691F0E048
:10E9F200AE0FBF1FEC91E07409F401C001C04FC01B
:10EA0200EB89A9E0EA9FF001E750F74FE081EF7050
:10EA1200E43058F4EB89EA9FF001E750F74FDF0149
:10EA220080E0EFE00E9415CE3AC0E5E0EF83E2E03D
:10EA3200EE83EB89EA93A3E00E94356CEB89A9E0AF
:10EA4200EA9FF001E850F74FE081EF70EA3098F466
:10EA5200EB89EA9FF001E850F74FDF0180E0EFE039
:10EA62000E9415CEE6E6EA93EC89E15FEA93A0E024
:10EA7200B0E00E946527EBEAF6E060E070E00E94F9
:10EA8200E5CDEF89F0E031966F2F660F660B762F9A
:10EA92000E94E5CD84E00E94E3CB289673C2EB8905
:10EAA200A9E0EA9FF001E550F74FA081A53058F4A4
:10EAB200EB89A9E0EA9FF001E550F74FDF01EC9105
:10EAC200EF5FEC9314C0EB89A9E0EA9FF001E550F7
:10EAD200F74FA0E0A083EB89A9E0EA9FF001E7509D
:10EAE200F74FDF01EC91E07FEC93E3E0EF834AC262
:10EAF200E330A0E0FA0709F045C2A889A03039F551
:10EB0200A7ECB8E0EB89FF2766277727E054FF4F91
:10EB12006F4F6BBFE691F0E0AE0FBF1FAC91A2301A
:10EB2200A8F4AF85A03089F4A9E7B8E0EB89FF2704
:10EB320066277727E055FF4F6F4F6BBFE691F0E0F6
:10EB4200AE0FBF1FEC91E07409F401C001C050C0C8
:10EB5200EB89A9E0EA9FF001E750F74FE081EF70FF
:10EB6200E33058F4EB89EA9FF001E750F74FDF01F9
:10EB720080E0EFE00E9415CE3AC0E5E0EF83E2E0EC
:10EB8200EE83EB89EA93A3E00E94356CEB89A9E05E
:10EB9200EA9FF001E850F74FE081EF70EA3098F415
:10EBA200EB89EA9FF001E850F74FDF0180E0EFE0E8
:10EBB2000E9415CEE6E6EA93EC89E15FEA93A0E0D3
:10EBC200B0E00E946527EAEBF6E060E070E00E94A8
:10EBD200E5CDEF89F0E031966F2F660F660B762F49
:10EBE2000E94E5CD84E00E94E3CB2896CBC114C0FD
:10EBF200EB89A9E0EA9FF001E750F74FE081EF705F
:10EC0200E13050F0EB89EA9FF001E750F74FDF0166
:10EC120080E0EFE00E9419CEA885A63309F4B2C1C4
:10EC2200A5E4B1E0EB89F0E0BD01A7E0B0E00E940D
:10EC320011CDDB01AE0FBF1F14960E944FCEFF71A4
:10EC4200ED87FE87EB89A9E0EA9FF001E650F74FD6
:10EC5200A081A73B79F4E091EE08E770E13049F436
:10EC6200EB89A9E0EA9FF001E950F74FE081E170FA
:10EC720009F401C035C0A2E9B9E0EB89FF27662794
:10EC82007727E052FF4F6F4F6BBFE691F0E00E9493
:10EC9200D8CCAE0FBF1F1196EC91EA8BE03029F46D
:10ECA200ED85FE850E94EACC19C0EA89EC5EEA8B0A
:10ECB200AA89A83CA8F4AD85BE8588279927F0E0EB
:10ECC2006F2F660F660B762F0E9419CDDF01CB01E5
:10ECD200E8ECF0E060E070E00E946FCDED87FE8727
:10ECE200EB89A9E0EA9FF001E250F74FDF01ED91D5
:10ECF200FD91DF01ED85FE85AE17BF0708F48CC0DC
:10ED0200EB89A9E0EA9FF001E950F74FDF01EC91AE
:10ED1200EB7FEC93EB89A9E0EA9FF001E950F74F12
:10ED2200E081E87091F4EB89EA9FF001E950F74F36
:10ED3200DF01EC91E860EC93EB89A9E0EA9FF00136
:10ED4200E550F74FA0E0A08366C0EB89A9E0EA9FF7
:10ED5200F001E550F74FDF01EC91EF5FEC93EB89A7
:10ED6200A9E0EA9FF001E550F74FE081EF93A5E4B7
:10ED7200B1E0EB89F0E0BD01A7E0B0E00E9411CD67
:10ED8200DB01AE0FBF1F16960E9453CEAF91AE1796
:10ED920008F441C0E4E0EF83E2E0EE83EB89EA931A
:10EDA200A4E00E94356CEB89A9E0EA9FF001E850EB
:10EDB200F74FE081EF70EA30D8F4EB89EA9FF00177
:10EDC200E850F74FDF0180E0EFE00E9415CEE7E662
:10EDD200EA93EC89E15FEA93ED89A9E0EA9FF00109
:10EDE200E250F74FDF01ED91FD91DF010E946527AF
:10EDF200E9ECF6E060E070E00E94E5CDEF89F0E03A
:10EE020031966F2F660F660B762F0E94E5CD84E058
:10EE12000E94E3CB2896B6C0EB89A9E0EA9FF001F5
:10EE2200E950F74FE081E87089F0EB89EA9FF00141
:10EE3200E950F74FDF01EC91E77FEC93EB89A9E012
:10EE4200EA9FF001E550F74FA0E0A083A5E4B1E00E
:10EE5200EB89F0E0BD01A7E0B0E00E9411CDDB013B
:10EE6200AE0FBF1F11960E944FCEFF70ED87FE8737
:10EE7200AD85BE8500240A160B0608F083C0EB8917
:10EE8200A9E0EA9FF001E250F74FDF01ED91FD9119
:10EE9200AD85BE85EA17FB0708F062C0EB89A9E0E1
:10EEA200EA9FF001E550F74FE081EF93A5E4B1E06E
:10EEB200EB89F0E0BD01A7E0B0E00E9411CDDB01DB
:10EEC200AE0FBF1F13960E9453CEAF91AE1758F4E8
:10EED200EB89A9E0EA9FF001E550F74FDF01EC91E1
:10EEE200EF5FEC933CC0EB89A9E0EA9FF001E950A7
:10EEF200F74FE081E47099F5EB89EA9FF001E95060
:10EF0200F74FDF01EC91E460EC93EB89EA93A2E026
:10EF12000E94356CEB89A9E0EA9FF001E850F74FB7
:10EF2200E081EF70EA30D8F4EB89EA9FF001E85013
:10EF3200F74FDF0180E0EFE00E9415CEE5E6EA93AD
:10EF4200EC89E15FEA93ED89A9E0EA9FF001E250E2
:10EF5200F74FDF01ED91FD91DF010E94652712C09D
:10EF6200EB89A9E0EA9FF001E550F74FA0E0A0830A
:10EF7200EB89A9E0EA9FF001E950F74FDF01EC913C
:10EF8200EB7FEC93D0C0EB89A9E0EA9FF001E2505D
:10EF9200F74FA0E0B0E0A083B183EB89A9E0EA9F3C
:10EFA200F001E450F74FA0E0B0E0A083B183A88560
:10EFB200A63389F0A5E4B1E0EB89F0E0BD01A7E05A
:10EFC200B0E00E9411CDDB01AE0FBF1F12960E946E
:10EFD20053CEE07809F4A7C0EF81F0E0309709F052
:10EFE2006CC0E889E03009F09EC0A3E9B8E0EB8983
:10EFF200FF2766277727E055FF4F6F4F6BBFE691DC
:10F00200F0E0AE0FBF1FEC91E07459F4EB89A9E078
:10F01200EA9FF001E750F74FDF01EC91E07FEC93BC
:10F022004BC0EB89A9E0EA9FF001E750F74FE0817E
:10F03200EF70EF3058F4EB89EA9FF001E750F74F99
:10F04200DF0180E0EFE00E9415CE36C0E1E0EF8301
:10F05200EB89A9E0EA9FF001E750F74FDF01EC915D
:10F06200E07FEC93EB89EA93A1E00E94356CEB8997
:10F07200A9E0EA9FF001E850F74FE081EF70EA3033
:10F08200D8F4EB89EA9FF001E850F74FDF0180E006
:10F09200EFE00E9415CEE4E6EA93EC89E15FEA93A1
:10F0A200ED89A9E0EA9FF001E250F74FDF01ED910F
:10F0B200FD91DF010E94652736C0E130A0E0FA072A
:10F0C20091F5A3E9B8E0EB89FF2766277727E0559A
:10F0D200FF4F6F4F6BBFE691F0E0AE0FBF1FEC9199
:10F0E200E07409F5EB89A9E0EA9FF001E750F74FD8
:10F0F200E081EF70EF3058F4EB89EA9FF001E750BE
:10F10200F74FDF0180E0EFE00E9415CE0CC0E0E097
:10F11200EF83EB89A9E0EA9FF001E750F74FDF01A7
:10F12200EC91E07FEC93AE81A230B1F5AB890E9405
:10F132000361EB89A9E0EA9FF001E850F74FE08113
:10F14200E07419F4A885A63339F5EB89FF27662701
:10F152007727E056FF4F6F4F6BBF06900A8AEA8906
:10F16200A9E0EA9FF001E950F74FDF01EC91EE7F51
:10F17200EC93EA89A9E0EA9FF001E950F74FDF0139
:10F18200EF81E770E295E07F0E2EEC91EF78E029B7
:10F19200EC93AA890E940361E091EF08E770E230E4
:10F1A20068F0EB89A9E0EA9FF001E950F74FE081AE
:10F1B200E295E770AE2FEF81EA1709F433C0E8ED6C
:10F1C200F6E060E070E00E94E5CDEF89F0E0319674
:10F1D2006F2F660F660B762F0E94E5CDEB8DA9E0AF
:10F1E200EA9FF001E950F74FE081E295E770FF27CF
:10F1F200662777270E94E5CDEB89FF2766277727C9
:10F202000E94E5CDE9A1FF27662777270E94E5CD79
:10F21200EA8DFF27662777270E94E5CD84E10E94C9
:10F22200E3CB6896EB89A9E0EA9FF001E950F74F3A
:10F23200DF01EF81E770E295E07F0E2EEC91EF782F
:10F24200E029EC93EB89E150EB8B48C9E091EF08A0
:10F25200E87009F475C0E9EFF6E060E070E00E9442
:10F26200E5CD80E00E94E3CB2496E0E0EB8BAB8916
:10F27200A03108F060C0EB89A9E0EA9FF001E950F3
:10F28200F74FE081E17009F452C0E3E0F7E060E09B
:10F2920070E00E94E5CDEF89F0E031966F2F660FA6
:10F2A200660B762F0E94E5CDA3E9B8E0EB8DFF2730
:10F2B20066277727E055FF4F6F4F6BBFE691F0E06F
:10F2C200AE0FBF1FEC91E07411F0E1E001C0E0E08D
:10F2D2000E94F1CC0E94E5CDA1E4B8E0EF8DFF27BA
:10F2E20066277727E054FF4F6F4F6BBFE691F0E040
:10F2F200EE0FFF1FAE0FBF1FED91FD91662777271F
:10F302000E94E5CDEBA1A9E0EA9FF001E250F74FA0
:10F31200DF01ED91FD91AAE0B0E00E9411CD6627D8
:10F3220077270E94E5CD80E10E94E3CB6496EB89CA
:10F33200EF5FEB8B9CCFE091EF08E77FE093EF0864
:10F342000E9463CC689608950E945CCCE0E05E2F38
:10F352002E2F3E2F0E2F10E01C3040F5A7E6B9E00D
:10F36200EE27A10FBE1F0E9453CEE03009F021E02C
:10F37200A9E01A9FF001E950F74FE081F0E00E9406
:10F38200E8CCE770F070E130A0E0FA0711F451E048
:10F392000BC0E430A0E0FA0711F431E005C0E5301B
:10F3A200A0E0FA0709F401E01F5FD6CF10E01830A1
:10F3B20040F5A3E7B9E0EE27A10FBE1F0E9453CE8E
:10F3C200E03009F021E0A9E01A9FF001E950F74F7F
:10F3D200E081F0E00E94E8CCE770F070E130A0E05C
:10F3E200FA0711F451E00BC0E430A0E0FA0711F47F
:10F3F20031E005C0E530A0E0FA0709F401E01F5F43
:10F40200D6CFA0EFB8E0E02FE170EE0FEE0F0E2E98
:10F41200EC91EB7FE029EC93A0EFB8E0E32FE170F1
:10F42200EE0FEE0FEE0F0E2EEC91E77FE029EC933C
:10F43200A0EFB8E0E22FE170E295E07FEE0F0E2E32
:10F44200EC91EF7DE029EC93A0EFB8E0E52FE170BD
:10F45200E295E07F0E2EEC91EF7EE029EC930E9484
:10F4620063CC269608951A93EDE1F7E060E070E030
:10F472000E94E5CD80E00E94E3CB2496ABE7B9E0A1
:10F48200E0E0F0E00E9467CE10E0103108F047C0E3
:10F49200A9E01A9FF001E850F74FDF01EC91E07FFD
:10F4A200EC93A9E01A9FF001E950F74FDF01EC91CC
:10F4B200EF77EC93A9E01A9FF001E750F74FDF01D5
:10F4C200EC91EF7EEC93A9E01A9FF001E750F74F21
:10F4D200DF01EC91E07FEC93A9E01A9FF001E95083
:10F4E200F74FE081F0E00E94E8CCE770F070E13085
:10F4F200A0E0FA0721F0E430A0E0FA0709F404C022
:10F50200E530A0E0FA0749F4A9E01A9FF001E950BA
:10F51200F74FDF01EC91EF78EC931F5FB6CF10E06D
:10F522001C3048F4A7E6B9E0EE27A10FBE1F0E94E7
:10F532006FCE1F5FF5CF199108950E945ECC3A2FCE
:10F54200373310F03C3308F064C000E010E01031B3
:10F5520008F05DC0A9E01A9FF001E650F74FA081C4
:10F562003A1709F052C0A9E01A9FF001E950F74F8B
:10F57200E081F0E00E94E8CCE770F070309761F42F
:10F582001A9FF001E950F74FE081E07811F0003066
:10F5920009F001C005E039C0E230A0E0FA0721F02D
:10F5A200E330A0E0FA07B9F4A9E01A9FF001E950AC
:10F5B200F74FE081E47011F002E00CC0A9E01A9F5D
:10F5C200F001E950F74FE081E07811F0003009F0E6
:10F5D20001C005E01AC0E130A0E0FA0751F4A9E049
:10F5E2001A9FF001E950F74FE081E07809F001E05D
:10F5F2000CC0E430A0E0FA0711F4E4E086C1E53083
:10F60200A0E0FA0711F4E3E080C11F5FA0CFE02F72
:10F612007CC1E32FEF501E2F103108F046C0A9E045
:10F622001A9FF001E950F74FE081F0E00E94E8CC28
:10F63200E770F070309751F41A9FF001E950F74FDC
:10F64200E081E07811F0E5E060C15EC1E230A0E067
:10F65200FA0721F0E330A0E0FA07A9F4A9E01A9F23
:10F66200F001E950F74FE081E47011F0E2E04DC1A2
:10F67200A9E01A9FF001E950F74FE081E07811F01C
:10F68200E5E043C141C1E130A0E0FA0711F4E1E055
:10F692003CC1E430A0E0FA0711F4E4E036C1E53001
:10F6A200A0E0FA0711F4E3E030C12EC167971A9384
:10F6B200FE013896FA93EA93E0E0EA93A0E1B0E023
:10F6C2000E945BC5FE013196FA93EA93E0E0EA9369
:10F6D200A7E0B0E00E945BC5EAE0EC83EF8310E0B4
:10F6E200103108F058C0E12FFF2766277727E05333
:10F6F200FF4F6F4F6BBFE691E03039F4ED81FE8131
:10F70200E070F07EE062F36006C0ED81FE81E070A1
:10F71200F07EE46FF160ED83FE83A5E4B1E0E12FBA
:10F72200F0E0BD01A7E0B0E00E9411CDE60FF71FA7
:10F73200FA93EA93FE013396FA93EA93A7E00E94C2
:10F742001426FE013896FA93EA93E9E2F7E060E0C4
:10F7520070E00E94E5CDE12FF0E031966F2F660F49
:10F76200660B762F0E94E5CD84E00E94A8CB2A96F4
:10F77200E12FF0E0A0E1B8E30E94D6CCEA0FFB1F34
:10F78200FA93EA93FE013A96FA93EA930E94C42806
:10F79200A8951F5FA5CF0E947A6218810C94CB8036
:10F7A2001A930A9310E0103108F06DC0E12FF0E0D7
:10F7B200309719F4E5B1E07222C0E130A0E0FA0717
:10F7C20019F4E2B1E1701BC0E230A0E0FA0719F4CB
:10F7D200E5B1E07414C0E330A0E0FA0719F4E4B331
:10F7E200E2700DC0E430A0E0FA0719F4EEB1E8705F
:10F7F20006C0E530A0E0FA0719F4E4B3E4700E2F76
:10F80200E3E3F7E060E070E00E94E5CDE12FF0E095
:10F8120031966F2F660F660B762F0E94E5CDA9E019
:10F822001A9FF001E950F74FE081E295E770FF2758
:10F83200662777270E94E5CD1A9FF001E950F74F1E
:10F84200E081E170FF27662777270E94E5CD01302E
:10F8520010F0E1E301C0E0E3FF27662777270E946B
:10F86200E5CDA9E01A9FF001E250F74FDF01ED91DB
:10F87200FD91662777270E94E5CD84E10E94E3CBC4
:10F8820068961F5F90CF0991199108951A9310E01D
:10F89200153080F4E12FF0E0E957F64F0F01A5EBA8
:10F8A200B1E0EE27A10FBE1F0E9453CED001EC9310
:10F8B2001F5FEECF0C9415830E945ECC3A2F10E0AE
:10F8C200103110F5A9E01A9FF001E650F74FA08120
:10F8D2003A17C1F4A9E01A9FF001E950F74FE0810D
:10F8E200E295E7700E2F1A9FF001E950F74FE08181
:10F8F200E47031F4013021F0043011F0053011F4DC
:10F90200E1E003C01F5FDCCFE0E00E9465CC2496FB
:10F91200089560971A93FE013196FA93EA93E0E014
:10F92200EA93A2E0B0E00E945BC510E0153080F5DA
:10F93200A5EBB1E0EE27A10FBE1F0E946FCEFE0124
:10F942003196FA93EA93E4E5F7E060E070E00E9412
:10F95200E5CDE12FF0E031966F2F660F660B762F23
:10F962000E94E5CD84E00E94A8CB2A96E12FF0E028
:10F97200A0E1B9E30E94D6CCEA0FFB1FFA93EA9307
:10F98200FE013396FA93EA930E94C4281F5FCECFFA
:10F9920018816196089562970E945CCCA6E2B1E05C
:10F9A2000E9453CEE07109F4F3C3A5E2B1E00E94D4
:10F9B20053CE0E2FA6E2B1E00E9453CEEF70ED8B34
:10F9C20000FF04C0E0919307E170F1F401FF04C06D
:10F9D200E0919407E170C1F402FF04C0E091950741
:10F9E200E17091F403FF04C0E0919607E17061F4C5
:10F9F200AD89A53040F0ED89F0E03197ED56F84F32
:10FA0200E081E17009F412C0A2E3B1E00E944FCE9E
:10FA1200FF70A4E8BDE0FF700F01ED91FD91E07071
:10FA2200F07FE029F129FE93EE93B2C3A1E3B1E0A6
:10FA32000E9453CEEE83E030C1F0AE810E948A3B39
:10FA4200E03091F0A2E3B1E00E944FCEFF70A4E853
:10FA5200BDE0FF700F01ED91FD91E070F07FE029B4
:10FA6200F129FE93EE9394C31BC0E091CF03E270A1
:10FA720021F0A091CE03A13008F412C0A2E3B1E0BC
:10FA82000E944FCEFF70A4E8BDE0FF700F01ED9120
:10FA9200FD91E070F07FE029F129FE93EE9378C3A7
:10FAA200E091840DF091850DFF7000240E160F0673
:10FAB20040F4A4E8BDE080E0EFEFFFE00E9443CE17
:10FAC20067C3A6E2B1E00E9453CEE295EF70E695DD
:10FAD200E170EB8BE03021F0A091CD0AA13008F467
:10FAE20001C056C3E0E0E093900D0E94E76C0E94D3
:10FAF200E835A6E00E945C27A1E00E9494BAE4E601
:10FB0200F7E060E070E00E94E5CD80E00E94E3CB88
:10FB1200249616981598E0E0E093E508E460E093F7
:10FB2200E508E064E093E5082898EDB5E093820DDE
:10FB3200E0E4EEBDEDB5E7FFFDCFEAE0EEBDEDB5E9
:10FB4200E7FFFDCFE091E508EEBDEDB5E7FFFDCFA4
:10FB5200289A07FF3FC0E2B1E67EE2B9E5B1EF7055
:10FB6200E5B95F98EEB1E77CEEB9E1B3EF7CE1BBBA
:10FB7200E4B3E87FE4BBE0E0E093E708E093E90860
:10FB82002898EDB5E093820DE2E4EEBDEDB5E7FF16
:10FB9200FDCFEAE0EEBDEDB5E7FFFDCFE091E7086E
:10FBA200EEBDEDB5E7FFFDCF289A2898EDB5E093BD
:10FBB200820DE4E4EEBDEDB5E7FFFDCFEAE0EEBD78
:10FBC200EDB5E7FFFDCFE091E908EEBDEDB5E7FF4A
:10FBD200FDCF289AE0E0E98BEA8B00FF0FC0E091AD
:10FBE2009307EC7021F452E0E1E0EA8B06C0E09169
:10FBF2009307EC70E43009F451E001C050E001FFDA
:10FC02000FC0E0919407EC7021F442E0E1E0EA8B4E
:10FC120006C0E0919407EC70E43009F441E001C0C1
:10FC220040E002FF11C0E0919507EC7029F4E2E098
:10FC3200EF8BE1E0E98B07C0E0919507EC70E430CF
:10FC420011F4E1E0EF8B02C0E0E0EF8B03FF11C0A3
:10FC5200E0919607EC7029F4E2E0EE8BE1E0E98BAB
:10FC620007C0E0919607EC70E43011F4E1E0EE8B0E
:10FC720002C0E0E0EE8BE0E0EC8BAD89A530E8F06D
:10FC8200ED89E1501E2FFF2766277727EC56FF4F9D
:10FC92006F4F6BBFE691E150E8B9E12FF0E0ED560E
:10FCA200F84FE081EC70E43029F4ED89EC8BE0E070
:10FCB200ED8B02C0E1E0EA8B02C0EFE3E8B9E0E0DD
:10FCC200EF87EE87ED87EC87EB8739E120E0E09361
:10FCD200B80DEF83EA87A6E2B1E00E9453CEE29527
:10FCE200EF70E695E695E170E88BA4E3B1E00E943F
:10FCF20053CEE887E987E0E0E093D800ECBDA4E1C9
:10FD0200B0E00E9427D0E0E0E093C100E093C2009F
:10FD12000E943838E1E0E0936900E0E0E4BD0E942F
:10FD2200CA82E0E0E0938000E0938500E0938400E3
:10FD3200E8E1E0938900E9E6E0938800E2E0E6BBCF
:10FD4200E0936F00E0E0E0937A00F894E0E8E0935B
:10FD52006100E6E0E09361007894EAE0E0938100DC
:10FD6200E1E8ECBBE1E0E3BF8895A895E091B80D2E
:10FD7200AF81EA0FEF83E0E0E093B80DAF81A530E9
:10FD820088F0EF81E550EF83A4EFB0E1ED91FD91B2
:10FD92006D917D91EF5FFF4F6F4F7F4F7E936E931B
:10FDA200FE93EE93E0E0EA87513089F4669B03C04C
:10FDB200E0E0EF870CC0E889E03039F4AF85A2308B
:10FDC20020F4EF85EF5FEF8702C0E1E0EA87413080
:10FDD20089F4679B03C0E0E0EE870CC0E889E0305D
:10FDE20039F4AE85A23020F4EE85EF5FEE8702C0D3
:10FDF200E2E0EA87AF89A13089F4799B0DC0E889F6
:10FE0200E03039F4AD85A23020F4ED85EF5FED8767
:10FE120002C0E3E0EA8702C0E0E0ED87AE89A130EC
:10FE220089F47A9B0DC0E889E03039F4AC85A230C0
:10FE320020F4EC85EF5FEC8702C0E4E0EA8702C0C1
:10FE4200E0E0EC87EC89E03089F0359B03C0E0E02C
:10FE5200EB870CC0E889E03039F4AB85A23020F49E
:10FE6200EB85EF5FEB8702C0E5E0EA87EA89E030E5
:10FE720019F4E989E030D1F0E0E5ECBDE1E0EDBD57
:10FE8200EA89E03009F0169AE989E03009F0159A1A
:10FE9200AD89A03019F4AC89A03029F088E592E050
:10FEA2000197F1F703C085E88A95F1F7523089F49A
:10FEB200669B0DC0E889E03039F4AF85A23020F4AA
:10FEC200EF85EF5FEF8702C0E1E0EA8702C0E0E082
:10FED200EF87423089F4679B0DC0E889E03039F43E
:10FEE200AE85A23020F4EE85EF5FEE8702C0E2E03D
:10FEF200EA8702C0E0E0EE87AF89A23089F4799BFD
:10FF020003C0E0E0ED870CC0E889E03039F4AD854C
:10FF1200A23020F4ED85EF5FED8702C0E3E0EA87CF
:10FF2200AE89A23089F47A9B03C0E0E0EC870CC072
:10FF3200E889E03039F4AC85A23020F4EC85EF5F3B
:10FF4200EC8702C0E4E0EA87AD89A13088F0359BF6
:10FF52000DC0E889E03039F4AB85A23020F4EB859E
:10FF6200EF5FEB8702C0E5E0EA8702C0E0E0EB87E3
:10FF7200EA89E03009F01698E989E03009F015982D
:10FF8200313018F131502030F9F020E0E091E508ED
:10FF9200ED7FE093E508E0E5ECBDE1E0EDBD2898FA
:10FFA200EDB5E093820DE0E4EEBDEDB5E7FFFDCFE8
:10FFB200EAE0EEBDEDB5E7FFFDCFE091E508EEBD6D
:10FFC200EDB5E7FFFDCF289A20C031E321E0E091B3
:10FFD200E508E260E093E508E0E5ECBDE1E0EDBDB7
:10FFE2002898EDB5E093820DE0E4EEBDEDB5E7FFB4
:0EFFF200FDCFEAE0EEBDEDB5E7FFFDCFE091FB
:020000021000EC
:02000000E50811
:10000200EEBDEDB5E7FFFDCF289AE0E0ECBDE09153
:10001200CF03E27029F0E09902C0489901C001C003
:1000220002C0E6E0EA87609902C0E7E0EA87EA8573
:10003200E03049F0A985A13020F0E985E150E98757
:1000420001C004C002C0E885E9878CCEF894E0E8DC
:10005200E0936100E0E0E09361007894EDBBE0930F
:100062008100E0936F00E1E5ECBDE1E0EDBD719A46
:10007200E6E0E093C200E8E9E093C100E0E0E0934B
:10008200C500E3E0E093C400EDE0E4BDE0E0E0930E
:10009200900DACE6B2E00E944FCEDF010E94CC048C
:1000A200A0E00E943D370E94B63A07FF02C00E94BC
:1000B2007A627ED0A2E3B1E00E944FCEFF70A4E844
:1000C200BDE0FF700F01ED91FD91E070F07FE0293E
:1000D200F129FE93EE93AA85A73099F4E091840D5D
:1000E200F091850DFF703A9758F4E091840DF091EC
:1000F200850DE070F07FEA60E093840DF093850D4A
:1001020012C0E091840DF091850DFF70359758F47F
:10011200E091840DF091850DE070F07FE560E09351
:10012200840DF093850DE0E0E093880DEFE6F7E0B3
:1001320060E070E00E94E5CDEE85FF276627772715
:100142000E94E5CD84E00E94E3CB2896A0E00E94C5
:1001520094BAA7E00E945C270E94EF35E889E0305C
:1001620029F0AA85A13010F0A53008F011C0EA8567
:10017200E150EA87AA85B0E0AD56B84FEC91E16054
:10018200EC93AA85B0E0AD56B84FEC91E06FEC93DA
:100192000E9463CC68960895EA93EFB7EA93E091E0
:1001A200B80DEF5FE093B80DE991EFBFE9911895B3
:1001B20022970E945CCC20E050E030E0EAD1ECE8EB
:1001C200F9E0FA93EA93E0E0EA93AEE3B0E00E944A
:1001D2005BC510E0173008F0F7C0E12FFF27662754
:1001E2007727E253FE4F6F4F6BBF4691A5E4B1E014
:1001F200E42FF0E0BD01A7E0B0E00E9411CDDB01E9
:10020200AE0FBF1F0E9453CEE73B09F0DBC0A2E94D
:10021200B9E0E12FF0E00E94D8CCAE0FBF1FEC9105
:10022200E160EC93113028F0143010F421E001C0A9
:1002320051E0ABE3B7E0E12FF0E0BD01A2E2B0E0B4
:100242000E9411CDDB01AE0FBF1F0E9453CEE030E2
:1002520059F0A2E9B9E0E12FF0E00E94D8CCAE0F4C
:10026200BF1FEC91E260EC93ABE3B7E0E12FF0E06B
:10027200BD01A2E2B0E00E9411CDDB01AE0FBF1FB3
:1002820011960E9453CEE03059F0A2E9B9E0E12F75
:10029200F0E00E94D8CCAE0FBF1FEC91E460EC936B
:1002A200ABE3B7E0E12FF0E0BD01A2E2B0E00E94D3
:1002B20011CDDB01AE0FBF1F12960E9453CEE0306C
:1002C20059F0A2E9B9E0E12FF0E00E94D8CCAE0FDC
:1002D200BF1FEC91E860EC93ABE3B7E0E12FF0E0F5
:1002E200BD01A2E2B0E00E9411CDDB01AE0FBF1F43
:1002F20013960E9453CEE03059F0A2E9B9E0E12F03
:10030200F0E00E94D8CCAE0FBF1FEC91E061EC93FD
:10031200ABE3B7E0E12FF0E0BD01A2E2B0E00E9462
:1003220011CDDB01AE0FBF1F14960E9453CEE030F9
:1003320059F0A2E9B9E0E12FF0E00E94D8CCAE0F6B
:10034200BF1FEC91E062EC93ABE3B7E0E12FF0E08A
:10035200BD01A2E2B0E00E9411CDDB01AE0FBF1FD2
:1003620018960E944BCE30976040704061F031E0A9
:10037200A2E9B9E0E12FF0E00E94D8CCAE0FBF1F96
:10038200EC91E064EC93ABE3B7E0E12FF0E0BD0168
:10039200A2E2B0E00E9411CDDB01AE0FBF1F539667
:1003A2000E944BCE30976040704061F031E0A2E98C
:1003B200B9E0E12FF0E00E94D8CCAE0FBF1FEC9164
:1003C200E068EC931F5F06CFE32FE170EE0F0E2E75
:1003D200E0918C09ED7FE029E0938C09E09192098C
:1003E200E17021F4203011F4503029F0E0918C09B1
:1003F200E160E0938C09E0919209E170A1F1A6E33A
:10040200B7E00E9453CEF0E0309711F4E7E629C03E
:10041200E130A0E0FA0711F4EFE623C0E230A0E0F9
:10042200FA0711F4E6E61DC0E330A0E0FA0711F482
:10043200E5E617C0E430A0E0FA0711F4E4E611C0E3
:10044200E530A0E0FA0711F4E3E60BC0E630A0E0E5
:10045200FA0711F4EBE605C0E730A0E0FA0719F459
:10046200E2E6E0938D09203009F446C0A7E3B7E045
:100472000E944FCEEE83FF83AE81BF81AA3FE0E0B0
:10048200BE0760F001E0EE81FF8166277727A0E0DA
:10049200B4E284EF90E00E946FCD1BC0AE81BF81B9
:1004A200939760F002E0EE81FF8166277727A0E84C
:1004B200B4E88EE190E00E946FCD0BC003E0EE81C4
:1004C200FF8166277727A0E9B0ED83E090E00E94E4
:1004D20093CDEE83FF83E0938E09F0938F09EF8132
:1004E200E0938700EE81E0938600E2E0E0938000F3
:1004F200E02FE85EE0938100503009F446C0A9E3A2
:10050200B7E00E944FCEEE83FF83AE81BF81AA3F48
:10051200E0E0BE0760F001E0EE81FF816627772709
:10052200A0E0B4E284EF90E00E946FCD1BC0AE81E8
:10053200BF81939760F002E0EE81FF816627772703
:10054200A0E8B4E88EE190E00E946FCD0BC003E01A
:10055200EE81FF8166277727A0E9B0ED83E090E086
:100562000E9493CDEE83FF83E0939009F09391096B
:10057200EF81E0939700EE81E0939600E2E0E09352
:100582009000E02FE85EE09391000E9463CC2896F1
:1005920008951A93E0E0E093B000E0918000E370E8
:1005A200E0938000E0919000E370E093900010E00F
:1005B2001730C0F4A2E9B9E0E12FF0E00E94D8CCF4
:1005C200AE0FBF1F1196E0E0EC93A2E9B9E0E12F74
:1005D200F0E00E94D8CCAE0FBF1FEC91ED7FEC9300
:1005E2001F5FE6CF10E01031F8F4A9E01A9FF00186
:1005F200E650F74FA081A73BA9F4A9E01A9FF001AA
:10060200E950F74FDF01EC91EE7FEC93A9E01A9FDE
:10061200F001E950F74FDF01EC91EF78EC93A12F55
:100622000E9403611F5FDFCF199108951A930A9305
:100632000A2FE02FFF2766277727E052FF4F6F4FE1
:100642006BBF1691183308F0CCC0A2E9B9E0E12FD4
:10065200F0E00E94D8CCAE0FBF1F1196E0E0EC9301
:10066200E12FF0E03097B1F4E0E0E093B000E091E8
:100672009209E47069F0ACE3B7E00E9453CEAE2F6A
:100682000E948A3BE03011F02C9A01C02C9801C0E4
:100692002C98A7C0E130A0E0FA07C1F4E0918000F5
:1006A200EF73E0938000E0919A09E47069F0AEE59F
:1006B200B7E00E9453CEAE2F0E948A3BE03011F089
:1006C2002D9A01C02D9801C02D988BC0E230A0E078
:1006D200FA07C1F4E0918000EF7CE0938000E091A2
:1006E200A209E47069F0A0E8B7E00E9453CEAE2FF1
:1006F2000E948A3BE03011F02E9A01C02E9801C070
:100702002E986FC0E330A0E0FA07C1F4E0918000B8
:10071200E37FE0938000E091AA09E47069F0A2EA25
:10072200B7E00E9453CEAE2F0E948A3BE03011F018
:100732002F9A01C02F9801C02F9853C0E430A0E037
:10074200FA07C1F4E0919000EF73E0939000E0911A
:10075200B209E47069F0A4ECB7E00E9453CEAE2F68
:100762000E948A3BE03011F0739A01C0739801C075
:10077200739837C0E530A0E0FA07C1F4E091900029
:10078200EF7CE0939000E091BA09E47069F0A6EE84
:10079200B7E00E9453CEAE2F0E948A3BE03011F0A8
:1007A200749A01C0749801C074981BC0E630A0E02E
:1007B200FA07B9F4E0919000E37FE0939000E091B2
:1007C200C209E47069F0A8E0B8E00E9453CEAE2FEF
:1007D2000E948A3BE03011F0759A01C0759801C001
:1007E2007598099119910895BA93AA9326970E9430
:1007F2005CCCE0918C09E17021F0E0918C09E2700F
:1008020009F4CCC1AC85BD85EC91E295E1703E2F37
:10081200303041F011960E94CECDEE83FF8368877F
:10082200798708C0AC85BD851196ED91FC91119731
:10083200EA87FB8710E0173008F0B0C1A2E9B9E0FF
:10084200E12FF0E00E94D8CCAE0FBF1FEC91E17017
:1008520009F4A2C1A2E9B9E0E12FF0E00E94D8CCEC
:10086200AE0FBF1FEC91E07409F4C5C03030B1F097
:10087200ABE3B7E0E12FF0E0BD01A2E2B0E00E94FD
:1008820011CDDB01AE0FBF1F18960E944BCEAE8179
:10089200BF81888599850E9409CD13C0ABE3B7E07B
:1008A200E12FF0E0BD01A2E2B0E00E9411CDDB0138
:1008B200AE0FBF1F18960E944FCEAA85BB850E941D
:1008C200F7CC2E2F203009F496C0ABE3B7E0E12F2E
:1008D200F0E0BD01A2E2B0E00E9411CDDB01AE0F5B
:1008E200BF1F1C960E9453CEEF700E2F013010F0E6
:1008F200083008F046C0AC85BD851596E02FF0E0C3
:100902003197AE0FBF1F4C915527542F4427ABE3AD
:10091200B7E0E12FF0E0BD01A2E2B0E00E9411CD0C
:10092200DB01AE0FBF1F1C960E9453CEE295EF7003
:100932000E2F013010F0083008F022C0AC85BD85C2
:100942001596E02FF0E03197AE0FBF1FEC91F0E06B
:100952004E2B5F2BA2E9B9E0E12FF0E00E94D8CC48
:10096200EA0FFB1F43835483A2E9B9E0E12FF0E0D1
:100972000E94D8CCAE0FBF1F1296E0915E04EC939A
:100982003AC0ABE3B7E0E12FF0E0BD01A2E2B0E094
:100992000E9411CDDB01AE0FBF1F1C960E9453CEE9
:1009A200E295EF700E2F013010F0083008F023C0EE
:1009B200A2E9B9E0E12FF0E00E94D8CCEA0FFB1FD8
:1009C20033960F01AC85BD851596E02FF0E0319787
:1009D200AE0FBF1FEC91D001F0E0ED93FC93A2E9C2
:1009E200B9E0E12FF0E00E94D8CCAE0FBF1F129603
:1009F200E0915E04EC93A2E9B9E0E12FF0E00E94FD
:100A0200D8CCAE0FBF1FEC91E07809F4C5C03030EE
:100A1200B1F0ABE3B7E0E12FF0E0BD01A2E2B0E05C
:100A22000E9411CDDB01AE0FBF1F53960E944BCE29
:100A3200AE81BF81888599850E9409CD13C0ABE341
:100A4200B7E0E12FF0E0BD01A2E2B0E00E9411CDDB
:100A5200DB01AE0FBF1F53960E944FCEAA85BB8506
:100A62000E94F7CC2E2F203009F496C0ABE3B7E0FA
:100A7200E12FF0E0BD01A2E2B0E00E9411CDDB0166
:100A8200AE0FBF1F57960E9453CEEF700E2F01304C
:100A920010F0083008F046C0AC85BD851596E02FF1
:100AA200F0E03197AE0FBF1F4C915527542F4427CA
:100AB200ABE3B7E0E12FF0E0BD01A2E2B0E00E94BB
:100AC20011CDDB01AE0FBF1F57960E9453CEE295A8
:100AD200EF700E2F013010F0083008F022C0AC8504
:100AE200BD851596E02FF0E03197AE0FBF1FEC9158
:100AF200F0E04E2B5F2BA2E9B9E0E12FF0E00E947B
:100B0200D8CCEA0FFB1F46835783A2E9B9E0E12F55
:100B1200F0E00E94D8CCAE0FBF1F1596E0915E04A4
:100B2200EC933AC0ABE3B7E0E12FF0E0BD01A2E203
:100B3200B0E00E9411CDDB01AE0FBF1F57960E949D
:100B420053CEE295EF700E2F013010F0083008F00E
:100B520023C0A2E9B9E0E12FF0E00E94D8CCEA0F6D
:100B6200FB1F36960F01AC85BD851596E02FF0E090
:100B72003197AE0FBF1FEC91D001F0E0ED93FC93E3
:100B8200A2E9B9E0E12FF0E00E94D8CCAE0FBF1F7E
:100B92001596E0915E04EC931F5F4DCE0E9463CCEC
:100BA2002E96089563970E945CCCE0918C09E170C7
:100BB20029F0E091EE08E770E13021F40E9463CC65
:100BC20069960895A7E2B1E00E9453CEE03011F495
:100BD200E0E007C0A7E2B1E00E9453CEAE2F0E9430
:100BE2008A3BEB8BA8E2B1E00E9453CEE03011F4D5
:100BF200E0E007C0A8E2B1E00E9453CEAE2F0E940F
:100C02008A3BEA8BA0E023FCA1E0E1E0EA27E8943A
:100C1200EE2309F0689423F810E0173010F00C94DA
:100C22002190A2E9B9E0E12FF0E00E94D8CCAE0F0A
:100C3200BF1FEC91E17011F40C941E90E12FFF277D
:100C420066277727E253FE4F6F4F6BBF06900C8AE1
:100C5200EC89A9E0EA9FF001E950F74FE081E295C3
:100C6200E770E98BA2E9B9E0E12FF0E00E94D8CC6D
:100C7200AE0FBF1FEC91E270A1F0ABE3B7E0E12F42
:100C8200F0E0BD01A2E2B0E00E9411CDDB01AE0FA7
:100C9200BF1F0E9453CEAE2F0E948A3BE03009F460
:100CA20042C0EB89E03089F0A5E4B1E0EC89F0E0E4
:100CB200BD01A7E0B0E00E9411CDDB01AE0FBF1F66
:100CC20012960E9453CEE07151F5EA89E03089F024
:100CD200A5E4B1E0EC89F0E0BD01A7E0B0E00E943C
:100CE20011CDDB01AE0FBF1F12960E9453CEE072F0
:100CF200B1F4E091F408E03089F0A5E4B1E0EC89C8
:100D0200F0E0BD01A7E0B0E00E9411CDDB01AE0F23
:100D1200BF1F12960E9453CEE07409F402C030E065
:100D220001C031E001C030E050E0303009F451C47C
:100D3200A2E9B9E0E12FF0E00E94D8CCAE0FBF1FCC
:100D4200EC91E87009F4BDC0ABE3B7E0E12FF0E04D
:100D5200BD01A2E2B0E00E9411CDDB01AE0FBF1FC8
:100D620012960E9453CEE88BA889A83B09F053C083
:100D7200E0917508F091760834960E94EACC0E2F25
:100D8200A6ECB1E00E9453CEEE8BA7ECB1E00E943C
:100D920053CEED8BAE89A017E8F50E1758F5A02FAC
:100DA200BB27EE89F0E0AE1BBF0BAE87BF87ABE37C
:100DB200B7E0E12FF0E0BD01A2E2B0E00E9411CD68
:100DC200DB01AE0FBF1F15960E9453CEF0E0AE8539
:100DD200BF850E9411CDEE87FF87AD89BB27EE89C3
:100DE200F0E00E94F5CDEA1BFB0BAE85BF850E94A9
:100DF20057CD0FC0ABE3B7E0E12FF0E0BD01A2E2B7
:100E0200B0E00E9411CDDB01AE0FBF1F15960E940C
:100E120053CE5E0F56C0A889A93B09F052C0E0919B
:100E22007708F091780834960E94EACC0E2FAAEC4B
:100E3200B1E00E9453CEEE8BABECB1E00E9453CEF8
:100E4200ED8BAE89A017E8F50E1758F5A02FBB273A
:100E5200EE89F0E0AE1BBF0BAE87BF87ABE3B7E016
:100E6200E12FF0E0BD01A2E2B0E00E9411CDDB0172
:100E7200AE0FBF1F15960E9453CEF0E0AE85BF8520
:100E82000E9411CDEE87FF87AD89BB27EE89F0E086
:100E92000E94F5CDEA1BFB0BAE85BF850E9457CDA4
:100EA2000FC0ABE3B7E0E12FF0E0BD01A2E2B0E09A
:100EB2000E9411CDDB01AE0FBF1F15960E9453CECB
:100EC2005E0FA2E9B9E0E12FF0E00E94D8CCAE0FAC
:100ED200BF1FEC91E07109F4C0C0ABE3B7E0E12FB2
:100EE200F0E0BD01A2E2B0E00E9411CDDB01AE0F45
:100EF200BF1F13960E9453CEE88BA889A83B09F026
:100F020053C0E0917508F091760834960E94EACCBD
:100F12000E2FA6ECB1E00E9453CEEE8BA7ECB1E00F
:100F22000E9453CEED8BAE89A017E8F50E1758F547
:100F3200A02FBB27EE89F0E0AE1BBF0BAE87BF87A9
:100F4200ABE3B7E0E12FF0E0BD01A2E2B0E00E9426
:100F520011CDDB01AE0FBF1F16960E9453CEF0E0FB
:100F6200AE85BF850E9411CDEE87FF87AD89BB2775
:100F7200EE89F0E00E94F5CDEA1BFB0BAE85BF8542
:100F82000E9457CD0FC0ABE3B7E0E12FF0E0BD0107
:100F9200A2E2B0E00E9411CDDB01AE0FBF1F169698
:100FA2000E9453CE5E0F56C0A889A93B09F052C0D9
:100FB200E0917708F091780834960E94EACC0E2FDF
:100FC200AAECB1E00E9453CEEE8BABECB1E00E94F2
:100FD20053CEED8BAE89A017E8F50E1758F5A02F6A
:100FE200BB27EE89F0E0AE1BBF0BAE87BF87ABE33A
:100FF200B7E0E12FF0E0BD01A2E2B0E00E9411CD26
:10100200DB01AE0FBF1F16960E9453CEF0E0AE85F5
:10101200BF850E9411CDEE87FF87AD89BB27EE8980
:10102200F0E00E94F5CDEA1BFB0BAE85BF850E9466
:1010320057CD0FC0ABE3B7E0E12FF0E0BD01A2E274
:10104200B0E00E9411CDDB01AE0FBF1F16960E94C9
:1010520053CE5E0F553608F054E6A2E9B9E0E12F0F
:10106200F0E00E94D8CCAE0FBF1FEC91E07209F401
:10107200C0C0ABE3B7E0E12FF0E0BD01A2E2B0E017
:101082000E9411CDDB01AE0FBF1F14960E9453CEFA
:10109200E88BA889A83B09F053C0E0917508F0914C
:1010A200760834960E94EACC0E2FA6ECB1E00E949C
:1010B20053CEEE8BA7ECB1E00E9453CEED8BAE89FE
:1010C200A017E8F50E1758F5A02FBB27EE89F0E020
:1010D200AE1BBF0BAE87BF87ABE3B7E0E12FF0E0FB
:1010E200BD01A2E2B0E00E9411CDDB01AE0FBF1F35
:1010F20017960E9453CEF0E0AE85BF850E9411CDB7
:10110200EE87FF87AD89BB27EE89F0E00E94F5CD1F
:10111200EA1BFB0BAE85BF850E9457CD0FC0ABE328
:10112200B7E0E12FF0E0BD01A2E2B0E00E9411CDF4
:10113200DB01AE0FBF1F17960E9453CE5E0F56C043
:10114200A889A93B09F052C0E0917708F09178088C
:1011520034960E94EACC0E2FAAECB1E00E9453CE44
:10116200EE8BABECB1E00E9453CEED8BAE89A017B3
:10117200E8F50E1758F5A02FBB27EE89F0E0AE1B5D
:10118200BF0BAE87BF87ABE3B7E0E12FF0E0BD0155
:10119200A2E2B0E00E9411CDDB01AE0FBF1F179695
:1011A2000E9453CEF0E0AE85BF850E9411CDEE873E
:1011B200FF87AD89BB27EE89F0E00E94F5CDEA1BDF
:1011C200FB0BAE85BF850E9457CD0FC0ABE3B7E0E6
:1011D200E12FF0E0BD01A2E2B0E00E9411CDDB01FF
:1011E200AE0FBF1F17960E9453CE5E0F553608F002
:1011F20054E6A2E9B9E0E12FF0E00E94D8CCAE0FAC
:10120200BF1FEC91E07461F0A2E9B9E0E12FF0E0D8
:101212000E94D8CCAE0FBF1F1296AC91A13008F439
:1012220083C0A2E9B9E0E12FF0E00E94D8CCAE0F72
:10123200BF1F1296EC91E150EC93A2E9B9E0E12FC5
:10124200F0E00E94D8CCAE0FBF1F1296EC91E030B6
:1012520071F4A2E9B9E0E12FF0E00E94D8CCAE0F20
:10126200BF1F1396E0E0F0E0ED93FC935DC0A2E9AE
:10127200B9E0E12FF0E00E94D8CCAE0FBF1F139669
:10128200ED91FD91FF93EF93ABE3B7E0E12FF0E037
:10129200BD01A2E2B0E00E9411CDDB01AE0FBF1F83
:1012A2001D960E944FCEAF91BF91EA23FB23EE879A
:1012B200FF87ABE3B7E0E12FF0E0BD01A2E2B0E0CF
:1012C2000E9411CDDB01AE0FBF1F1F960E944BCEB5
:1012D200DF01CB01EE85FF85662777270E94ECCEE2
:1012E2000E9475CFEE83FF8368877987AE81BF81C5
:1012F20088859985E0E0F0E068EC72E40E9407D00E
:1013020009F008F401C00FC0EE81FF81688579857C
:10131200A0E0B0E080E09FE30E9426CF0E94B3CE1F
:101322005E0F553608F054E6A2E9B9E0E12FF0E08D
:101332000E94D8CCAE0FBF1FEC91E07861F0A2E919
:10134200B9E0E12FF0E00E94D8CCAE0FBF1F159696
:10135200AC91A13008F483C0A2E9B9E0E12FF0E03A
:101362000E94D8CCAE0FBF1F1596EC91E150EC93C2
:10137200A2E9B9E0E12FF0E00E94D8CCAE0FBF1F86
:101382001596EC91E03071F4A2E9B9E0E12FF0E0BA
:101392000E94D8CCAE0FBF1F1696E0E0F0E0ED93AE
:1013A200FC935DC0A2E9B9E0E12FF0E00E94D8CC45
:1013B200AE0FBF1F1696ED91FD91FF93EF93ABE336
:1013C200B7E0E12FF0E0BD01A2E2B0E00E9411CD52
:1013D200DB01AE0FBF1F58960E944FCEAF91BF9157
:1013E200EA23FB23EE87FF87ABE3B7E0E12FF0E0D0
:1013F200BD01A2E2B0E00E9411CDDB01AE0FBF1F22
:101402005A960E944BCEDF01CB01EE85FF856627FF
:1014120077270E94ECCE0E9475CFEE83FF83688708
:101422007987AE81BF8188859985E0E0F0E068EC3C
:1014320072E40E9407D009F008F401C00FC0EE81E7
:10144200FF8168857985A0E0B0E080E09FE30E949B
:1014520026CF0E94B3CE5E0F553608F054E6A2E9BD
:10146200B9E0E12FF0E00E94D8CCAE0FBF1FEC91A3
:10147200E072A1F0ABE3B7E0E12FF0E0BD01A2E240
:10148200B0E00E9411CDDB01AE0FBF1F14960E9487
:1014920053CEAE2F0E948A3BE03009F40EC0ABE37C
:1014A200B7E0E12FF0E0BD01A2E2B0E00E9411CD71
:1014B200DB01AE0FBF1F17965BC0A2E9B9E0E12FB7
:1014C200F0E00E94D8CCAE0FBF1FEC91E071A1F00A
:1014D200ABE3B7E0E12FF0E0BD01A2E2B0E00E9491
:1014E20011CDDB01AE0FBF1F13960E9453CEAE2F5C
:1014F2000E948A3BE03009F40EC0ABE3B7E0E12F73
:10150200F0E0BD01A2E2B0E00E9411CDDB01AE0F1E
:10151200BF1F16962DC0A2E9B9E0E12FF0E00E94AC
:10152200D8CCAE0FBF1FEC91E870A1F0ABE3B7E0EF
:10153200E12FF0E0BD01A2E2B0E00E9411CDDB019B
:10154200AE0FBF1F12960E9453CEAE2F0E948A3B4F
:10155200E03009F410C0ABE3B7E0E12FF0E0BD01E9
:10156200A2E2B0E00E9411CDDB01AE0FBF1F1596C3
:101572000E9453CE5E2F533608F054E6ABE3B7E039
:10158200E12FF0E0BD01A2E2B0E00E9411CDDB014B
:10159200AE0FBF1F5E960E9453CE4E2FABE3B7E055
:1015A200E12FF0E0BD01A2E2B0E00E9411CDDB012B
:1015B200AE0FBF1F5F960E9453CEE88F513010F0DE
:1015C200541708F002C0542F04C0E88D5E1708F0CB
:1015D200588D303041F0513030F0A989A03011F0EF
:1015E200A13009F401C01FC0A2E9B9E0E12FF0E087
:1015F2000E94D8CCAE0FBF1F1196E0E0EC93EC89AD
:10160200A9E0EA9FF001E550F74FA0E0A083EC8942
:10161200A9E0EA9FF001E750F74FDF01EC91E07F8C
:10162200EC93E2E0E98B550FA989A23019F0A330BF
:1016320009F0EDC0A2E9B9E0E12FF0E00E94D8CCB8
:10164200AE0FBF1F11962C91251708F06DC0ABE3AA
:10165200B7E0E12FF0E0BD01A2E2B0E00E9411CDBF
:10166200DB01AE0FBF1F90960E9453CEEF8BAF8966
:10167200A13008F458C0AF3190F123FE18C0EF89B1
:10168200F0E0A0E9B1E00E946ACD0E2F023008F02E
:101692000150A22FBB27EE27A00FBE1FE52FF0E0BF
:1016A200AE17BF071CF4E02FE20F5E2F17C0AF8901
:1016B200ECE3EA17E1E008F4EE270E2EE22FF0E069
:1016C2003296DF01E52FF0E00E94FDCCE02119F017
:1016D200E22FEE5F02C0E22FEF5F5E2F24C0EF89A0
:1016E200F0E0A8ECB0E00E946ACD0E2F023370F455
:1016F200A22FBB27EE27A00FBE1FE52FF0E0AE17EB
:10170200BF071CF4E02FE20F5E2F0DC0A22FBB27F4
:10171200EE27A00FBE1FE52FF0E0AE17BF0718F4AB
:10172200E02FE20F5E2F70C0521708F06DC0ABE3DE
:10173200B7E0E12FF0E0BD01A2E2B0E00E9411CDDE
:10174200DB01AE0FBF1F91960E9453CEEF8BAF8984
:10175200A13008F459C0AF3190F123FE19C0EF89CE
:10176200F0E0A0E9B1E00E946ACD0E2F023008F04D
:101772000150A52FBB27E02FF0E0EA0FFB1FA22F9D
:10178200B0E0EA17FB071CF4E22FE01B5E2F16C045
:10179200AF89ECE3EA17E1E008F4EE270E2EE52F1D
:1017A200F0E03296A22FB0E00E9403CDE02119F0C2
:1017B200E22FE25002C0E22FE1505E2F25C0EF89F6
:1017C200F0E0A8ECB0E00E946ACD0E2F023370F474
:1017D200A52FBB27F0E0EA0FFB1FA22FB0E0EA170C
:1017E200FB071CF4E22FE01B5E2F0EC0A52FBB27C8
:1017F200E02FF0E0EA0FFB1FA22FB0E0EA17FB0791
:1018020018F4E22FE01B5E2F593C08F058ECA2E9D5
:10181200B9E0E12FF0E00E94D8CCEA0FFB1F518320
:10182200503009F430E0303029F4A989A03011F0A9
:10183200A13009F416C0EC89A9E0EA9FF001E75053
:10184200F74FDF01EC91E07FEC93EC89A9E0EA9F8E
:10185200F001E950F74FDF01EC91EB7FEC93E0E010
:10186200E98BA989A43011F0A53009F450E0E12FE9
:10187200F0E0309709F054C05030B1F4E0E0E0936A
:10188200B000E0919209E47069F0ACE3B7E00E9425
:1018920053CEAE2F0E948A3BE03011F02C9A01C049
:1018A2002C9801C02C983BC0573CB0F0E0E0E0938C
:1018B200B000E0919209E47069F0ACE3B7E00E94F5
:1018C20053CEAE2F0E948A3BE03011F02C9801C01B
:1018D2002C9A01C02C9A23C0E0919209E47091F0F5
:1018E200ACE3B7E00E9453CEAE2F0E948A3BE030B9
:1018F20021F0E0918D09E06102C0E0918D09E09351
:10190200B00004C0E0918D09E093B000F52FE0E053
:10191200DF01E8ECF0E00E9457CDE093B3002FC363
:10192200E130A0E0FA0709F083C05030C1F4E09141
:101932008000EF73E0938000E0919A09E47069F00F
:10194200AEE5B7E00E9453CEAE2F0E948A3BE03054
:1019520011F02D9A01C02D9801C02D9868C0583CF5
:10196200C0F0E0918000EF73E0938000E0919A096B
:10197200E47069F0AEE5B7E00E9453CEAE2F0E944C
:101982008A3BE03011F02D9801C02D9A01C02D9AAA
:101992004EC0E0918E09F0918F0966277727EA877A
:1019A200FB876C877D87E52FF0E0AA85BB858C8558
:1019B2009D856F2F660F660B762F0E9419CDEA87E1
:1019C200FB876C877D87AA85BB858C859D85E8EC26
:1019D200F0E060E070E00E946FCDEE87FF87E0915B
:1019E2008E09F0918F09AE85BF85EA17FB0710F4C7
:1019F200EE87FF87EF85E0938900EE85E09388000C
:101A0200E0918000E068E0938000AEE5B7E00E94DC
:101A120053CEAE2F0E948A3BE03021F0E09180004D
:101A2200E06403C0E0918000EB7FE0938000A7C2F6
:101A3200E230A0E0FA0709F083C05030C1F4E0912F
:101A42008000EF7CE0938000E091A209E47069F0ED
:101A5200A0E8B7E00E9453CEAE2F0E948A3BE0304E
:101A620011F02E9A01C02E9801C02E9868C0583CE1
:101A7200C0F0E0918000EF7CE0938000E091A20949
:101A8200E47069F0A0E8B7E00E9453CEAE2F0E9446
:101A92008A3BE03011F02E9801C02E9A01C02E9A96
:101AA2004EC0E0918E09F0918F0966277727EA8769
:101AB200FB876C877D87E52FF0E0AA85BB858C8547
:101AC2009D856F2F660F660B762F0E9419CDEA87D0
:101AD200FB876C877D87AA85BB858C859D85E8EC15
:101AE200F0E060E070E00E946FCDEE87FF87E0914A
:101AF2008E09F0918F09AE85BF85EA17FB0710F4B6
:101B0200EE87FF87EF85E0938B00EE85E0938A00F6
:101B1200E0918000E062E0938000A0E8B7E00E94DC
:101B220053CEAE2F0E948A3BE03021F0E09180003C
:101B3200E06103C0E0918000EF7EE09380001FC26D
:101B4200E330A0E0FA0709F083C05030C1F4E0911D
:101B52008000E37FE0938000E091AA09E47069F0DD
:101B6200A2EAB7E00E9453CEAE2F0E948A3BE03039
:101B720011F02F9A01C02F9801C02F9868C0583CCD
:101B8200C0F0E0918000E37FE0938000E091AA0939
:101B9200E47069F0A2EAB7E00E9453CEAE2F0E9431
:101BA2008A3BE03011F02F9801C02F9A01C02F9A82
:101BB2004EC0E0918E09F0918F0966277727EA8758
:101BC200FB876C877D87E52FF0E0AA85BB858C8536
:101BD2009D856F2F660F660B762F0E9419CDEA87BF
:101BE200FB876C877D87AA85BB858C859D85E8EC04
:101BF200F0E060E070E00E946FCDEE87FF87E09139
